:10000000004000202570000065700000677000004F
:1000100000000000000000000000000000000000E0
:1000200000000000000000000000000069700000F7
:1000300000000000000000006B7000006D70000008
:100040006F700000ED510000A17400006F7000009F
:100050006F700000000000006F7000006F70000003
:100060006F70000071770000553100006F70000064
:100070006F7000006F7000006F7000006F70000004
:100080006F700000097900006F7000006F70000051
:100090006F7000006F7000006F7000006F700000E4
:1000A0006F7000006F700000000000000000000092
:1000B0000000000000000000000000000000000040
:1000C00010B5064C2378002B07D1054B002B02D02E
:1000D000044800E000BF0123237010BD600200202F
:1000E0000000000030E30000044B10B5002B03D0EB
:1000F0000349044800E000BF10BDC04600000000F6
:100100006402002030E30000164B002B00D1144B9A
:100110009D46402292029A1A924600218B460F4633
:100120001348144A121A0BF097F90F4B002B00D00A
:1001300098470E4B002B00D0984700200021040068
:100140000D000D48002802D00C4800E000BF0BF065
:1001500043F92000290007F0C1F90BF017F9C04658
:100160000000080000400020000000000000000027
:1001700060020020B42F00200000000000000000FA
:1001800002000120104011D1042A0ED91368180969
:1001900080B2002809D001388000031D11180979A8
:1001A000002902D001309842F8D170470020FCE7C6
:1001B0000378002B03D05AB2002A01DB01307047CC
:1001C0003F229343C03B59424B41C01803789343AD
:1001D000802BF4D10130F9E710B500240378002B0F
:1001E00001D1200010BDFFF7E3FF0134F6E770B541
:1001F000002204000D00411C092003F0C7FA00286A
:1002000006D001236200134343600023A34200DBB6
:1002100070BD9A00A958821891600133F6E770B555
:10022000012803DC1C2001F047F870BD01230D6894
:1002300011201D42F7D04868184206D1042804D97D
:100240000F2302681340042B01D00E20EBE703F0CC
:10025000FBF86D100400002D03DDFFF7BDFFA84281
:1002600006DA1220DFE72000FFF7A2FF0400013DBD
:10027000012DF8D120787F2809DDDF280BDCF82359
:100280003F22DB00800118406378134018430123AC
:1002900040001843C9E7EF280BDCFC226378120109
:1002A0009B0113403F220007000C0343A07810403D
:1002B000ECE7F72812DCFC22637892021B03134060
:1002C000E0228004520310403F221843E378134099
:1002D000FC220343A07812018001E8E7012040429C
:1002E000D5E7F8B54D680F00EB0706D4042D04D907
:1002F0000F232E683340092B03D00B2000F0DCFFC6
:10030000F8BD6B683609B6B25C10731EA3420FD8F5
:100310000321200008F05CFF6421642803DC010055
:10032000032800DA03212800891903F061FA050087
:100330002B6800201B099BB2013B9C42E0D23A682B
:10034000A31C9B005A510123013464001C436C60C0
:10035000D6E7F0B585B0012803DC1C2000F0ACFF27
:100360002CE001274B683A000093022806D08B68E6
:100370003B4203D05F10002F00DC17000124009BDC
:10038000234200D0B2E0042B00D8AFE01B680D6818
:100390000F2619003140042925D1254205D1042D0D
:1003A00003D92B681E40042E01D00E20D6E70098FA
:1003B000FFF7E6FEB84203DA0120404205B0F0BD87
:1003C000009803F041F80600280003F03DF8010012
:1003D000781E30180BF0F6FB0028EDD0801B0130A2
:1003E00040002043EAE709293DD1009B5B685B1090
:1003F00001939F42E0DC25422CD1042D2AD92B68A1
:100400003340042B26D1280003F01EF803960290F7
:100410007E1C009AB300D058854201D17800E0E7F5
:1004200020420ED104280CD90368039A1340042BF0
:1004300007D103F009F8010002980BF08DFB0028AA
:10044000ECD0019B37009E42E2DDB5E71F00019B27
:100450009F42B1DC7B1C00999A008A58AA42F5D1D0
:1004600078000124BDE7032940D11A0992B25B0F3D
:1004700092000B40D31A01939F429DDC254229D163
:10048000042D27D92A681640032E19D1100980B2ED
:10049000520F800032402C1D801A019B26181B1A17
:1004A0000193009B781E0433019A904200DD83E79C
:1004B00022001918B2420FD316D101304000D0E704
:1004C000042E07D1280002F0BFFF04002800FFF728
:1004D00057FEE2E70F2041E70D78AC461578AC45B2
:1004E00002D101310132E5E70130DDE7212035E7B6
:1004F00010B502F08DFF43000120184310BD00002D
:10050000C30711D404280FD90F2302681340032B0B
:100510000AD119400133591AC0234907DB05194094
:10052000024B1A40114301607047C046FFFFFF9F16
:10053000F7B507000E001C20012F06DD4C680123D3
:1005400022001A40009203D10D2000F0B5FE53E0C6
:10055000022F02D08A681A42F6D0012335681D4264
:1005600000D0A9E0042D00D8A6E01C41002C00DC3E
:100570001C000F2029680840092828D16B685B10EF
:100580000093022F05D0B368009A5B109A4200DDF9
:100590000093009B01221D1B0135EB43DB171D401F
:1005A000691C092003F0F2F8071E09D001236D0031
:1005B0001D4303003268083345600099A14201DA07
:1005C0003800FEBD0134A100515802C3F5E70428EC
:1005D00045D1280002F038FFFFF7FEFD0190022F01
:1005E00004D0B3685B10984200DD0193019BA342E5
:1005F00004DA002003F03CF90700E1E7280002F0EC
:1006000023FF0700009BA34221DB2800009702F094
:100610001BFF05003800FFF7CBFD019B01340700ED
:10062000A342F7DA009BC41A200003F021F9071E49
:10063000C6D002F009FF0190306802F005FF2200E9
:10064000009B591B411801980AF0EAFEB8E73800F0
:10065000FFF7AEFD009B070001330093D2E70328AC
:100660002AD10B099BB2490F9B000140591A022F56
:1006700004D0B2685210914200DD1100A14205DAA7
:1006800000220320110003F081F8B5E703200E1BC0
:10069000331DD9170140C9188910002203F076F8DC
:1006A000071E00D18CE7013631000334FFF728FF25
:1006B000381D29193200C7E7212046E7F8B5002880
:1006C00005DC1C2000F0F8FD05002800F8BD01261F
:1006D0000C6826400FD06410E343DB171C40E11C7C
:1006E00089100022032003F051F8051EEDD02100EF
:1006F000FFF706FFE9E7042C01D80025E5E70F2303
:1007000022681340042B1BD12000FFF739FDC31CC6
:1007100007000320D9170140C9188910320003F0DF
:1007200035F8051ED1D03900FFF7EAFE200002F0AF
:100730008BFE2B1D01003A0018000AF071FEC4E781
:10074000092BDAD10320636832005F10FB1CD91734
:100750000140C918891003F019F8051ECDD03900E1
:10076000FFF7CEFEFF20BE42AFDA0122B300E3184E
:100770009B68134208D01341FF2B00DD0300D943CF
:10078000C917AA190B4013710136ECE710B57F2980
:1007900002DC0170013010BD1A4B99420CDC402381
:1007A0008A115B42134303703F230B40802149426F
:1007B000194341700230EEE7134B994210DC2023BD
:1007C0000A135B4213433F24802203708B11524271
:1007D0002340214013430A43437082700330DAE719
:1007E0000A4B9942D7DCF0230370603B4370113B06
:1007F0008A11FF3B1A4382703F2211401943C17096
:100800000430C8E7FF070000FFFF0000FF0F0100F2
:10081000F0B50D0085B0002803DC1C2000F04CFD75
:100820000DE009680122080010400AD002AC114115
:100830002000FFF7ABFF011B200003F025F80400A8
:100840001AE004293FD90F230C682340092B3AD121
:100850004B685B10019303239C46019B9A420EDD7B
:1008600003F006F8041E07D02E68012502F0ECFD07
:100870002F00019B9D421DDD200005B0F0BD01321F
:100880009300CC580123234001D10D20C6E764100A
:100890007F2C0DDD0D4E0223B44209DD0C4E634664
:1008A000B44205DD00270B4EE30FA6427B419B00BF
:1008B000C018D2E70135AB00F1583942E5D04910F4
:1008C000FFF764FFD5E72120A8E7C046FF07000037
:1008D000FFFF0000FF0F010010B5040001200840D9
:1008E00010D104290DD90F230A681340042B08D115
:1008F000080002F0A9FD010020000BF02DF9434291
:10090000584110BD0020FCE7F7B50F00012803DCBB
:100910001C2000F0D1FCFEBD01264D682E4006D102
:10092000042D04D90F222B681A40092A01D00B206C
:10093000EFE76A681B099BB25410A34200D85C1E03
:1009400039681E48FFF7C8FF01230190002813D122
:1009500039681B48FFF7C0FF002811D0002C0DD0CC
:100960000123621C013C9C409200535123436B6065
:1009700004E00136B200AB50B442FADA0020CAE714
:100980003B680D20DA07C4D55B10002B11DD9C42BB
:100990000FDB9B00A200291DEB1889180433994234
:1009A00009D10123013C9C40AA181C4353606C6090
:1009B000E4E71220ADE758681860EFE7EBCA0000E3
:1009C000EFCA0000002310B50C000B70C30705D55B
:1009D0000D49421020000BF083F808E00B49002875
:1009E00002D0042804D10A4920000BF099F810BD68
:1009F0000428FCD90F2302681340042BF7D102F01E
:100A000023FD04490200E5E7E8D40000F4CA000031
:100A1000FACA0000FFCA0000F0B593B006000291C8
:100A20001C20012E1DDD029B01251B681C002C4093
:100A300000D0ADE0042B00D8E6E01A680F231A407E
:100A4000092A4AD10394039A029992008A581700FE
:100A50002F4005D1042A03D910681840092806D070
:100A6000222000F029FC0190019813B0F0BD5268DB
:100A70005210A418039A013203929642E3D1611CEA
:100A8000012202F083FE0190002802D1002301938D
:100A9000EAE7019B6400190025435D600831029A72
:100AA000BB00D05802684368120992B25B109A42A8
:100AB00000D8531E0022934209DCDA43D2171340B8
:100AC0009B00C918039B01379F42E8DBCCE79400E9
:100AD0000519AD6801320D51EDE72700032A59D100
:100AE0000193029ABB00D3582B42B9D1042BB7D93A
:100AF000186801990140032939D1020992B2430FC4
:100B000092000B40D31A1C190137BE42E9D10320D1
:100B1000E31CD9170140C9188910002202F036FEE3
:100B200001900028B2D000252100FFF7E9FC019BCD
:100B30001E1D029AAB00D45801231C421FD1042C65
:100B40001DD90F2123681940032918D1180980B233
:100B50005B0F80000B40C01A0023834213DBC343AA
:100B6000DB17184001353618BD42E2DB7CE704296B
:100B700000D075E71800FFF703FB2418C4E7200036
:100B8000FFF7FEFAE8E7E2181279F2540133E4E7DE
:100B900000273C000F25029ABB00D35801221342C4
:100BA00034D1042B32D9186801002940042935D1E9
:100BB0001800FFF7E5FA24180137BE42EBD12000F8
:100BC00002F056FE0190002800D15FE7029FB600B8
:100BD000BB19041D029301233D681D4229D1042D38
:100BE00027D90F262B681E40042E37D12800FFF787
:100BF000C7FA0600280002F027FC0100200032009E
:100C00000AF00EFCA41922E02700C3E7180005A98A
:100C1000FFF7D8FE05A80AF0A9FFCCE7032900D00A
:100C20001EE7020992B2430F92000B40D31A1C191F
:100C3000C2E705A92800FFF7C5FE05A80AF096FF40
:100C400005A90500020020000AF0EAFB6419029BD6
:100C50000437BB42BFD10023237005E7032EF6D132
:100C60001A0992B25B0F92001E40961B291DC5E720
:100C7000F0B50D0095B0002806DC1C2000F01CFB30
:100C80000400200015B0F0BD0C68012123000B40CA
:100C9000009306D1042C04D922680F331A40092A84
:100CA00001D00B20EAE7626852100392002A03DCAD
:100CB000009802F0DDFDE3E73F4A019201280BD0E6
:100CC0006868084208D1042806D902681340042B3A
:100CD00002D102F0B9FB019001980AF047FF06002B
:100CE0000F27039B0834013B04935E43039B029050
:100CF0009B001B19059301232068184251D1042839
:100D00004FD903683B40042B52D1FFF739FA059BBA
:100D100004343618A342EED1300002F0A9FD041EBF
:100D2000AFD02B680593029B002B03D0686802F0BC
:100D30008BFB0190200002F087FB0500009B059AC9
:100D40009B00D3189F68380002F07EFB0123060049
:100D50001F4201D1042F04D807A93800FFF732FE43
:100D600007AE30000AF002FF070002003100280041
:100D70000AF056FB029BED19002B0AD0049B009A47
:100D8000934206DD2800029A01990AF049FB029B72
:100D9000ED18009B01330093009A039B9342CDD141
:100DA0006FE707A9FFF70EFE07A80AF0DFFEAEE720
:100DB00002F04AFBF9E7C0468BCF000010B50024D3
:100DC000A04207DD0B6801341C4003D05C10E343F4
:100DD000DB171C40611C0122092002F0D7FC00280F
:100DE00003D0012364001C43446010BD0A6870B541
:100DF00010000125284034D1042A32D90F24136869
:100E000049681C40092C17D154681B099BB22C411E
:100E1000A34200D85C1E844205DC022001339842C4
:100E200006DB00200FE085005519A9600130F2E7CC
:100E3000840011510130F2E7032C12D1294203D171
:100E4000132000F039FA70BD4910FF29F8D81B09AA
:100E50009BB204329B00D3189342E2D91170013245
:100E6000FAE70B2000F028FADBE700000123F7B5D2
:100E700000254E680F0033400093AB420ED11D0099
:100E8000042E0BD90F2233681A40092A10D1726838
:100E90001B099BB25510AB4200D85D1E3968CB07C9
:100EA00017D54C10002C01DDA5421DDA122032E0CE
:100EB000042A04D13000FFF763F90500EEE7009D36
:100EC000032AEBD11D09ADB25B0FAD001340ED1A43
:100ED000E4E72E48FFF700FD002814D00AF09CFD3F
:100EE000290008F05BFA4C1C009B002B4CD1042E0F
:100EF0004AD932680F331340092B10D10134A400B2
:100F0000A4592000FEBD39682148FFF7E5FC2C00FC
:100F10000028E9D1113000F0CFF90400F1E7042BEB
:100F20002AD1300002F090FA0500FFF755F9A042EF
:100F3000BCDB012C1ADC300002F086FA009028009D
:100F4000FFF736F9461B300002F092FC041ED8D0A1
:100F500002F07AFA0190786802F076FA009B32008B
:100F6000E91A411801980AF05BFACAE72800FFF76E
:100F70001FF9013C0500DCE7032B05D13419E478A7
:100F8000023B64001C43BCE70B20C4E7E4CA00003A
:100F9000EFCA0000F7B54D680F002A0001210A4092
:100FA0002FD1042D2DD90F242B68BE681C40092C8D
:100FB00014D169681B099BB24C100192A34200D85E
:100FC0005C1E39682A48FFF787FC00282DD00F23C4
:100FD0002A681340092B1DD1012317E0032C10D1DF
:100FE0000E4203D1132000F067F9FEBD721001928A
:100FF000FF2AF7D81A0992B25B0F92001C40141B0B
:10100000DFE70B20EFE701339A00AE509C42FADA9B
:101010000020EAE7032BFBD12B0001335A1BA2422D
:10102000F6DC6A461279DA70F7E73968CB0706D53D
:101030004910002901DD8C4209DA1220D3E70D485E
:10104000FFF74AFC2100002801D11130CBE70F2324
:101050002A681340092B03D1013189004E51D7E78B
:10106000032BD5D16B461B796D18EB70D0E7C046CA
:10107000EBCA0000EFCA000010B501240868204246
:101080001AD1042818D90F2102681140092901D169
:10109000406810BD032908D113099BB2500F9B0073
:1010A0000840181A40002043F3E7042904D102F055
:1010B000CBF9FFF791F8F5E70B2000F0FDF8E8E732
:1010C00010B5034A0B21034804F088F910BDC0464F
:1010D0008CCA000084CA00000020704704207047BA
:1010E0000120704710B5002002F0C2FB10BD0020A7
:1010F0007047002070470020704700207047002094
:1011000070470020704700207047002070470000A3
:1011100010B5034A0C21034804F060F910BDC04625
:1011200074CB0000D4CB000010B50124044002D0E1
:101130004410200010BD042810D90F23026813406A
:10114000042B07D102F080F921000A220AF0D6FD13
:101150000400EEE7032B01D10430F5E70D22014B2B
:101160001A70E6E7A0020020012210B5024018D153
:10117000042802D903681A0992B201230B4012D144
:10118000042902D90B681B099BB20024934206D1A3
:1011900004309B000431C318984206D30124200078
:1011A00010BD0022E9E70023EFE704780A78002C5D
:1011B00001D1002AF2D0013001319442ECD0002458
:1011C000EDE70000F7B50700009101933049314B7E
:1011D000002A02D002220A70013A00261A601B6817
:1011E000CE54BE4200DBF7BD009AB300D058294B65
:1011F000274D1C68C8239B0065191C1B012318423E
:1012000006D0254A4310210028000AF037FC09E0E7
:10121000224A002802D004281BD1214A210028009C
:101220000AF02CFC1A4C20000AF0A0FC194A019B81
:101230001060002B0BD07B1EB34208DD194B984287
:1012400005D8431C1360202222540022E2540136A8
:10125000C7E7042819D90F2301680B40042B04D1D8
:1012600002F0F2F8104A0300CDE7092B03D14368DE
:101270000E4A5B10C7E7032B08D10A0992B2490F47
:1012800092000B40D31A0A4ABDE70123094ABAE784
:10129000A1020020C4050020E8D40000F4CA000028
:1012A000FACA00001F03000013DB000044CE000058
:1012B00053CE00005ECE0000014B18700020704736
:1012C000A002002070B501F033FE094C0100251D7D
:1012D0001F2228000AF062FC28000AF047FC0423C1
:1012E00004308008000118432060200070BDC04613
:1012F0007C020020C368F0B59D00836889B05D1949
:101300000300183306930369069A9F00069B029018
:10131000DF19436901939B00D3180393CD4B1B78CE
:10132000002B26D17F222B68CB491C1213409B0037
:101330005B58043501929F46029B587804F06AFC82
:101340000023029A137027E0C24B1B78002B10D1A8
:101350002B68019A1C121340BF4A9B009B5804350E
:10136000E9E7069B3A1DD11ABA4BD82928DD1A2283
:101370001A70029BB74C9B6821780193EA1A029B72
:1013800092109B7812021A43029B587804F04AFC90
:101390000023029A23701370029B069A9B680193A4
:1013A000ED1A029BAD10DD60069BFE1A029BB61083
:1013B0001E61039B9B1A029A9B10536109B0F0BDFA
:1013C0001B783C60002B01D01700D2E72B680199F5
:1013D0001C120B40A0499B005B5817000435AAE77C
:1013E000069B3A1DD11A9B4BD82902DD1A221A708E
:1013F000BFE728681B78291D3860002B02D0170032
:101400000D00B6E76B6801991C120B4092499B00D6
:101410005B58170008358EE7069B3A1DD11A8D4B95
:10142000D82902DD1A221A70A3E7A4001B782C1910
:101430003C60002B01D017009BE72B6801991C1220
:101440000B4085499B005B581700043573E7069BEA
:101450003A1DD11A7F4BD82902DD1A221A7088E76B
:101460007E49A40061581B783960002B01D0170019
:101470007FE72B6801991C120B4077499B005B5852
:101480001700043557E7043F744B3A68A400E25054
:10149000704B1B78002B00D06BE72B68019A1C1255
:1014A00013406D4A9B009B58043544E76B4BA400E6
:1014B000E058FFF739FE043F06003868FFF734FEB6
:1014C00036180120654B76000643E650614B1B78C9
:1014D000002B00D04DE72B68019A1C1213405E4A86
:1014E0009B009B58043526E7069B3A1DD11A594BA1
:1014F000D82902DD1A221A703BE70698039C0121C5
:10150000A04202D221000C3909681B783960002BF7
:1015100001D017002DE72B6801991C120B404E4992
:101520009B005B581700043505E7069B3A1DD11A4E
:10153000484BD82902DD1A221A701AE70699039837
:1015400081420FD203000C3B1B6845495B106418B5
:10155000E41AA40023583B603E4B1B78002B05D0B7
:10156000170006E7182119700023F4E72B6801998A
:101570001C120B4038499B005B5817000435DAE613
:10158000069B039A934219D213000C3B1B68344A02
:10159000043FA4185B10E31A039A39689B00995022
:1015A0002C4B1B78002B00D0E3E62B68019A1C1211
:1015B0001340294A9B009B580435BCE61822254B52
:1015C0001A70EDE7069B039A93422DD2244B3E1FDF
:1015D000E31814000C3C04932368049A5B10D31A9C
:1015E000039A9B009858FFF79FFD07903068FFF71C
:1015F0009BFD2468049B64101C1B079BA4001F1800
:1016000001207F00039B0743E7503700114B1B78F5
:10161000002B00D0ADE62B68019A1C1213400E4A35
:101620009B009B58043586E618220A4B1A70EDE79A
:10163000069B3A1DD11A074BD82902DD1A221A70CF
:1016400097E60399A40061581B783960002B09D0F4
:1016500017008EE6A002002044CC0000802D002060
:10166000FDFFFF3F2B6801991C120B40D9499B00DD
:101670005B58170004355EE6043F039B3A68A400FC
:10168000E250D54B1B78002B00D072E62B68019AF4
:101690001C121340CF4A9B009B5804354BE6039B1A
:1016A000A4001C192368043F38685E10FFF73CFD56
:1016B00036180120C84B76001B7806432660002BA5
:1016C00000D056E62B68019A1C121340C14A9B00B9
:1016D0009B5804352FE6069BA4003F1BBE4CBB4223
:1016E0000CD82378002B00D043E62B68019A1C12FB
:1016F0001340B84A9B009B5804351CE6B74801F0DC
:1017000093FE2378002B00D033E62B68019A1C123D
:101710001340B04A9B009B5804350CE6A300ED181B
:10172000002C00DA38E6AC4B1B78002B00D020E60A
:101730002B68019A1C121340A64A9B009B58043543
:10174000F9E5043F3B68042B04D1A300ED18002CFD
:1017500000DA21E6A04B1B78002B00D009E62B68AD
:10176000019A1C1213409B4A9B009B580435E2E5EA
:10177000043F3B68042B04D0A300ED18002C00DAD2
:101780000AE6954B1B78002B00D0F2E52B68019AF6
:101790001C1213408F4A9B009B580435CBE53A1F1F
:1017A00013685B10013B06D401215B00A4000B43CE
:1017B0002D191360F0E5884B17001B78002B00D023
:1017C000D7E52B68019A1C121340824A9B009B5854
:1017D0000435B0E53A00069B0C32D31AD82B03DD52
:1017E0001A227D4B1A70C4E5FF2361005B0019408B
:1017F000FE3BFF3B19433960029906988968241221
:1018000004916D1A0299AD1089782D020D43039948
:101810009D40091A891099401D430B43BB60029BF0
:101820007D609C70E4B26E4BE4000392E358029A30
:101830009360694A1278002A03D008331D00039F81
:1018400097E51D00019A9B680C351C121340614AF4
:101850009B009B58039F6EE53B1F1C68039A069BE9
:1018600093422DD10A20E3070CD4042C13D90F2363
:1018700022681340042B11D1200001F0E5FD0AF08D
:1018800075F90630643003F0E3FD00280FD1043D04
:10189000069B039380E50720042CF3D02000431E11
:1018A0009841FA234042FF3318400730EAE7029B91
:1018B0002100587804F0C8F90023029A1370E7E772
:1018C000039B039A0C3B1B6802995B109B00D31A85
:1018D0000C3B1C601F1D1300083B1B685A108A70CC
:1018E000D2B23F49D2005B0055589B0A029A9B0036
:1018F0009560ED18039B069A043B1B685B109B00E8
:10190000D3180393344B1B78002B00D031E52B68A0
:10191000019A1C1213402F4A9B009B5804350AE57C
:101920003B1F1868FFF700FCA40006003F1B1E28A1
:1019300027DC00280DDC284B1B78002B00D018E595
:101940002B68019A1C121340224A9B009B580435B5
:10195000F1E401F0DBFA033E361801F0D7FA214B2F
:10196000801B9842F9D81C4B1B78002B00D000E557
:101970002B68019A1C121340164A9B009B58043591
:10198000D9E40123029A137001F0C0FA029B0A38CD
:1019900086195E6000E53B1F1868FFF7C5FBA400D1
:1019A00006003F1B00280DDC0B4B1B78002B00D0E2
:1019B000DFE42B68019A1C121340064A9B009B58D7
:1019C0000435B8E4084B984210DD1D22024B1A7012
:1019D000CFE4C04644CC0000A002002070CE00003E
:1019E000882500203F420F0080EE36000123029A36
:1019F000137001F08BFAFA239B005E43029B0A3EB0
:101A000030185860C8E4A300FF1A002320001A0011
:101A10003900FFF7D7FBD44ED44C3168200001F0D9
:101A200033FFD34B31681860200003F0C1FF3168E9
:101A3000200004F010F9CF4B1B78002B00D098E465
:101A40002B68019A1C121340CB4A9B009B5804350B
:101A500071E4C84BA4001B783F1B002B00D088E426
:101A60002B68019A1C121340C34A9B009B580435F3
:101A700061E4029803F050FDBE4B1B78002B00D0B0
:101A800077E42B68019A1C121340BB4A9B009B58B9
:101A9000043550E43B1F1B68002B3ED13B000C3B40
:101AA0001B68DA072CD5390001225B105800083971
:101AB00002430A60002B44DD012259001143381F04
:101AC00001603900083909681141CB1A39000C3915
:101AD0000968114224D09B189340A4001343039A31
:101AE000A350A44B1B78002B00D042E42B68019A32
:101AF0001C121340A04A9B009B580435FFF71BFCA7
:101B0000042B06D90F211A680A40092A01D15B6803
:101B1000C9E71922974B1A702BE45B10013BC9E708
:101B2000042909D90F200A680240092A04D1023386
:101B30009B005B58A400D2E719228E4B1A70FFF766
:101B400018FC0435CDE7A300069AFB189B1AD82B86
:101B500013DC0122631E002C14DC864B1B78002B47
:101B600001D0FFF706FC2B68019A1C121340824A31
:101B70009B009B580435FFF7DEFB1A227D4B1A7041
:101B8000FFF7F7FB3A601C000437E3E7069A3B1DBA
:101B90009B1A784ED82B03DD1A233370FFF7E9FB2D
:101BA000069B039AA40093422AD23B1F1868FFF7B2
:101BB000BBFA011E21DD039B0C3B1A6852108242C6
:101BC0001BDB9007801A6D4B4018C018039B8000E8
:101BD000C2583B1B1A60674B3F1B1B780437002B16
:101BE00001D0FFF7C6FB2B68019A1C121340624A12
:101BF0009B009B580435FFF79EFB20233370EAE7D8
:101C00001823FBE75A4BA4001A683B1B1F001A60FD
:101C1000584B04371B78002B01D0FFF7AAFB2B6829
:101C2000019A1C121340544A9B009B580435FFF73D
:101C300082FB3B1F1A68042A11D1A4002D194D4BB9
:101C40001B78002B01D0FFF794FB2B68019A1C1224
:101C50001340494A9B009B580435FFF76CFB1F005B
:101C6000EDE73A1F1368042B04D0002313603A00F9
:101C7000A4002D193F4B1B78002B02D01700FFF753
:101C800078FB2B6801991C120B403B499B005B5869
:101C900017000435FFF74FFBA3009C46FE1A002CEB
:101CA00017DC1C22334B1A70002333606346FF1A83
:101CB000304B04371B78002B01D0FFF75AFB2B6801
:101CC000019A1C1213402C4A9B009B580435FFF7C5
:101CD00032FB002033685A108300F15801230B4077
:101CE00003D10D21234A1170DFE749108A4200DD3C
:101CF0000A0001308442EFDC012352001343D4E791
:101D0000A3009C46FE1A002C17DC1C22194B1A70EB
:101D1000002333606346FF1A164B04371B78002BF1
:101D200001D0FFF726FB2B68019A1C121340124AC0
:101D30009B009B580435FFF7FEFA002033685A10C9
:101D40008300F15801230B4003D10D21094A117082
:101D5000DFE749108A4200DA0A0001308442EFDCF2
:101D6000012352001343D4E7C4050020A102002040
:101D700008000020A002002044CC0000FCFFFF3F30
:101D80003B00083B1868FFF7CFF93B1F06001868B7
:101D9000FFF7CAF90023864200DA0433A4003A1B95
:101DA00017001360E54B04371B78002B01D0FFF7B9
:101DB000E0FA2B68019A1C121340E14A9B009B58E1
:101DC0000435FFF7B8FA3B00083B1868FFF7ACF999
:101DD0003B1F06001868FFF7A7F9F30FC217B042C0
:101DE0005341A4003A1B17009B001360D34B0437E8
:101DF0001B78002B01D0FFF7BCFA2B68019A1C124C
:101E00001340CF4A9B009B580435FFF794FA3B00E0
:101E1000083B18683B1F1968A600BE1B04238142BB
:101E200002D0042802D80023336018E001239C4626
:101E30001842F8D10F2302681A40042AF3D16346EE
:101E40001942F0D10429EED90B680B321340042B50
:101E5000E9D1FFF789F9431E984180003060B74B04
:101E6000A4001B783F1B0437002B01D0FFF781FA39
:101E70002B68019A1C121340B14A9B009B580435F1
:101E8000FFF759FA3B00083B18683B1F1968A6008A
:101E9000BE1B0023814202D0042802D804233360F1
:101EA00018E001239C461842F8D10F2302681A401B
:101EB000042AF3D163461942F0D10429EED90B6804
:101EC0000B321340042BE9D1FFF74EF9434258413E
:101ED00080003060994BA4001B783F1B0437002B17
:101EE00001D0FFF746FA2B68019A1C121340944A5E
:101EF0009B009B580435FFF71EFA3B00083B18680F
:101F0000FFF712F93B1F06001868FFF70DF9F317EA
:101F1000C20F86425341A4003A1B17009B00136076
:101F2000864B04371B78002B01D0FFF722FA2B6871
:101F3000019A1C121340824A9B009B580435FFF7FC
:101F4000FAF93B00083B1868FFF7EEF83B1F060064
:101F50001868FFF7E9F80023864200DD0433A40087
:101F60003A1B17001360754B04371B78002B01D008
:101F7000FFF7FFF92B68019A1C121340704A9B006F
:101F80009B580435FFF7D7F93B1F1B68A400043B9F
:101F90005A1E93413A1B17009B001360674B04378E
:101FA0001B78002B01D0FFF7E4F92B68019A1C1273
:101FB0001340634A9B009B580435FFF7BCF93B0074
:101FC000083B1868FFF7B0F83B1F06001868FFF7DA
:101FD000ABF832180120A4003B1B1F005200024343
:101FE0001A60564B04371B78002B01D0FFF7C1F95C
:101FF0002B68019A1C121340514A9B009B580435D0
:10200000FFF799F93B00083B1868FFF78DF83B1F75
:1020100006001868FFF788F8321A0120A4003B1B5D
:102020001F00520002431A60444B04371B78002BF8
:1020300001D0FFF79EF92B68019A1C121340404A09
:102040009B009B580435FFF776F93B00083B186866
:10205000FFF76AF83B1F06001868FFF765F80200F3
:102060000120A4003B1B1F007243520002431A6070
:10207000324B04371B78002B01D0FFF77AF92B681D
:10208000019A1C1213402E4A9B009B580435FFF7FF
:1020900052F93B1F1868FFF747F8061E17D11F2398
:1020A000264A1370A4003B1B1F001E60234B0437FD
:1020B0001B78002B01D0FFF75CF92B68019A1C12EA
:1020C00013401F4A9B009B580435FFF734F93B002F
:1020D000083B1868FFF728F8310007F079F8012667
:1020E00040000643DEE73B1F1868FFF71DF8061E99
:1020F00017D11F23114A1370A4003B1B1F001E6041
:102100000E4B04371B78002B01D0FFF732F92B68F8
:10211000019A1C1213400A4A9B009B580435FFF792
:102120000AF93B00083B1868FEF7FEFF310007F094
:1021300035F9012649000E43DEE7C046A002002023
:1021400044CC00003B1F1868FEF7EEFFC217801852
:1021500050400122A4003B1B1F00400010431860A8
:10216000F14B04371B78002B01D0FFF702F92B68E5
:10217000019A1C121340ED4A9B009B580435FFF74F
:10218000DAF8A300FE1A3068012C24D1FEF7CCFF48
:102190000494079009F040FC0799002900DC012114
:1021A00007F0FCF8049BA400C91801234900194357
:1021B000DD4B3F1B1B7831600437002B01D0FFF74C
:1021C000D8F82B68019A1C121340D84A9B009B58E0
:1021D0000435FFF7B0F8FEF7A7FF04907068FEF72C
:1021E000A3FF049B0130C31A0793D3E7A300FE1A91
:1021F00031002000049301F0CDFC049B3060FF1AF5
:10220000C94B04371B78002B01D0FFF7B2F82B68BD
:10221000019A1C121340C54A9B009B580435FFF7D6
:102220008AF83B00083B1868FEF77EFF3B1F06005C
:102230001868FEF779FF02000120A4003B1B1F0075
:102240003240520002431A60B74B04371B78002B10
:1022500001D0FFF78EF82B68019A1C121340B34A85
:102260009B009B580435FFF766F83B00083B186855
:10227000FEF75AFF06003B1F1868FEF755FF3200B5
:1022800002430120A4003B1B1F00520002431A60BE
:10229000A54B04371B78002B01D0FFF76AF82B6899
:1022A000019A1C121340A14A9B009B580435FFF76A
:1022B00042F83B00083B1868FEF736FF06003B1F5C
:1022C0001868FEF731FF320042400120A4003B1B9A
:1022D0001F00520002431A60934B04371B78002BF7
:1022E00001D0FFF746F82B68019A1C1213408F4A61
:1022F0009B009B580435FFF71EF83B1F1868FEF73C
:1023000013FFC0430122A4003B1B1F0040001043E9
:102310001860854B04371B78002B01D0FFF729F894
:102320002B68019A1C121340804A9B009B5804356D
:10233000FFF701F83B00083B1868FEF7F5FE0600C2
:102340003B1F1868FEF7F0FE320082405100012268
:10235000A4003B1B1F000A431A60734B04371B7811
:10236000002B01D0FFF705F82B68019A1C121340CF
:102370006E4A9B009B580435FEF7DDFF3B00083B8F
:102380001868FEF7D1FE06003B1F1868FEF7CCFE6A
:102390003200024151000122A4003B1B1F000A43EE
:1023A0001A60614B04371B78002B01D0FEF7E1FF68
:1023B0002B68019A1C1213405C4A9B009B58043501
:1023C000FEF7B9FF3B000C3B1868FEF7ADFE3B0083
:1023D000083B06001868FEF7A7FEF1170200C317B6
:1023E000300007F02DF83B1F049005911868FEF7A8
:1023F0009BFE02000498059906F0D6FF43000120D9
:10240000A4003E1B37001843474B30601B7804374D
:10241000002B01D0FEF7ADFF2B68019A1C12134070
:10242000424A9B009B580435FEF785FFA300FE1A25
:10243000310020000493FEF7C1FC049B3060FF1ABA
:10244000394B04371B78002B01D0FEF792FF2B6825
:10245000019A1C121340354A9B009B580435FEF725
:102460006AFFA300FF1A39002000FEF7BFFC2E4BC5
:102470001B78002B01D0FEF77CFF2B68019A1C1201
:1024800013402A4A9B009B580435FEF754FFA300D3
:10249000FE1A310020000493FEF7E8FC049B306034
:1024A000FF1A214B04371B78002B01D0FEF761FF88
:1024B0002B68019A1C1213401C4A9B009B58043540
:1024C000FEF739FFA300FF1A39002000FEF762FD76
:1024D000154B1B78002B01D0FEF74BFF2B68019AA0
:1024E0001C121340114A9B009B580435FEF723FF32
:1024F000A300FE1A310020000493FEF7BDFD049BEB
:102500003060FF1A084B04371B78002B01D0FEF710
:1025100030FF2B68019A1C121340044A9B009B5801
:102520000435FEF708FFC046A002002044CC00009E
:102530003B1F186800F088FF3A00083A1268030051
:10254000A400D10729D4042A0CD910680F22104006
:10255000013808280FD806F09DFD052026220E0E12
:102560000E0E2400EE49180009F0F6FA43425841D5
:102570003B1B80001860EB4B3F1B1B780437002B84
:1025800001D0FEF7F6FE2B68019A1C121340E64AB2
:102590009B009B580435FEF7CEFEE449E3E7E4498F
:1025A000E1E7E449DFE7E449DDE7069B3E1DF31A76
:1025B000DC4CD82B03DD1A232370FEF7DAFE00F083
:1025C000AFFC43000120184323783860002B02D071
:1025D0003700FEF7CEFE2B68019A1C121340D24A38
:1025E0009B009B5837000435FEF7A5FE069B3E1D59
:1025F000F31ACC4CD82B03DD1A232370FEF7B9FE57
:1026000000F084FCCD4B4000184001231843237890
:102610003860002B02D03700FEF7ABFE2B68019A22
:102620001C121340C04A9B009B5837000435FEF72C
:1026300082FE0123A600BE1B20001A003100FEF717
:10264000C1FDBF4C2068643002F002FF002802D1B7
:10265000043DFEF7A1FE029B21685A78B94803F0B9
:1026600008FB0123029A3700137000F04FFCB64BB1
:1026700022681B68063253431818029B5860FEF705
:102680008BFEA600BE1B2000012300223100FEF7B6
:1026900099FDAB4C2068643002F0DAFE0028D7D0F8
:1026A000A84803F075F8DCE7A4003E1BFEF70AFE1D
:1026B00037009C4B30601B780437002B01D0FEF7AD
:1026C00058FE2B68019A1C121340974A9B009B5896
:1026D0000435FEF730FE934BA4001B783F1B002B04
:1026E00001D0FEF746FE2B68019A1C1213408E4A59
:1026F0009B009B580435FEF71EFEA4003E1B3000D5
:1027000000F03DFC3700874B30601B780437002B0E
:1027100001D0FEF72EFE2B68019A1C121340824A4C
:102720009B009B580435FEF706FEA4003E1B3000BC
:1027300000F027FC37007B4B30601B780437002B00
:1027400001D0FEF716FE2B68019A1C121340764A40
:102750009B009B580435FEF7EEFDA300FE1A3100E6
:102760002000049300F010FC049B3060FF1A6D4BB6
:1027700004371B78002B01D0FEF7FBFD2B68019A74
:102780001C121340684A9B009B580435FEF7D3FD8A
:10279000A4003F1B380000F029FC624B1B78002B83
:1027A00001D0FEF7E6FD2B68019A1C1213405E4A29
:1027B0009B009B580435FEF7BEFDA300FE1A3100B6
:1027C0002000049300F03AFC049B3060FF1A554B44
:1027D00004371B78002B01D0FEF7CBFD2B68019A44
:1027E0001C121340504A9B009B580435FEF7A3FD72
:1027F000A4003F1B380000F063FC4A4B1B78002B01
:1028000001D0FEF7B6FD2B68019A1C121340464A10
:102810009B009B580435FEF78EFD0121200000F03F
:1028200037FC404B1B78002B01D0FEF7A2FD2B6834
:10283000019A1C1213403C4A9B009B580435FEF73A
:102840007AFD0021200000F023FC364B1B78002B82
:1028500001D0FEF78EFD2B68019A1C121340324AFC
:102860009B009B580435FEF766FDA4003E1B30001C
:1028700000F048FC37002B4B30601B780437002BEE
:1028800001D0FEF776FD2B68019A1C121340264AF0
:102890009B009B580435FEF74EFDA4003E1B300004
:1028A00000F044FC37001F4B30601B780437002BCE
:1028B00001D0FEF75EFD2B68019A1C1213401A4AE4
:1028C0009B009B580435FEF736FDA4003F1B3800E3
:1028D00000F006FC134B1B78002B01D0FEF749FDDE
:1028E0002B68019A1C1213400F4A9B009B58043519
:1028F000FEF721FDA4003F1B380003F09BFC094BB1
:102900001B78002B01D0FEF734FD2B68019A1C12B6
:102910001340054A9B009B580435FEF70CFDC0464A
:1029200080CE0000A002002044CC000088CE000031
:102930008FCE000096CE00009BCE0000FEFFFF7FF2
:10294000C4050020A102002004000020A4003E1BBA
:10295000300003F01FFD3700CD4B30601B7804378B
:10296000002B01D0FEF705FD2B68019A1C121340C5
:10297000C84A9B009B580435FEF7DDFCA4003F1BB2
:10298000380003F027FCC24B1B78002B01D0FEF768
:10299000F0FC2B68019A1C121340BE4A9B009B5806
:1029A0000435FEF7C8FCA4003E1B300003F028FCF1
:1029B0003700B74B30601B780437002B01D0FEF78F
:1029C000D8FC2B68019A1C121340B24A9B009B58FA
:1029D0000435FEF7B0FCA300FF1A3900200001F017
:1029E000F7FBAB4B1B78002B01D0FEF7C2FC2B682A
:1029F000019A1C121340A74A9B009B580435FEF70E
:102A00009AFCA300FF1A3900200001F017FAA04B2E
:102A10001B78002B01D0FEF7ACFC2B68019A1C122E
:102A200013409C4A9B009B580435FEF784FCA3008E
:102A3000FF1A3900200001F003FB954B1B78002B97
:102A400001D0FEF796FC2B68019A1C121340914AA4
:102A50009B009B580435FEF76EFCA300FF1A39005B
:102A6000200001F015FB8A4B1B78002B01D0FEF7EC
:102A700080FC2B68019A1C121340864A9B009B58CD
:102A80000435FEF758FCA300FE1A31002000049321
:102A900003F0E0FC049B3060FF1A7D4B04371B7889
:102AA000002B01D0FEF765FC2B68019A1C12134025
:102AB000784A9B009B580435FEF73DFCA300FE1AA4
:102AC00031002000049303F0CDFC049B3060FF1A1A
:102AD0006F4B04371B78002B01D0FEF74AFC2B68A4
:102AE000019A1C1213406B4A9B009B580435FEF759
:102AF00022FCA300FE1A31002000049303F0BAFC6C
:102B0000049B3060FF1A624B04371B78002B01D006
:102B1000FEF72FFC2B68019A1C1213405D4A9B00A4
:102B20009B580435FEF707FCA300FE1A3100200075
:102B3000049303F0A7FC049B3060FF1A544B043746
:102B40001B78002B01D0FEF714FC2B68019A1C1295
:102B50001340504A9B009B580435FEF7ECFBA30042
:102B6000FF1A3900200001F0A1F9494B1B78002B16
:102B700001D0FEF7FEFB2B68019A1C121340454A58
:102B80009B009B580435FEF7D6FBA300FF1A3900C3
:102B9000200001F0A5FA3E4B1B78002B01D0FEF778
:102BA000E8FB2B68019A1C1213403A4A9B009B5881
:102BB0000435FEF7C0FBA300FE1A31002000049389
:102BC00001F00AFA049B3060FF1A314B04371B787E
:102BD000002B01D0FEF7CDFB2B68019A1C1213408D
:102BE0002C4A9B009B580435FEF7A5FBA300FF1A57
:102BF0003900200001F0B8F9254B1B78002B01D0DB
:102C0000FEF7B7FB2B68019A1C121340214A9B0068
:102C10009B580435FEF78FFB069B029AFB1A9B100C
:102C20001361A300FF1A3900200002F0EFFD184BDA
:102C30001B78002B01D0FEF79CFB2B68019A1C121D
:102C40001340144A9B009B580435FEF774FB069B07
:102C5000029AFB1A9B101361A300FE1A3100200098
:102C6000049302F0D3FD049B3060FF1A084B043735
:102C70001B78002B01D0FEF77CFB2B68019A1C12FD
:102C80001340044A9B009B580435FEF754FBC04692
:102C9000A002002044CC00000023F7B55A1E019288
:102CA000002B07DA01F0AAFA02F0E0FE03F040F888
:102CB0001923019300263000194B1968B14212DD27
:102CC000184B1A6801328A420FDAF0241A601D6824
:102CD000154F6C43E35D002B1FD0E419022B06D186
:102CE0002000FEF707FB019BD8E70022EDE7012B50
:102CF0000DD1002801D100F009F9F0226A43BB1878
:102D00005B680A49C31A8B4201D80223BB54F023E3
:102D10005D43054BEB5C022BE2D00136CCE7C046AD
:102D2000C805002000000020281C00203F420F00A2
:102D3000012200210A4B0B481A6119500430195026
:102D4000A2210420C9005850C121C020890080025E
:102D500058501A60044BFC311960044B1A707047CC
:102D600000A000400405000000E100E0EC050020A8
:102D700004207047F8B550C9012322001A40101EE4
:102D80002DD03340181E2AD064100020192C26D8CC
:102D90001D4B761035009E4200DD1D001B4F3B5D34
:102DA000012B05D00121200004F02EFD01233B550D
:102DB000174B1B78002B01D1FFF7BAFF0023154AF0
:102DC0009E420DDCFF2514491448D65CB44202D162
:102DD0005E007052D5540133042BF6D10420F8BDA7
:102DE000D15C8C4203D10C4A5B009D52F6E7013363
:102DF000042BF5D10023D15CFF2901D1D454F2E793
:102E00000133042BF7D1E9E788130000D005002037
:102E1000EC0500201C0000200E000020DC05000056
:102E2000F8B530C9012623003340181E1BD02B00F3
:102E30003340181E17D034410020192C13D8174FD7
:102E40003B5DB34204D03100200004F0DDFC3E5570
:102E500069100800124A1038124B904204D901221E
:102E600052421A600420F8BD1C600F4806F0B0F909
:102E70000E4B18800E4B1B78002B02D1FFF758FF2A
:102E8000F0E701220B4B9A64A922D2009A588018CD
:102E9000A82280B2D2009850E4E7C046D0050020B6
:102EA000908601001800002020A107000C000020DF
:102EB000EC05002000A00040030010B50120002B0D
:102EC00002DC1B30FEF7F8F910BD0420704710B586
:102ED000002803DC1C20FEF7EFF910BD0B68002072
:102EE000DB07FAD40D30F6E701220020054B064936
:102EF0001A61585004310330585008318018585026
:102F00001A60704700800040040500000122034B56
:102F10001A64A822D20098587047C046008000402A
:102F200010B5FFF7F3FFFA21890006F0C7F810BDCE
:102F300000487047F8CE00001A20704770B5054E63
:102F40000400335C0D008B4202D004F05DFC35556B
:102F500070BDC046D005002070B50024064D635DED
:102F6000012B05D10021200004F04EFC0023635505
:102F700001341A2CF2D170BDD005002070470D200D
:102F80007047352070470000F8B501240B68060033
:102F90000D00234204D10D20FEF78EF92000F8BD6C
:102FA0005B102000052BFAD80E4A9B009C580E4F50
:102FB0003B5D002B05D00021200004F025FC002300
:102FC0003B55012E06DD6B68042B03D10221200046
:102FD00004F01AFC200004F0C5FA0124400020434C
:102FE000DDE7C046E0CE0000D0050020F8B50126A0
:102FF0000568354202D04468344203D10D20FEF703
:103000005BF9F8BD6D10192DFBD80A4F7B5D012BC4
:1030100004D03100280004F0F7FB7E550649641007
:103020008C4202DCE143C9172140280004F020FB58
:10303000E7E7C046D0050020FF03000070B501247B
:103040000D68254204D10D20FEF736F9200070BD31
:103050006D10192D17D80024012804DD4C68043C9C
:1030600063425C416400094E735DA34204D02100B9
:10307000280004F0C9FB7455280004F0F9FB030094
:103080000420012BE3D00020E1E7C046D00500205A
:1030900070B504000D0019280ED8084E335C012BC2
:1030A00004D0012104F0B0FB012333552900200096
:1030B0004D1EA94104F0C6FB70BDC046D0050020DE
:1030C000036810B5DA0703D40D20FEF7F5F810BD3C
:1030D0004168581004394A425141FFF7D9FFF6E7D9
:1030E00037B569460A00064B30CB30C20368022070
:1030F000042B02D100F0A4FF37BD00F0C9FFFBE7AD
:10310000A8CE000010B5084C237D002B05D000216F
:10311000142004F079FB00232375142004F0A8FB8D
:1031200043425841800010BDD005002010B5084C26
:10313000A37D002B05D00021162004F065FB0023A1
:10314000A375162004F094FB43425841800010BD43
:10315000D0050020F7B5304D304E6B6C002B15D0EC
:10316000A8240023E40037596B642D4B186800280D
:103170000CDB2C4B19784A425141C9B2197004F04A
:1031800061FB294B1B88DF19BFB23751AB6C002B99
:1031900039D00021254B264FF458A9643A780C34D5
:1031A0000193244D8A4206D02B68032B03D8224A70
:1031B000D05C04F047FB2B68204A0133134004D550
:1031C0000422013B5242134301331B4900228C4627
:1031D0002B60042B18D06046C05C591CFF2802D11C
:1031E0000B000122F5E7002A00D02B60012104F03A
:1031F00029FB01233B702B68114A5B009B5AE418A2
:10320000019BA4B2F450F7BD01235B422B60002365
:103210003B700C4BF3E7C046FCA0004000A0004010
:1032200018000020EB0500200C00002044050000E1
:10323000EA050020CC0500201C00002003000080CF
:103240000E00002050460000084B094AFF201A805B
:103250005A809A80DA800023064A07491370074A89
:10326000087048708870C870136070470E000020A6
:10327000DC050000EA0500201C000020CC05002031
:103280000122024B52421A607047C04618000020CB
:1032900010B5034A0621034802F0A0F810BDC0464D
:1032A000B0CE00001AD60000E12170B549021448E2
:1032B00003F050FFFFF718FE0A2004F04DF9002339
:1032C000FF21104A995401331A2BFBD1012200200F
:1032D0000D4B01001A6004230C4A0D4D1468002C9C
:1032E000FCD02C680002013B20431160002BF5D17B
:1032F0000122084B1A6004F0E9F801F0CBF870BD28
:10330000B01B0020D005002000D0004000D10040BC
:1033100008D5004004D00040F8B50B4E070030003F
:103320000D0003F05FFF0400A84200DD2C003D000B
:10333000EB1B9C4205DD300003F05EFF2870013579
:10334000F6E72000F8BDC046B01B002010B5010014
:10335000014803F007FF10BDB01B002010B5054C5D
:10336000200003F00DFFE1212000490203F0F2FEEE
:1033700010BDC046B01B0020C3070CD4064B1B6811
:10338000834208D8054B1B68984204D8031F1B686A
:10339000002B00D018007047F8050020F40500202D
:1033A0000023012210B50A48990001334250642BD2
:1033B000FAD1084C084B00211A602000074A08F097
:1033C0004BF8074B074A6360074B1A6010BDC046B5
:1033D000802D0020FC05002008000020D4090000FA
:1033E0003027000000060020F005002010B5044B37
:1033F000044A1A60044B054A1A60FFF7D1FF10BD5A
:10340000F8050020FC050020F4050020D00F002066
:10341000044B1B681868000980B20238C343DB17ED
:1034200018407047F005002000B59BB00200054928
:1034300001A808F055FB01A802F0C6F902F078FCDB
:10344000FCE7C0467BCF00000B4BC20704D4042826
:1034500004D80A4B00D00A4B180070470F220368AB
:103460001A40031D042AF7D0064B092AF4D0064B54
:10347000032AF1D0054BEFE755CF0000FACA000050
:10348000F4CA00005FCF00006FCF000066CF0000DD
:103490000020064A0649131F186013681B099BB2D7
:1034A00002339B00D2188A42F5D3704700060020F1
:1034B000D00F0020F7B50F240126314B314A19688F
:1034C000314B324D186813681F002740072F26D84C
:1034D00013681B099BB202339B00D218AA42F2D395
:1034E00000242B4EA500AD192868FFF745FF0134D5
:1034F0002860642CF6D1274C2068FFF73DFF206040
:10350000254C2068002802D0FFF736FF20600025F8
:10351000224B1B680093009B9D4214DBF7BD1B09E7
:103520009BB29B00D3189A42D2D01F68374208D171
:10353000B94206D2B84204D3043F3F68002F00D0FE
:103540001F60043BEFE7F0236B43154A9B181A7882
:10355000002A01D10135DEE71F693C2300266B43B9
:10356000DB199B0001930136BB1BF3D4019BB40014
:103570001C1B0B4B1C19A069FFF7FEFEA061F2E7B4
:10358000F805002000060020F4050020D00F0020E0
:10359000802D002008000020D00F0020C80500204A
:1035A000281C0020F7B50124204246D1234B1B687C
:1035B0009C46984241D3224B1B68019398423CD8C9
:1035C000031F1B68002B38D10200036800941B09FD
:1035D0009BB2002B0FD10099131F196090422CD081
:1035E00015682B1F1B68990069180C68013B146053
:1035F0000A602A00EDE79D0055192968009C2142C8
:1036000019D18C4517D8019C8C4214D30E1F3468F5
:10361000002C10D10F680F343C40072C08D92F60C4
:10362000151F2B600B680A601B099BB20A00D0E7CC
:1036300000993160CDE7013BCBE7F7BDF8050020ED
:10364000F40500200D4970B50A000D4D1368141FD4
:103650001B0926689BB2981C002E0BD000238A42BF
:1036600000D00B0023608300C91880001218AA4202
:10367000ECD370BD1B011360F7E7C04600060020C5
:10368000D00F0020F8B5124C27000F223B681D090F
:10369000ADB213420DD06E1CB600A74204D032006A
:1036A0003900200007F0C5FE0022A3190436A41932
:1036B0001A600235AD00074B7F199F42E5D31B1BF3
:1036C0009B10013B1B012360034B1C60F8BDC046EF
:1036D00000060020D00F0020F0050020F0B59BB0C0
:1036E000FFF714FC00240700214AA300D05801343E
:1036F000FFF758FF642CF7D11E4B1868FFF752FFF5
:103700001D4B1868002801D0FFF74CFF00261B4B0B
:103710001B689E4217DBFFF795FFFFF7CBFEFFF715
:10372000B1FFFFF7F3FB164BC21B1B6815491B6863
:1037300001A81B099BB2023B08F0D2F901A802F0D4
:1037400043F81BB0F0BDF02575430F4BED182B78F7
:10375000002B01D10136DAE72B695C1E002CF9DB66
:10376000A300EB189869FFF71DFF013CF6E7C04680
:10377000802D002008000020D00F0020C805002068
:10378000F005002035CF0000281C0020F7B5174DAC
:103790004F1C2B6806001B680C001B099BB2019292
:1037A0009F420BDBFFF79AFF2B681B681B099BB23C
:1037B0009F4203DB0A20FDF77FFDFEBD2868A71CA2
:1037C000BA00DB1B81181B010B6029600021031F5D
:1037D00019600F231E4003002401264340C3083A0A
:1037E0009A189A42E9D9019902C3FAE7F005002034
:1037F000F7B503000122134004000D000193002BD4
:103800002BD1174B1B68834227D8164B1B6883426A
:1038100023D90F23144F386000681840FFF7B6FF14
:10382000019B3C68061E3B6017D0236804301B09CF
:103830009BB29D4200DD1D00AA00211D251F07F03F
:10384000EFFDFFF725FE2E60FFF734FE00232B600F
:103850002268064B1340236034002000FEBDC046A2
:10386000F8050020F4050020D00F0020F0FF0F0025
:103870000323043010B5C11719400918891000221C
:103880000420FFF783FF10BD70B5050008000C0091
:10389000FFF7EEFF0023002804D170BDE95CC218D9
:1038A00011710133A342F9DBE343DB171C40002312
:1038B00004192371F1E7F0B50C009BB0022804DC79
:1038C0001C20FDF7F9FC1BB0F0BD0123086818426D
:1038D00006D1042804D90F2601683140042901D0FB
:1038E0000E20EEE761680D001D40F9D10429F7D9DB
:1038F0000A683240042AF3D1A2681A4201D10D208D
:10390000DFE7FFF7A1FD06006068FFF79DFDA768F0
:10391000010001AC7F103000257002F0C6FF3900B5
:103920006423220003F026F8200008F01FF90100AC
:103930002000FFF7A9FFC6E710B51C4CA544041EE4
:1039400002D1FFF795FF0BE002F0C8FE0138062810
:1039500028D805F09FFB090911182904240000202C
:103960008023DB009D4410BD200002F033FF011BCB
:103970002000FFF789FFF3E7200002F0D9FE4300A3
:1039800001201843ECE780226946D200200002F0B3
:10399000E6FE684608F0EAF801006846E9E7042117
:1039A0000348E6E70020CCE70420D9E700FCFFFF4E
:1039B000C4CF000070B50C00022803DC1C20FDF70A
:1039C0007BFC70BD01230868184206D1042804D985
:1039D0000F2501682940042901D00E20EFE7616816
:1039E0001942FAD10429F8D90A682A40042AF4D1E4
:1039F000A2681A4201D10D20E1E7FFF725FD05007D
:103A00006068FFF721FDA46801006410280002F03F
:103A10004CFF210002F089FFFFF78EFFD1E770B560
:103A20000D00012803DC1C20FDF746FC70BD0124BD
:103A30000868204206D1042804D90F2102680A40F0
:103A4000042A01D00E20EFE76A682242FAD1042A44
:103A5000F8D913680B40042BF4D1FFF7F5FC0600EE
:103A60006868FFF7F1FC0100300002F01EFF02F071
:103A7000A0FF40002043D9E7F8B507000C001C2048
:103A8000012F0BDD01250868284206D1042804D93E
:103A90000F2102680A40042A03D00E20FDF70CFC17
:103AA000F8BD62682A42F8D1042AF6D913680B409F
:103AB000042BF2D1FFF7C8FC06006068FFF7C4FCD6
:103AC0000100022F14D0A4682C4211D064103000E1
:103AD00002F0EBFE050002F001FE012811D1002CDE
:103AE00002DD0135012C06D12800FFF725FFD7E7BD
:103AF00001246442EBE7280002F078FE013C050057
:103B0000F0E70228F0D1002CEEDD0135012CEBD0DE
:103B100000222800110002F09BFE02F067FE013C2B
:103B20000500F3E710B501240868044016D04410DE
:103B3000200005F0E1FD154905F0ACFC07F092FB13
:103B400003F0DAFF0022124B06F046FD03F07CFF83
:103B500007F018FB43000120184310BD042810D9BA
:103B60000F2302681340042B07D1FFF76DFC2100DF
:103B70000A2208F0C3F80400DAE7032B01D104306D
:103B8000F5E70D20FDF798FBD2E7C046D3023739A1
:103B90000000D040086870B501240500254006D11A
:103BA000042804D90F2302681340042B03D00E20ED
:103BB000FDF782FB70BDFFF747FC03782900233B2C
:103BC0005A4253411022C01808F098F880239B05F0
:103BD000C218044B9A4201D91420E9E7400020435F
:103BE000E8E7C046FFFFFF3F10B5034A0621034840
:103BF00001F0F4FB10BDC04694CF00008CCF000054
:103C00000020704710B51E20FDF756FB10BD10B503
:103C10001E20FDF751FB10BD10B51E20FDF74CFB1B
:103C200010BD10B51E20FDF747FB10BD10B51E20BE
:103C3000FDF742FB10BD10B51E20FDF73DFB10BD8A
:103C400010B51E20FDF738FB10BD10B51E20FDF786
:103C500033FB10BD10B51E20FDF72EFB10BD10B5B7
:103C60001E20FDF729FB10BD10B5034A0B210348A8
:103C700001F0B4FB10BDC04600D0000058D00000D9
:103C80000120034B1860034B1B68834018437047A7
:103C9000F40F0020D40F0020F0B5EFF310810123C2
:103CA000194083F31088134C134AA4461268134E2C
:103CB000013A9340124F134A002B17D01468034265
:103CC0000FD03D682C60C046C046C046C046C046C6
:103CD000C046C046C0460C4C1568246825605B0889
:103CE000EAE765462C6014683460F8E781F31088D1
:103CF000F0BDC04608050050200000200C05005013
:103D0000E00F0020E80F0020DC0F002030B585B068
:103D100001AD0C220649280007F082FB0024285D33
:103D200001210134FFF70AF90C2CF8D105B030BDA0
:103D3000EDD00000F7B56A46394B01AD13800F2373
:103D40009370384B2B800A23AB70FFF7DFF8364BAC
:103D5000364CC0182368984201D20023236026689D
:103D6000002E3DD16B469F5D01213800FFF7E6F83C
:103D700001360021380003F065FD032EF2D1002644
:103D8000AF5D01213800FFF7D9F801360121380075
:103D900003F058FD032EF3D1C8200138C046C046B9
:103DA000C046C046C046C046C046C046C046C046E3
:103DB000C046C046F1D100212878FFF7BFF86878E7
:103DC0000021FFF7BBF8A8780021FFF7B7F8FFF74D
:103DD0009DF8FA2300251B01C01820602800FEBDB5
:103DE000FFF794F8236800259842F7D3032003F0E7
:103DF000B9FB0600042003F0B5FB36180A2003F0D7
:103E0000B1FB0B4B9B1B181A0A4BA84206DB186030
:103E10000023094A236013600125DFE71D60F7E7EF
:103E20000D0E00000304000010270000EC0F00201E
:103E3000E3030000D40F0020F40F00200022054B04
:103E400010B51A60044B1B68934201D002F0E6FBE8
:103E5000002010BDF00F0020D41A002010B5041E61
:103E600010DA1A240A4BA400E25801239340094AAD
:103E700009491360094A1160094A0A4911600A4A4E
:103E8000136010BDFFF758F8A042EADDEAE7C0462C
:103E9000F0DD0000E80F002008050050E00F0020D2
:103EA000DC0F00200C050050180500502B4BF7B517
:103EB0001B680C00002B03D101204042FFF7CEFF0E
:103EC00024680126250035401AD0FF226310120213
:103ED00060121040DAB21043FF221B02120413409A
:103EE00018431F4B1B68202B06D1B4401D4BA40E5A
:103EF000A400E35800021843FFF7CEFE0020FEBDE9
:103F0000042CFBD90F2322681340092BF6D1FF277D
:103F100063683F025B100193019B9D42EEDAAB00A8
:103F2000E3189B68334216D05A105812D1B2384069
:103F30000843FF21120209040A401043084A12688C
:103F4000202A06D15B009B0E06499B0002025858AE
:103F50001043FFF7A1FE0135DEE7C046E80F002061
:103F600020000020D4D200000200086810B5C3076A
:103F70000FD540101823012A03DD4A68042A00D116
:103F80000833054A1360FEF7F9FFFFF767FF0020CB
:103F900010BD01204042EDE72000002010B50124B3
:103FA000044002D04410200010BD042810D90F2373
:103FB00002681340042B07D1FFF746FA21000A22BA
:103FC00007F09CFE0400EEE7032B01D10430F5E777
:103FD0000D20FDF771F9E6E70868F8B5C3071AD5B3
:103FE000FFF7DCFF0300203B5E2B25D80520434371
:103FF00001221D180020114E9D4219D005211024C8
:10400000F75C3C4200D0801801395200641000294E
:10401000F7D10133F0E704280ED90F2203681A40C4
:10402000042A09D11B099BB2002B05D00379DAE7DA
:10403000012340001843F8BD0120FCE7F9D000003F
:1040400070B508680D00FFF7A9FF04006868FFF766
:10405000A5FF621E0100042A14D8451E042D11D8A4
:1040600005236B439B18012215009D402B00064839
:1040700005682B430360054B1B68002B02D0200012
:1040800002F0CDFA002070BDF00F0020D41A0020FD
:1040900070B508680D00FFF781FF04006868FFF73E
:1040A0007DFF621E0100042A13D8451E042D10D87E
:1040B00005236B439B1801229A40074803689343EA
:1040C0000360064B1B68002B03D00022200002F087
:1040D000A6FA002070BDC046F00F0020D41A0020C0
:1040E000F0B5050089B008680C00FFF757FF06908F
:1040F000022D36DD6068FFF751FF0190A068FFF7E1
:104100004DFF04000127231D661E0793731C0293B5
:10411000079B9E4235D0052373430593019B019D68
:1041200005330493049BAB421ED0042E16D86B1E9D
:10413000042B13D80122059B2349013B5B199A40AC
:104140009446224A0B681068069A3A4003920DD0B2
:1041500062461A430A60012200280DD17F00013512
:10416000E0E701240194CDE7029ECFE76246934346
:104170000B600028F2D0039A0299280002F04FFA4F
:10418000ECE7019B1E1D042E1AD8012C18D1002526
:1041900005273B0021006B439B1999400B000A4AFD
:1041A000013511689943094B11601B68002B05D03C
:1041B000019B0022581D290002F031FA052DE8D19B
:1041C000002009B0F0BDC046F00F0020D41A002036
:1041D000086810B5C30703D5FFF7E0FE054B18606C
:1041E000054B1B68002B03D0024B186802F018FA2D
:1041F000002010BDF00F0020D41A00207FB5A04C85
:104200002368002B0AD19F4A1268002A06D19E4BD0
:104210001B68002B01D0FFF78DFD7FBD9B4D2A68E9
:10422000002A26D1984A1268002A1BD0FFF782FD87
:104230000028F2D0FFF76AFD924B24681A681C60D0
:10424000002A16D0002C14D101AD0C229049280070
:1042500007F0E6F8285D00210134FEF76FFE0C2C14
:10426000F8D1DAE7874A1268002AE5D1002BE3D0BB
:10427000E0E700210D2003F0E5FA00210E2003F015
:10428000E1FA00210F2003F0DDFA2E68012E5DD047
:10429000022E00D1A2E0002E51D101363100794C1E
:1042A00004202368994303F0CDFA042123680520F4
:1042B00019404B42594103F0C5FA102123680620EA
:1042C00019404B42594103F0BDFA8021236809018E
:1042D00019404B4259410C2003F0B4FA8021236865
:1042E000090219404B4259410B2003F0ABFA8021DF
:1042F0002368490219404B4259410A2003F0A2FAAF
:1043000080212368890219404B425941092003F05A
:1043100099FA80212368C90219404B42594108206B
:1043200003F090FA802321681B0319404B42594146
:10433000072003F087FA31000D2003F083FA2B6881
:104340000321581C05F02AF8296066E702214D4C2C
:104350000720236819404B42594103F073FA0820A3
:10436000216801404B42594103F06CFA80212368D7
:10437000C90019404B425941052003F063FA8021DE
:104380002368490119404B425941062003F05AFA6B
:1043900080212368C90119404B425941042003F090
:1043A00051FA80212368890319404B4259410A2060
:1043B00003F048FA802321681B0419404B425941FD
:1043C000092003F03FFA31000C2003F03BFA3100E2
:1043D0000B2003F037FA31000E20AEE72021294CE4
:1043E0000720236819404B42594103F02BFA402122
:1043F0002368082019404B42594103F023FA8021D9
:104400002368092019404B42594103F01BFA8021CF
:104410002368490019404B4259410A2003F012FA1F
:1044200080212368890019404B4259410B2003F039
:1044300009FA80212368890119404B4259410C2017
:1044400003F000FA80212368490319404B42594187
:10445000062003F0F7F980212368C90319404B4275
:104460005941042003F0EEF9802321685B041940D0
:104470004B425941052003F0E5F901210F205CE78B
:10448000F00F0020E40F0020F40F0020D80F0020D0
:10449000EDD00000012010B54042FFF7DFFC002006
:1044A000FFF7FAFB10BD000010B5034A09210348CD
:1044B00000F094FF10BDC046D4D300001CD400000F
:1044C00030B502248025094B094AED009C505C5907
:1044D000002CFCD0A124E400884202D30021995092
:1044E00030BD8025ED0018514019F5E700E001408E
:1044F0000405000010B5002806D1C020B0214002FC
:104500008902FFF7DDFF10BDB02080218002C902C3
:10451000F7E7000043425841064B40421840B023A1
:104520009B02C018036800201A0E532A01D11B02F7
:10453000180A704700C0FEFF30B501248025054BE6
:10454000054AED009C505C59002CFCD00160002114
:10455000995030BD00E0014004050000434258413D
:10456000074B40421840B0239B02C018A62310B549
:104570000902DB05090A1943FFF7DEFF10BDC0463B
:1045800000C0FEFF70B5012480250D4B0D4EED00DF
:104590009C515C59002CFCD0002902DC00229A516D
:1045A00070BD557814782D02254394780139240480
:1045B0002543D478043224062C4310C0ECE7C046CF
:1045C00000E001400405000070B505004B680A00DA
:1045D0009C1C2100A400FFF7D5FF281970BD000026
:1045E000134B1B68002B0CD08022B023D2029B02FD
:1045F00000280BD11A1D5B681B0E522B00D1100036
:104600007047B022C02392025B02F1E782420DD9CB
:1046100003681B0E522B09D1436802339B00C0185C
:10462000824203D903681B0E522BE9D00020E7E732
:10463000F8100020F0B50020B7B00024FFF7D0FF3D
:10464000270005002600002D2ED1284D2868FFF7F1
:1046500061FF32003B0001900094254904A807F057
:104660003FFA04A801F0B0F8224B64201C682B68C4
:10467000A0215A425341204A5B421340B022920289
:104680009B18E41A6043490204F0A2FDA0225202E2
:10469000030000921949220004A807F021FA04A897
:1046A00001F092F837B0F0BDFF226B6829689C4694
:1046B0000233FF180B12013613409C4200DA1C0033
:1046C000FF200A14024003926246014001920091C9
:1046D000039A0B4904A807F003FA04A801F074F840
:1046E0002800FFF77DFF0500ADE7C046F810002069
:1046F00026D50000FC10002000C0FEFFD0D4000032
:1047000012D5000070B50020FFF704FF040001205F
:10471000FFF700FF844200DA04000A4B1D686A427A
:10472000554128001D60FFF7E5FEA0226B425202B2
:104730001340054A28009B18044A611C1360FFF7C8
:104740000DFF70BDF810002004800100FC10002057
:10475000F8B50020FFF7DEFE07000120FFF7DAFEC4
:104760003E00204D0643204C0DD18021C020C902BF
:104770004002FFF7A5FE01213000FFF7EFFE1B4BC3
:104780002E6023601DE0874209DD0023B0212B60ED
:10479000164B8902236023680020012517E00123BE
:1047A00080212B60124BC9022360F4E7120E522ABB
:1047B00008D0002800D023600E4801F005F8FFF76C
:1047C000A1FFF8BD28005A68023292009B188B4264
:1047D00005D21A68561CE9D10028F2D0D1E7216031
:1047E000EFE7C046F8100020FC1000200480010014
:1047F00004C00200EBD4000070B50020FFF7F0FE0B
:10480000FF260500002801D1280070BD03681C1494
:104810003440FFF7E5FEDA2CF4D10500F2E70000A2
:104820008022F0B55200A1B00021674806F014FEC6
:10483000802200215200654806F00EFE644BFF27DF
:104840001B681A00049353425A4110000592FFF767
:1048500051FE049C0020631E9C415E4B64421C4040
:104860005D4BE418FFF7C8FF0600002E2DD1049819
:10487000FFF750FE411C0598FFF770FE059A574D53
:10488000534B2C601A60FEF769FD514B64201B6886
:10489000A0215A4253414F4A5B421340B0222C6838
:1048A00092029B18E41A6043490204F091FCA02292
:1048B0005202030000924A49220007A807F010F9AB
:1048C00007A800F081FF21B0F0BD32681314121266
:1048D0003A403B4003921A000A3A092A49D83A4B17
:1048E000039A995C002931D110223E4806F0B4FDAC
:1048F00035002B6803991A123A40914209D11A14D3
:104900003A400B2A27D0132A2DD00A2A01D1354B41
:104910001D602800FFF764FE051EEAD1314B1968BF
:1049200000290FD02000FFF74FFE04002D4B5B192C
:104930005968002903D02000FFF746FE0400043523
:104940000C2DF3D1204B0121039A99543000FFF72D
:1049500047FE060089E73B40022BDADC214A9B0038
:10496000D3185D60D5E7102200211E4806F074FDC3
:10497000CFE71A00153A082AE8D8144A0399525C7E
:10498000002AE3D13500152B00D015003000036854
:104990001A143A40152A0FD01D2A00D10025FFF71E
:1049A0001FFE0028F3D1002D04D020002900FFF7BE
:1049B0000BFE0400054BC6E7039A1B123B409A42CC
:1049C000EDD10500EBE7C046F80F002000110020F4
:1049D000F810002000C0FEFF04C00200FC10002000
:1049E000B5D40000102F002010B5FFF719FF10BD3F
:1049F000F0B585B0039203220333DC17294D144030
:104A0000E4182B68284F5A42534180225B42D2025D
:104A1000A4103B409B18A21C0291244E91000091CF
:104A20000190316800980A18934215D2FFF7F8FEFA
:104A30002B685A42534180225B421F40D202BF186A
:104A40003368009A9B189F4206D2194800F0BCFEBA
:104A50000025280005B0F0BD029B356819066B469D
:104A60001A7BA423DB051343FF222F00090C1943F3
:104A7000019B12041B04134019432800FFF75CFD3F
:104A80000837281D21003760FFF756FD002C04D0A1
:104A90000A9A21003800FFF775FD009B083BFF18BC
:104AA0003760D6E7F810002000C0FEFFFC100020A1
:104AB0008FD4000070B59AB0FFF74AFEFF221E4C5B
:104AC000D2000021200006F0C7FCFF25FFF794FE6E
:104AD0000026002814D10200C300E3580130591EFB
:104AE0008B41D218FF28F7D1144901A806F0F8FF2E
:104AF00001A800F069FE124800F066FE1AB070BD11
:104B000003681A142A400A2A0AD11A122A40FF2AD4
:104B100003D0D200A1180B71A050FFF761FDD8E7B8
:104B2000132AFAD11B122B40FF2BF6D0DB00E21820
:104B30001671E650F1E7C046882500205BD50000DD
:104B40006FD500000021094B094A596001315160BD
:104B500059680029FCD000211961012393600222C9
:104B6000044B8131FF315A501A607047FC100040ED
:104B70000010004000E100E00222064B0121DA674C
:104B80000022054B5A61054A11615A69002AFCD07E
:104B90007047C04604E100E0FC10004000100040F7
:104BA00010B5044C2378002B01D0FFF7E5FF00205F
:104BB000207010BD01120020802301205B055B6E78
:104BC0005B001843704700000120024B1B685B002C
:104BD00018437047841200200120024B1B685B00C1
:104BE00018437047240000200120024B1B685B0023
:104BF000184370478812002070B504000D0016009D
:104C0000FEF78EF9802301215B055A6E267000267F
:104C100053006170E1706272010A5A0A6071A171F9
:104C2000A272010C5A0C000E5B0EA6702571E17188
:104C30002072E272237370BD10B5044C200006F0A0
:104C400095FF01002000FEF71FFE10BD8D12002011
:104C50000E4B10B51B680E4C5A1C0FD00D4C002B80
:104C60000CD00D4C012B09D00C4C022B06D0094C5A
:104C7000042B03D00A4C052B00D1074C200006F072
:104C800075FF01002000FEF7FFFD10BD2800002089
:104C900000D6000088CE00000BD600008FCE0000AA
:104CA00005D6000070B5214C2278002A3DD1204B5A
:104CB00001215A608022D20511605A68002AFCD076
:104CC000002207201B4B1C4901255A50043958501B
:104CD00008315A5019481A4958501A491A485A5016
:104CE0001A495A50A622D2009D50082218495A50FB
:104CF0000431585002201749585017491748585046
:104D0000174804395850182016495850C1218900B5
:104D10005A500539FF395858921802435A501249CF
:104D2000124A9950FFF70EFF257070BD0112002046
:104D3000FC000040001000400C0500007469627522
:104D40001C05000024050000200004022C050000C2
:104D500014050000340500003C050000FFFF0000C2
:104D6000211001005405000002120020040500007B
:104D700070B50E4B06001B78002B01D1FFF792FF98
:104D800000200B4D2C7884420ED00A4B202219783B
:104D90000323091B1940084B4901C918300006F0CC
:104DA0003FFB0120013C2C7070BDC0460112002069
:104DB0008C1200200012002002120020002370B587
:104DC00088B0984235DD0D6801262C0034409C42A5
:104DD0002FD12300042D2CD90F222B681A40230039
:104DE000092A26D16A683F2A23DD6846FFF7C0FFFB
:104DF000230000281DD06B4619783300A14203DB45
:104E00006B461B5D5B003343A200AA18013493601C
:104E1000202CF2D1092169444A780B7812021A43F6
:104E20008B781B041A43CB781B061343024A13608A
:104E30000423180008B070BD8812002070B5454BDF
:104E40008AB01B78002B01D1FFF72CFF02AC2000A9
:104E5000FFF78EFF002802D100200AB070BD237832
:104E60000B2BF9D96378012BF6D1E378012BF3D121
:104E700000231120384E394D33602B70684423795C
:104E8000374A41781360027809021143827812048C
:104E90001143C27812060A4332490A60002B0ED130
:104EA000152169444A780B7812021A438B781B0447
:104EB0001A43CB781B0613433360002318E0012B01
:104EC0001AD1152169444A780B7812021A438B785B
:104ED0001B041A43CB781A211B06134333600E239D
:104EE000627C6944934200DD130000229A422CD177
:104EF00000220420EA54B0E7022B03D1627B103376
:104F00001621EEE7042B0DD11521082269446846CD
:104F100006F086FA0098019902F006FD06F032F9D3
:104F20003060CAE7052BC8D11521082269446846BC
:104F300006F076FA0098019902F0F6FC06F022F9E4
:104F40003060627D0A231E21CBE7885CA8540132C1
:104F5000CCE7C04601120020841200208D120020F0
:104F6000280000208812002010B5134B04001B7885
:104F7000002B01D1FFF796FEFFF7FEFD00200F4A40
:104F80000F49104B54505860013010605868002889
:104F9000FCD0002018610130906018690028FCD016
:104FA000094B0A481B785B011B185350FFF7E4FDBF
:104FB000FFF7C8FD10BDC0460112002000100040E0
:104FC00004050000FC100040001200200212002026
:104FD00010B588B000281DDD0A68012113000B40C0
:104FE00018D1042A16D90F2014682040092811D19D
:104FF00050683F280EDD9800101880680024084291
:1050000001D04010C4B26846C4540133202BF2D101
:10501000FFF7AAFF002008B010BD000010B500285F
:1050200013DD0C68E30710D56410532C0DD8084B22
:105030001B78002B01D1FFF735FEFFF79DFDA12363
:10504000044ADB00D450FFF77DFD002010BDC046B0
:10505000011200200010004010B500280EDD0C6881
:10506000E3070BD56410FF2C08D8054B1B78002BE9
:1050700001D1FFF717FE034A034BD450002010BDA7
:1050800001120020001000402405000013B5002884
:1050900014DD0C68E30711D5094B64100093094B2C
:1050A0000193072C0AD8084B1B78002B01D1FFF77E
:1050B000F9FD6B46054A1957054BD150002016BD26
:1050C000E2ECF0F4F8FC00040112002000100040B3
:1050D0000C05000070B588B0002820DD01240868A8
:1050E00004401CD104281AD90F2302681340042B52
:1050F00015D1FEF7A9F9060006F038FD05001228C3
:1051000000D912252A0002210D326846FFF774FDEE
:105110006B465D73A54205DC6846FFF725FF00205E
:1051200008B070BD2300325D6B449A730134F1E71F
:10513000F0B50D008BB0012832DD086801220400B3
:1051400014402DD104282BD90F2301680B40042BC8
:1051500026D16B68134223D0FEF776F96E680700FC
:105160007310019306F002FD05000E2800D90E25EC
:105170002A000121113202A8FFF73EFD6A4612798A
:1051800002AB5A7302AA73129373019B76141B0E1F
:10519000D67313745574A54205DC02A8FFF7E4FE2C
:1051A00000200BB0F0BD3A5D02A963189A74013477
:1051B000F1E730B589B0002814DD0C68E30711D59C
:1051C000102268460021FFF717FD6B466A466510FE
:1051D0005D73684663122D0E64149373D473157453
:1051E000FFF7C2FE002009B030BD0000174B184A7F
:1051F0005968002903D00021596001319160196973
:1052000000291FD0002018618023DB00D3581149EA
:10521000012B18D1A923DB00D3585B420B600E4948
:105220000B78032B01D801330B7003200B490B784B
:10523000013303400B700A495B015B180949535065
:105240000123936070470860FAE7C046FC100040F5
:1052500000100040240000208C12002000120020CA
:10526000021200200405000010B5034A1021034873
:1052700000F0B4F810BDC04680D5000077D500001E
:10528000044A05491368C85401339B059B0D1360FC
:105290007047C046BC160020BC12002070B5114CEF
:1052A000114A2368834202DC0023236016E0155C68
:1052B000411C2E00FA3E012E05D899420FDA555CAA
:1052C000013D1F2D01D90800ECE70100151A565CBD
:1052D0006E5401318B42FADC181A206070BD1570D3
:1052E000FAE7C046C81A0020C816002010B5FDF71E
:1052F0000DFE064B1A68824201D900221A601B6813
:10530000C31A034898428041404210BDB8120020A1
:10531000204E000010B5094C094A236812689342D8
:1053200000D110BD074AD05CFEF710F80028F8D075
:10533000236801339B059B0D2360ECE7C01600201A
:10534000BC160020BC12002010B50400064B074A12
:105350001B6812689B1ADB439B059B0DA34200DB75
:1053600010BDFFF7D7FFF1E7BC160020C0160020E4
:10537000F7B5050056680191B000441C06301700CF
:10538000FFF7E2FFFB20FFF77BFF1C20FFF778FF12
:10539000E8B2FFF775FFE0B22412FFF771FFE0B249
:1053A000FFF76EFF6B461879FFF76AFF0025AE42E4
:1053B00000DCF7BDAB00FB189C680135E0B2FFF7DD
:1053C0005FFF2012C0B2FFF75BFF2014C0B2FFF7EF
:1053D00057FF200EFFF754FFE9E7000070B5074EB6
:1053E00033680B2B08DC0C255D43054C0133285139
:1053F00064196160A260336070BDC046C4160020AD
:10540000202F002010B5FBF75BFEFFF74DF8FBF7F0
:105410007FFEFDF73DFFFEF7E7FBFEF725FCFFF7FC
:1054200023FF00F0FBFE01F0FDF801F047FB10BD8B
:10543000962210B512010021034806F00DF8002253
:10544000024B1A6010BDC046281C0020C805002071
:10545000064B074A1B6812689B1ADB439B059B0D92
:105460000122834200DC002210007047BC1600209D
:10547000C0160020F8B505000C0016001F1E0ED146
:105480000320FFF7E5FF002808D0FA20FFF7F8FE19
:10549000E8B2FFF7F5FEE0B2FFF7F2FEF8BD501DEF
:1054A000FFF7D6FF0028F9D0FB20FFF7E9FEE8B2AE
:1054B000FFF7E6FEE0B2FFF7E3FEF0B2FFF7E0FE33
:1054C0003012C0B2FFF7DCFE3C00E31B9E42E5DD7C
:1054D0002078FFF7D5FE0134F7E7000070B500240F
:1054E000F0250B4B1B68A34202DCFFF7A1FF70BD48
:1054F0002B006343074A9B181A78002A05D0597875
:10550000002311201A00FFF7B5FF0134E9E7C04678
:10551000C8050020281C0020F8B507000024F0254D
:105520002B0063430C4A01349E18B74211D03178E6
:1055300000290BD00133D15C002311201A00FFF7A2
:1055400099FF2A000021300005F086FF0A2CE7D1E0
:10555000F8BD024B1C60F9E7281C0020C80500209C
:10556000F0B5150001222F00754C1740A54401909D
:105570000291002F11D005AB1A706A105A70120EEA
:105580001A710522691299706D140299DD70FFF786
:1055900071FFCF239B009D44F0BD042D1ED90F2029
:1055A0002A681040042826D1022304AA2800137177
:1055B000FDF74AFF040006F0D9FA624B984200D981
:1055C0001800B84204DC421C05AB02990198DEE7E2
:1055D00001377B1EE35C05AAD355F2E7042D00D00A
:1055E000A9E0032304AA043D13716B425D4105AB9E
:1055F00055710222E9E709287ED1042205AB1A7011
:105600006A68511000916946521209789A70009A9E
:1056100059701F2A01DD202200926A46127806ACDA
:10562000DA70009BBB4202DC05ABE21ACDE7012633
:10563000BB00EB189868064006D1042837D90F2123
:105640000368194002290CD10123237043106370B1
:1056500042121B0E4014A270E07023710534013712
:10566000DFE7042921D102232370FDF7EDFE03902B
:1056700006F07CFAA31C0C2809D86070864201D180
:105680009C19ECE7039A925D9A550136F6E70C22D5
:105690006270039A925D9A550136092EF9D12E2334
:1056A000E372237363730E34D9E7012907D103230F
:1056B000043823704342584160700234CFE709290F
:1056C00009D10423237043685A1062705B12A370DF
:1056D000E6700434C3E703290BD105232370006867
:1056E000020992B2430F92000B40D31A63701B124F
:1056F000EDE726700134B2E7032800D049E7052121
:1057000005AB1970110989B2520F890002408A1A3B
:10571000111299705A701100642A00DD642104206E
:10572000D970C9B2041FA14201DC04324DE72C5CE0
:105730001C540130F6E7002D00D02AE751E7C0469F
:10574000C4FCFFFF2303000070B502000024F02119
:105750000D4E0800604380194578954203D001340E
:105760000A2CF6D170BDF022002105F075FE074A23
:105770001368013BA34200D11460002329001A00E2
:105780001120FFF777FEEDE7281C0020C805002058
:1057900010B5B2B002236A460400137006F0E6F9B1
:1057A000C72800D9C7200023984207DC421C6B465B
:1057B000FE211420FFF75EFE32B010BD69460133B2
:1057C0005A1EA25CCA54EFE730B5B3B002236A4652
:1057D0000500137006F0CAF90400C72800D9C724D1
:1057E00000239C420BDC20003230FFF7ADFD621C31
:1057F0006B46FF211420FFF73DFE33B030BD6946F4
:1058000001335A1EAA5CCA54EBE70000F0B5BBB0E6
:1058100004900C00012803DC1B20FBF74DFD51E038
:105820002A4B08680293C30709D4042807D90F2319
:1058300002681340042B02D1FDF706FE0290234BB1
:1058400060680393C30709D4042807D90F230268AB
:105850001340042B02D1FDF7F7FD039000271C4BEA
:105860001B680693069BBB420BDC039B194A009303
:10587000C821029B08A806F001F908A8FFF7A4FFB9
:10588000CAE70C267E43144B0299F618306806F0DE
:1058900063F9051E05D17368B6680793079B9D429F
:1058A00001DB0137DEE730680399059606F054F90D
:1058B0000836002808D121000498059B08310238D9
:1058C0005B6898473BB0F0BD0135E7E78BCF000040
:1058D000C4160020DCD60000202F0020F7B5234B93
:1058E00006001B68F02100930023009A9A4211DC05
:1058F0000024F0231A006243019201991C4A5518B2
:105900002F78002F12D001340A2CF3D11948FFF759
:105910005BFF29E00A005A43154882185078B042CC
:1059200002D11278002A1FD10133DEE7F0223900BC
:10593000280005F091FD02230D4A0199EB605354B4
:105940000D4AF1008A58009B6E70AE70AA602F61FC
:105950006F61A34202DC054B01341C60002331005F
:105960001A001020FFF786FDF7BDC046C8050020CD
:10597000281C002025DB00008825002010B5FFF73B
:10598000ADFDFF24084AE3005B429B18074AD35C45
:10599000043B012B03D8E043C0B2FFF79FFF013C5B
:1059A000002CEFD110BDC046FC0700008825002068
:1059B000F7B50F00FF247F2501901E4AE300D31A9C
:1059C0001D4A9A181278062A01D0032A20D1FF22F4
:1059D000D2009B18186883682B401C2B18D1C36811
:1059E0001A002A40042A13D102692A40192A0FD129
:1059F0001B0A01339B000C30C018FDF725FD03780E
:105A00000600002B10D006F0B1F80023B84209D0F0
:105A1000013C002CD1D1F7BD019AF15CD25C9142DE
:105A2000F6D101339F42F7DCE043C0B2FFF756FFE7
:105A3000EEE7C04688250020FC07000070B5050091
:105A4000FF24084AE3005B429B18074AD35CAB4241
:105A500003D1E043C0B2FFF741FF013C002CF0D17D
:105A600070BDC046FC07000088250020F7B5FDF793
:105A70004DFA514B1A68824201D900221A601A6805
:105A80004E49821A8A4200D883E01860FDF748FA2E
:105A9000071E00D101370020FDF734FB01900020E4
:105AA000FDF744FB019B0090454C464D002B14D064
:105AB0002368002B00D07AE02B682760002B00D1F0
:105AC00071E0414B01261B78002B63D10920FFF7C1
:105AD000B5FF3E4B1E703C4B1E70009B002B12D03E
:105AE0002B68002B0FD123682F60002B1ED0374B63
:105AF00001261B78002B52D10920FFF79FFF334B63
:105B00001E70314B1E702368002B0FD02F4E327841
:105B1000002A0BD19F4200D227602368FB1A312B49
:105B200004D90720FFF78AFF012333702B68002B6D
:105B30000FD0254E3278002A0BD1BB4200D92F60FE
:105B40002B68FF1A312F04D90820FFF777FF0123B4
:105B500033702368002B0CD0019B002B09D11B4E06
:105B60003378002B02D10720FFF768FF0023236062
:105B700033702B68002B0CD0009B002B09D1124CEA
:105B80002378002B02D10820FFF758FF00232B6059
:105B90002370F7BD0720FFF751FF0C4B9CE708204F
:105BA000FFF74CFFADE7009B002B9CD1ABE7009AC1
:105BB000002A95D1AAE7C046B41200200F270000A2
:105BC000A4120020AC120020B0120020A812002065
:105BD00037B500240500FFF781FC01A80194FDF70B
:105BE0007FFA21002000FEF729F9FEF707FBFDF7F9
:105BF0002BFBFDF745FBFEF74DFCFDF7ADF9A5428C
:105C000004D0FDF7CDFB0248FFF7DEFD37BDC046EF
:105C100016DB0000002310B501001A001120FFF769
:105C200029FC10BD07B56B46197069465A701312EE
:105C30008B701314120ECB700A716B460100052293
:105C40001320FFF717FC07BD10B50A000100122052
:105C5000FFF786FC10BD70B5050008000C0032305F
:105C6000FFF772FB2B00220000211B20FFF702FC34
:105C700070BD10B50C000300110014202200FFF7C6
:105C8000F9FB10BD012370B5FF24084A41185B429F
:105C9000884201D3D84370BD06781D0A2340734063
:105CA0009B009B5801306B40F2E7C046F8D60000DD
:105CB00013B50400FE2813D80A4BC200D0580028A0
:105CC0000ED0436808309900FFF7DCFF01900920EF
:105CD000FFF73AFB01AB042221001720FFF7CAFBB4
:105CE00013BDC04688250020F7B50190FEF784FD5E
:105CF00001250400FF276D42002C01D12800FEBDC4
:105D0000266833143B40152B0DD121000198083132
:105D100005F022FF002801D135123D402000FEF79A
:105D20005FFC0400E8E71D2BF8D101256D42F5E783
:105D3000F0B580279DB0FFF7EDFAA54CA54D206882
:105D4000FF00391A4019FDF7E7FA23680600C31867
:105D50002360002B0ED11DB0F0BD2068391A281821
:105D6000FDF7DAFA236806001B182360FDF7CEF86A
:105D7000994B1860002EF0DC2B78FA2B00D037E11D
:105D80002368022B07DCFFF7B1FA0028E3D00120DB
:105D9000FFF784FADFE76878AC78023818282BD848
:105DA00003F082F919002C00300034003700400065
:105DB0002A004A007C0086008A00A000F10002014F
:105DC0002A002A002A002A002A002A002A002A0083
:105DD0002A002A001001FF2C0ED02000FFF7B4FC8F
:105DE00000227E4BE100CA505B181A71210000921C
:105DF00013001320FEF7FCFD0320C9E72000FFF786
:105E00006DFDF9E72000FFF79FFCF5E7FFF7B6FD12
:105E1000F2E7FFF763FB0020FFF7DAFE7048FFF7B9
:105E2000D3FCE9E7632CE7D86E4BA200D2582100DF
:105E30001520FFF795FBDFE7FEF7DEFCFF270400E8
:105E4000002CD9D025682B143B40152B04D0200002
:105E5000FEF7C6FB0400F3E72000083005F086FEDD
:105E600006000530FFF770FAFB20FFF709FA2D1244
:105E70001D20FFF705FAE8B2FFF702FAF0B2FFF7CC
:105E8000FFF93012C0B2FFF7FBF925002B1B9E4231
:105E9000DDDD287AFFF7F4F90135F7E700211D2051
:105EA00000910B000A00FEF7A3FDFDF779FAA3E7C6
:105EB0002000FFF7FDFE9FE7FDF73AF803AC4A4AE2
:105EC00064210090494B200005F0D8FD02232000FA
:105ED000237005F04BFE2300020000211620FFF77F
:105EE000C9FA89E700243D4AE300D558002D27D0A0
:105EF0006B689E00701DFFF727FA2B00002532000B
:105F0000083321000120FFF7B5FA2F00FEF774FCDB
:105F10002E00002818D1002F04D03A0001212000C3
:105F2000FFF726FA002D04D02A0002212000FFF7F7
:105F30001FFA002E04D0320000212000FFF718FACB
:105F40000134FF2CCFD157E7FF2103681A120A4012
:105F5000A24209D11A140A400B2A08D10B400CD0D6
:105F6000012B0CD0022B0CD0FEF73AFBD1E7132A01
:105F7000FAD100252F002E00F6E70600F4E707000F
:105F8000F2E70500F0E70024FFF7A8FA220021005D
:105F900000942300DA20FEF72BFDFF222100D2001F
:105FA0000E4805F059FA80E7012C02D1FEF742FBBA
:105FB00022E7022C02D1FEF717FD1DE70120FFF7B3
:105FC00007FE19E7002321001A001A2087E7C046C0
:105FD000C81A0020C8160020B8120020882500200A
:105FE000F8DA0000802D00200FDB00000ADB000043
:105FF000FB2B00D0CBE62268042A00DCC3E62E7916
:10600000E878574B360206439E4200DDBFE6331D5B
:106010009A4200DCB7E6EB5CFE2B00D0B7E66B786B
:10602000AC78771E1B2B61D019D8072B47D0082BD3
:106030001CD0012B18D1FF2C16D02000FFF784FBB9
:106040006D79484AB31E009221002A000A20FEF70B
:10605000CFFC454BE400E0501B191D7104E01D2BE3
:1060600056D048D31E2B6AD0701D91E6632CFBD806
:106070006A79022A13D0032A1BD0012AF4D1E979C4
:10608000AB79090219432B7AA4001B0419436B7ADC
:106090001B060B435B001343344AA350E4E7002F75
:1060A000E2DDB11E2F48FDF7EFFB304BA400E050BE
:1060B000DAE7AB79A4005A1E93419B00ECE7632F0B
:1060C000D2DC03AD3A002A49280005F0A9F90023E3
:1060D0002800EB55FFF708FE0028C5DB234B8000A6
:1060E000C25821001520FFF73BFABDE739002048D0
:1060F000FFF75EFCB8E7FF2CB6D06A79022AB3D866
:1061000018490B2000912100B31EFEF771FCABE78C
:10611000632F00DD6327002303A99F420ADCFB43B2
:106120000022DB173B40CB181A70152000917B1C16
:106130002100EAE7EA185279CA540133EDE7012C4D
:1061400092D1002F90DD6B79002B03D01C00322BF5
:1061500000DD322464235C43064B1C6084E7C046A8
:10616000F6030000CE16002088250020802D002098
:10617000CD160020040000200120704710B5064C09
:10618000200000F0D1FD0549200000F0F5FD0122BE
:10619000034B1A6010BDC046F81A0020801A060092
:1061A000CC1A002010B501210D20FCF7C7FE0121FB
:1061B0000E20FCF7C3FE00210F20FCF7BFFE044CAD
:1061C000200000F0EDFC1021200000F005FD10BDC6
:1061D000D81A002010B504680D20E30703D5641019
:1061E000FF2C03D91720FBF767F810BDFFF7DAFF84
:1061F000E1B2024800F012FD0020F6E7D81A0020B4
:1062000010B5FFF7CFFF0021034800F007FD430062
:106210000120184310BDC046D81A002010B5034A0B
:1062200008210348FFF7DAF810BDC0463CDB000048
:106230007CDB0000F8B5012306681E4205D04568E6
:106240001D4202D084681C4203D10D20FBF734F8B4
:10625000F8BD76101520802EF8D86D101620FF2D71
:10626000F4D86410FF2C01D91720EFE70B4B1B6803
:10627000002B01D1FFF782FF094FF1B2380000F087
:1062800012FEE9B2380000F015FDE1B2380000F06E
:1062900011FD380000F072FE0020D9E7CC1A002072
:1062A000F81A0020F7B501221400904222DD0D6893
:1062B0002A421FD01D4B15411B684C68002B01D191
:1062C000FFF75CFFE9B201272500194E3D40300081
:1062D00000F0E9FD002D0FD03C413000E1B200F0AC
:1062E000E9FC300000F04AFE0024A04202D0232046
:1062F000FAF7E2FF2000FEBD042CF2D90F2322683A
:106300001340092BEDD163685B100193019BAB42F5
:10631000E7DDAB00E3189968394204D04910C9B2EF
:10632000300000F0C7FC0135F0E7C046CC1A002071
:10633000F81A0020154B70B51B6805000E00002BE5
:1063400001D1FFF71BFF124CEDB22900200000F035
:10635000AAFDF1B2200000F0ADFC0021200000F009
:10636000ADFD002801D0404270BD72B60122290067
:10637000200000F093FD62B6200000F08CFC0028A5
:10638000F2D0200000F08CFCEEE7C046CC1A0020D2
:10639000F81A002010B501240368234202D0416896
:1063A000214203D10D20FAF787FF10BD5810802835
:1063B00001D91520F7E74910FF2901D91620F2E786
:1063C000FFF7B8FF40002043EFE710B504000128B5
:1063D00014D105211820FFF7ADFF7F282BDC030027
:1063E0007F3301DA7F204042C8235B4258437F213C
:1063F00002F0EEFE052C00D1404210BD032811D161
:1064000001001820FFF796FF7F2814DC03007F337C
:1064100001DA7F204042C8235B4258437F2102F0CB
:10642000D7FEEAE70020052CF5D107211830FFF749
:1064300081FF7F2802DD0138FF38D0E703007F337A
:1064400001DA7F204042C8235B4258437F2102F09B
:10645000BFFED1E710B50120FFF7B7FF43000120D1
:10646000184310BD10B50320FFF7AFFF4300012014
:10647000184310BD10B50520FFF7A7FF430001200A
:10648000184310BD10B508211820FFF753FF030073
:10649000C00FC0180123401015304000184310BD34
:1064A000F8B501231C0098422BDD0F683B4228D031
:1064B0004E6835001D4024D1042E22D90F223168A8
:1064C0000A40092A1DD173685C10202C00DD2024AD
:1064D000144B1B68002B01D1FFF750FE72B67F10E2
:1064E000F9B2114F2200380000F0D8FC62B6A54284
:1064F00014DA380000F0CFFB002804D101246D002D
:106500002C432000F8BD380000F0CAFB0122AB008C
:106510004000F31810439860AD18E8E764000125C7
:10652000EEE7C046CC1A0020F81A002070B52B4BBD
:1065300086B01B68002B02D10120FFF746FF01AD9A
:1065400014220021280004F087FF254E1821300076
:1065500000F0A9FC0321300000F0ACFB002130006A
:1065600000F0ACFC041E13D172B6052218213000D5
:1065700000F094FC62B6300000F08DFB002802D0E1
:10658000300000F08DFBA3000134E850052CF2D15F
:10659000019B7F2B01DD013BFF3BAA687F2A01DDC8
:1065A000013AFF3A29697F2901DD0139FF39C82005
:1065B000434342434843DB11D2115243C0115B4372
:1065C00040439B18181804F013FE01F0DDFA04F0A4
:1065D000D9FD43000120184306B070BDD01A002039
:1065E000F81A0020002070470120704700207047F3
:1065F000002070470120704700207047002070473E
:10660000002070470020704700207047002070472E
:106610000020704700207047002070477047704787
:106620007047000010B5034A0E210348FEF7D6FE5E
:1066300010BDC046CCDB00003CDC00000378013B11
:106640001F2B00D970470130F8E710B5FFF7F6FFB0
:106650000378002B0BD00130222B11D10378002BB3
:1066600003D0421C222B03D11000FFF7E7FF10BD1F
:106670005C2B03D14378002B00D0821C1000EDE787
:106680003A2BF2D02C2BF0D07B2B0BD1FFF7D6FF7F
:106690000378002BE9D07D2B01D10130E5E7FFF72E
:1066A000D4FFF5E720225B2B14D1FFF7C7FF037857
:1066B000002BDAD05D2BF0D0FFF7C7FFF7E7202BD8
:1066C000D3DD2C2BD3D0190091435D29CFD0222BC1
:1066D000CDD001300378002BF1D1C6E7002210B5F0
:1066E000904216D0FFF7AAFF03780422222B10D085
:1066F000023A7B2B0DD0013A5B2B0AD019003039BE
:106700000232092905D92D2B05D1417830390929C3
:106710000AD8100010BD0522742BFAD00132662B66
:10672000F7D001326E2BF4D0581E83415A42F0E765
:1067300070B5FFF783FF037801222D2B01D180185C
:10674000023A00230A2502E06B430130CB1801789E
:106750003039CCB2092CF7D95A43100070BDF8B5C6
:106760000C001500FFF76AFF0378222B02D00023EC
:106770002370F8BD0D236A1E210008250C260A2768
:106780009C4601300378222B02D100230B70F0E7E6
:10679000002BFAD0441C5C2B0BD14378841C622B59
:1067A0000ED0662B0ED06E2B0ED0722B0ED0742B0B
:1067B0000ED0002AE9DD0B70013A01312000E1E73B
:1067C0002B00F6E73300F4E73B00F2E76346F0E71F
:1067D0000923EEE710B50400FFF737FFA04202D906
:1067E0000378202B00D910BD0138F7E710B5002839
:1067F00015D00378002B13D0FFF720FF202103785A
:1068000002008B4300205D2B09D01000FFF71DFF15
:1068100003782C3B5A425341C018FFF70FFF10BDBD
:106820001800FCE70300002070B50C0081420EDD6B
:106830001A785B2A0BD1581CFFF700FF0125AC42E8
:1068400005D0FFF7D3FF002801D00135F7E770BD71
:1068500070B50C001500002901D000230B70002832
:1068600020D00378002B1ED0FFF7E8FE0378060047
:106870002C2B03D10130FFF7E1FE06003378002016
:106880007D2B0FD0844204D02A0021003000FFF776
:1068900066FF3000FFF7D9FE03783A2B02D10130B2
:1068A000FFF7CCFE70BD1800FCE7F0B50D0004004A
:1068B0009DB02E78002E35D02E21280005F03EF90F
:1068C000071E14D0431B0193303E092E14D8280014
:1068D000FFF72EFF01002000FFF7A4FF0400002CAB
:1068E00020D0002F1ED0019B0133ED18E1E72800D6
:1068F00005F03CF90190E7E723787B2B11D1601C70
:10690000642203A9FFF7A4FF041E0BD0019A2900FB
:1069100003A805F032F90028E1D02000FFF795FE2A
:10692000EEE7002420001DB0F0BD70B5050000208A
:106930000C0081421DDD2800FFF7D0FE0300681C1B
:10694000012B14D00020022B13D10022681C11004F
:10695000FFF77EFF012C0CD0FFF748FF002211004B
:10696000FFF776FF013CF5E7FFF740FF013C012C04
:10697000FAD170BDF8B5050000200C0016001F000C
:1069800081420DDD2800FFF7A9FE03000020022B45
:1069900006D1681C3A003100FFF75AFF012C00D1E4
:1069A000F8BDFFF723FF3A003100FFF751FF013C2C
:1069B000F4E710B50024A04218D0FFF73FFE03789B
:1069C0007B2B0AD1013000221100FFF741FF002884
:1069D0000CD0FFF73AFE0134F5E75B2B06D101300E
:1069E000FFF704FF002801D00134F9E7200010BDB3
:1069F000F8B5002816DD0D68EB0713D56D10013DC5
:106A00000124FDF7F9FE0026FF27644200280CD17F
:106A1000002E21D0300005F0A9F801003000FCF76D
:106A200033FFF8BD01256D42EAE703681A143A40C6
:106A3000152A0BD11B123B409C4200DA1C009D42E0
:106A400001D106000836FDF7CBFDDFE71D2AFAD19C
:106A5000012400266442F6E701200134640020434B
:106A6000DFE7000010B508680C00FCF7EDFCFFF74D
:106A70003BF9002803DB6268024B8000C250002013
:106A800010BDC046802D002010B50868FCF7DCFC66
:106A9000FFF72AF90123002802DB024B8000C358CC
:106AA000180010BD802D002010B50868FCF7CCFC44
:106AB000FFF71AF9C043C00F800010BD10B5034A9C
:106AC00004210348FEF78AFC10BDC046CCDC000060
:106AD000C5DC000010B5FCF7E7FBFCF787FCFEF710
:106AE00091FC0448FEF770FEFDF7E4FFFEF746FF59
:106AF00010BDC0461BDD000010B5FCF7CDF810BD81
:106B000070B5002504AC24780573A94205D10A4B61
:106B10000A4A23210A4804F015FC01600949920041
:106B200052589B0002715B58A400837163588560C2
:106B300043710223C37170BD33DD000092DD00009C
:106B400041DD0000F0DD0000037B002B04D1437326
:106B50008373036101330373704700001FB5019114
:106B6000A02100240068C900D2B24450012A10D0EC
:106B7000A24209D0032A0AD0074A8350074B019A40
:106B8000C250012343501FBD02221343F4E70422E5
:106B9000FBE70622F9E7C046540500002405000083
:106BA00010B50400FFF7D0FFA1222368A179D2001D
:106BB00099506179064A2000995021790432995000
:106BC000044B19685A689B68FFF7C8FF10BDC046A0
:106BD0000C050000EC1A00204BB2002B0FDB8023C9
:106BE0003F290FD81F290FD80F290FD807290FD8F1
:106BF00003290FD81B060168074A8B507047802372
:106C00009B04F8E7DB04F6E71B05F4E75B05F2E716
:106C10009B05F0E7DB05EEE7240500000368074A63
:106C200099501A00FC32D1680029FCD0A321C90078
:106C300058580023C0B2D3607047C0461C050000FE
:106C400007B58022074BD2051A6000229A600232F3
:106C50001A7111230E320093034905330348FFF7DD
:106C60004FFF07BDEC1A002000300040D81A00206A
:106C7000F8B505000E0017000024BC4208D02B68B0
:106C8000315D1B6828009847002801D00134F4E7E3
:106C90002000F8BD704710B51C3000F0A9F910BDF8
:106CA00010B51C3000F096F910BD10B51C3000F086
:106CB000A5F910BD70B5437E0D00002B01D1002059
:106CC00070BD6430040000F0A2F90028F7D1200064
:106CD000290000F070F90120F2E70000F7B50193F8
:106CE000FA23002504009B0083600D4B45600833A8
:106CF00003601C300F00160000F052F920006430D1
:106D000000F04EF9074A2761B600B35820006375BA
:106D1000019B9B009B586576A576A375FEBDC0467A
:106D2000D0DD0000F0DD00000123A022C375837DCB
:106D30000E49C133FF33D2059B009950437DC133C7
:106D4000FF339B009950CC220169094B5204CA5071
:106D500005220169243BCA50827D01690833CA506B
:106D60000269417D034BD1507047C0460C060000BC
:106D7000240500000C050000A022002310B50469C2
:106D8000D200A3500A4CA1420FD90A4C8C425B415D
:106D900009495B420B40CD21C9045B1804690749CE
:106DA000635005210369995010BDCC235B04F5E7BE
:106DB000A086010090D00300000098FD240500008B
:106DC000F7B5040000200D000193824265D0160043
:106DD000402A00D9402627001C37380000F0F6F87A
:106DE000B1232269DB00D550802201232169920062
:106DF0008B50A27E002A03D122691362226913609C
:106E00000025731EAB4207D1019B002B04D08022CA
:106E10000221236992009950012223691A62236991
:106E2000FC33DA68002A02D19A6A002AF9D09A6AF9
:106E3000002A0BD1DA60A3232269DB00D158380085
:106E4000C9B2013500F0B7F8B542DAD3019B226927
:106E5000002B0FD11300FC339B6A002B0AD10133A6
:106E6000A376D3612369FC33DA6C002AFCD00022BC
:106E7000DA640AE000230121A37651611A00236934
:106E8000FC3399680029FCD09A602369FC339A6A24
:106E9000002A01D000229A62E8B2FEBD10B501239B
:106EA000FFF78EFF10BD0300AC3310B5040019705E
:106EB000643000F08BF80123637610BD00230200DC
:106EC00070B5AC3243760D001178B1220400006930
:106ED000D20081508022216992008B5022690133B7
:106EE00013622269936026006436300000F080F857
:106EF000002812D0300000F06DF81E4B2269D050EF
:106F00002369FC331A6A002A02D19A6A002AF9D04E
:106F10009A6A002A01D11A62E5E723690122002D4D
:106F20000DD11900FC31896A002908D1DA61236981
:106F3000FC33DA6C002AFCD00022DA6407E05A61E4
:106F40002369FC339A68002AFCD000229A60002052
:106F50002369FC339A6A82420BD098622169064AFF
:106F60008B588B501800022B03D0181F431E9841DA
:106F7000033070BD1C050000C404000010B50121E1
:106F8000FFF79CFF10BD000010B513231222024929
:106F90000248FFF7A3FE10BD00400040F81A002091
:106FA00010B540220021040004F056FA002320000E
:106FB0002364636410BD10B53F24026C531C23404E
:106FC000446C9C4201D08154036410BD00230364CF
:106FD00043647047436C026C934206D03F21C25C0D
:106FE00001330B4043641000704701204042FBE72F
:106FF000036C406C181A00D540307047436C026C2B
:10700000934201D0C05C704701204042FBE73F2221
:10701000036C406C01331340181A43425841C0B20C
:107020007047000003210A4802680A4302600948C9
:1070300002680A4302600849084A094B9B1A03DDAB
:10704000043BC858D050FBDC00F012F8F9F75CF8AC
:1070500024050040540500403CE3000000000020EF
:1070600060020020FEE7FEE7FEE7FEE7FEE7FEE740
:107070002D4B10B51A68D2B2012A0FD12B4A1268D3
:1070800012070BD12A4AE0241168F02208001040B0
:1070900021422DD12749096811422CD01A68D2B259
:1070A000012A12D12149096809070ED1F02020498F
:1070B00009680140402908D11E490968014204D1EC
:1070C0008020C121C005C90042501B68DBB2012BE2
:1070D0000DD1164B1B681B0709D1154B1A68F023FD
:1070E0001A40A02A0FD1134A12681A420ED010BDBE
:1070F0003028CFD0D2E7104A104911608021104AC1
:1071000009021160CAE7D02AF1D1ECE70D4B1A68E9
:10711000012A04D00C4A1A601A68012AFCD1C02244
:107120000A4B1A60E3E7C046E00F00F0E40F00F0FE
:10713000E80F00F0EC0F00F004050040DFFF07C08F
:10714000186C004000EC06407593000014EC0640FB
:107150000120704710B503681322DB69984710BD02
:1071600070470000054B0269D1500369FC331A6A6D
:10717000002AFCD0002201201A6270471C05000082
:10718000030010B55C331A781F231A401E3B190008
:107190009140114AD167C222042104699200A15092
:1071A000026953600269D360A02300220169DB00F9
:1071B000CA5001230169094A5B428B500169084AA0
:1071C0008B5001690C3A8B50016908328B50143096
:1071D000FFF7FCFE10BDC04604E100E00C05000016
:1071E0001405000010B51430FFF702FF10BD10B5F4
:1071F0001430FFF703FF10BD10B51430FFF7EAFE9F
:1072000010BD0000030070B55E331A780469724B3C
:10721000E25003005D331A780469704BE2500300BA
:1072200061331C7802696E4B012C00D09EE0050092
:107230005F352E78A225ED00565102006032157898
:10724000A1220669D200B5500269D4509623DB0012
:10725000994200D88CE096231B01994200D88AE01D
:1072600096235B01994200D888E096239B019942BE
:1072700000D885E0E1239B01994200D882E0962363
:10728000DB01994200D880E0E123DB01994200D87C
:107290007DE096231B02994200D87AE0E1231B028D
:1072A000994200D877E096235B02994200D874E0B7
:1072B000E1235B02994200D871E0E1239B029942ED
:1072C00000D86EE0474B994200D86CE0E123DB0226
:1072D000994200D86AE0E122002312038A425B410E
:1072E000414A5B421340802252059B1801693F4A84
:1072F0008B50A02304220169DB00CA5000210369DE
:10730000FC33D9600369FC331962012301690B6006
:1073100001698B60C1210469890062501F215C30C2
:1073200002780A4093406231314AFF3153500021C4
:10733000415600293CDA0F230B40083B2D4C9B089B
:107340009B001B1903242140A140FC348C40DD69C3
:10735000A5432C00C0258D4029002143D9611F235E
:10736000017819401E3B8B40136070BD00246CE710
:107370009E23DB02BAE79D231B03B7E71E4BB5E74D
:107380001E4BB3E7EC239B03B0E71D4BAEE71D4B51
:10739000ACE71D4BAAE71D4BA8E71D4BA6E71D4B0D
:1073A000A4E71D4BA2E78023DB049FE71B4B9DE76F
:1073B0008C080F4BA400E41803230B40FF21C025C9
:1073C000DB009940AD0066598E433100C0269E40D7
:1073D00033000B436351C2E70C05000014050000A5
:1073E0006C05000090D0030000D0BEFE2405000014
:1073F00000E100E000ED00E000B0130000502700C5
:1074000000A04E0000F0750000509D0000F0EB0061
:1074100000903A0100E0D70100B0AF0300705F07B1
:10742000F7B5009308AB1B7800250193FA230400FD
:107430009B0083600E4B45600833036014300F00DF
:107440001600FFF7ADFD23005C3327611E70009B23
:10745000084A9B00995823005D331970019B200056
:107460009B009A5823005E33DD701A70FEBDC04643
:107470006CDE0000F0DD0000036910B51A00FC327C
:10748000D2680400002A0AD0A322D20099581430EE
:10749000C9B2FFF790FD00222369FC33DA6010BD0A
:1074A00010B50248FFF7E8FF10BDC046B01B002032
:1074B0001D2307B502220093024901330248FFF75A
:1074C000AFFF07BD00200040B01B002010B5002812
:1074D00001D004F07DFA10BD7047000010B500F037
:1074E00011F8FFF7F9FF012000F000FAFFF7F2FAB8
:1074F000FFF702FB024B002BFAD000E000BFF7E7DA
:1075000000000000C420114B80001A58104911409F
:10751000C02212020A431A50C0218022490092025E
:107520005A501A608023A3220021DB05D200995013
:107530000122F9309A60074BFF301950C120023107
:1075400080001950403019501A60704700E100E087
:10755000FF00FFFF00100140014B18607047C0465C
:1075600074000020F7B500231E285AD8384B80003D
:10757000C258042A5BD007D8022A54D055D8042315
:10758000012A09D000234CE0062A54D051D31A2AEC
:1075900053D002231B2AF5D12E4A116808294ED94F
:1075A00009294FD00A240226A02001252A4AC0001A
:1075B00015502A482A4D07681C20BF00074029485B
:1075C000019700685759009027481B0207401F4346
:1075D000C02300989B020340FF20575157590002D7
:1075E00007401F43019B1F43009B58016023184025
:1075F00007433E43565101251C4B1560586800282F
:10760000FCD000205860A1230125DB00D358556031
:10761000A025ED0050511BB2A14202D015D2611A33
:10762000CB401800FEBD0823B6E71023B4E72023A3
:10763000B2E74023B0E78023AEE70123ACE708249C
:107640000026B1E70C000126AEE7091B8B40E8E7F6
:10765000F0DD000070000020007000402C000020D1
:107660000405000030000020FF00FFFFFC70004018
:10767000F0B51E285BD8364B8000C258354B1E68CB
:10768000002E30D1C227344BBF00D859334C0325CC
:107690000440C02000022043D851C0248020640050
:1076A000800018512E4F18602E4B803CD859FF3C5B
:1076B000A043D8510437D859A8432043D85108379C
:1076C000D8590C35A8438446072065462843D8512D
:1076D000A820C0001E50C1208026800076021E50C7
:1076E0001C601C4B1C60142500202B001E4C2E001F
:1076F00046433659771C1BD14343E250A023032550
:10770000C132FF329200DB05D550184B1A68082AA7
:1077100014D114234343E3189A6812485132FF32BC
:10772000920059601150DA68C1239B00C250F0BD2D
:107730009642E1D001300328D9D1F8E7082A02D9CE
:10774000083AD140E5E708239A1A9140E1E7C0469C
:10775000F0DD0000141C002000E100E0FF00FFFF4E
:107760000405000000900040340000207400002058
:107770002149F0B54A6C2148002A14D0A025A12641
:1077800000230124ED05F600C258571C06D0C71887
:107790007F68002F02D027009740AF5114333C2B55
:1077A000F2D100234B64A0230121DB0500260F004A
:1077B0009C4614234B43C3181A1F1268104C0E4DDD
:1077C000920014195219526C002A10D01A00143A5F
:1077D0001268551C09D0103B1B68FF2B05D03B00DD
:1077E000934065461A00074BEA50FC346664013149
:1077F0000429DED1F0BDC046FC90004034000020DA
:10780000009000400C05000000B51E2810D80C4A5E
:107810008000835803290BD8A0220800C133FF330E
:10782000D2059B0001F036FC020905070021D1506A
:1078300000BD0C21FBE70421F9E70321F7E7C0466F
:10784000F0DD00001E280AD8074B8000C258012333
:107850009340A022D205002902D104495350704719
:10786000A121C900FAE7C046F0DD00000C050000C8
:10787000030000201E2B0AD8A021A222C905D20095
:107880008858034A9B009B58D840012318407047F2
:10789000F0DD0000F7B506000D000C008B18019319
:1078A000019B671B9C4207D0336821781B6830001E
:1078B000984701340028F3D13800FEBD0849094A31
:1078C000094B10B51B688858FA22190A1B06184381
:1078D0009200002301F0B4FD4904C00B084310BD21
:1078E0000010014004050000181C002070B5041EA3
:1078F00009D0FFF7E3FF050000F014F8FFF7DEFF03
:10790000401BA042F8D370BD0022044B9A60044A89
:1079100013680133DBB213607047C046FC100140AE
:10792000181C002070470000F0B5C64600B5CB0F0C
:107930009846404A4B005B0D9A1882B00D00040037
:10794000132A2FDC002A49DB3B4F17413E000E4033
:10795000064323D07F08390029400C430AD0374919
:10796000BD438C4663445C425C418023DB0213418F
:10797000E4071D434146CE0031492B008E192200F9
:10798000346875682000290001F000FF0090019123
:107990000098019922002B0003F090F802B004BC7B
:1079A0009046F0BD332A08DD8023DB009A42F5D1F2
:1079B00002000B0001F0EAFEF0E7224A94460122A1
:1079C00063445242DA400242E8D052080242D1D027
:1079D00094438022D2051A411443CBE74B005B0845
:1079E0000343DBD00B031B0B1C4363422343802464
:1079F0004D0C24031B0B23406D042B4319004346FD
:107A0000DA000F4B9B181C685D6802000B00200019
:107A1000290001F0BBFE009001910098019922001D
:107A20002B0003F04BF842464B005B08D60733436C
:107A30001900B3E701FCFFFFFFFF0F00EEFBFFFFA4
:107A4000A0DE0000EDFBFFFFF8B5274A4B005B0D01
:107A50009A180C000700132A10DC002A36DB234B8F
:107A600013410B423AD080242403144100206418AF
:107A70009C430600250030002900F8BD332A0EDDA6
:107A800080230600DB000D009A42F4D102000B00B7
:107A90003800210001F07AFE06000D00EBE7144DDE
:107AA0000600AC46012563446D42DD40AC466346AA
:107AB0000D000342DFD033239A1A323B934018184B
:107AC000874200D94C1C63469843D2E7C90FCC07C4
:107AD0000020531CCDD1074B1C43CAE706000D0004
:107AE0000028C0D1C7E7C04601FCFFFFFFFF0F0021
:107AF000EDFBFFFF0000F03F30B5214A4B0087B09F
:107B00005B0893421EDD1F4A934205DD02000B0015
:107B100002F0D4FF07B030BD02AA00F095F80323AD
:107B20001840049A059B012813D002281DD0002874
:107B300014D00298039900F06FFB80231B069C462B
:107B40006144E7E7002300220093002301F0DEF800
:107B5000E0E70298039900F05FFBDBE7012402985D
:107B60000399009401F0D2F8D4E701240298039914
:107B7000009401F0CBF880231B069C466144C9E7C2
:107B8000FB21E93FFFFFEF7FF0B54746CE4680B5CA
:107B90008DB004000D0000F067FA294B06001B7839
:107BA0000F005BB29846013310D022002B0020005A
:107BB000290003F0CBFA8146002807D100220023D8
:107BC0002000290001F014FC002806D13000390003
:107BD0000DB00CBC90469946F0BD01230293194BA1
:107BE0000694079503934B460A93434604940595E0
:107BF000002B15D0002300221900100002F0E2F83B
:107C0000434608900991022B0ED103F0B9FB2123C2
:107C100003600A9B0193002B0CD1089E099FD5E7B6
:107C2000002300240893099402A801F0C1F9002858
:107C3000EFD1EAE703F0A4FB0A9B01930360ECE7B2
:107C400078000020B0DE0000F0B54E464546DE4626
:107C50005746E0B5E14B4C008FB09046894664082A
:107C60009C4200DC87E0DE4B9C4222DCDD4A00299E
:107C700000DC92E0DC4B02F021FFDB4B06000F0042
:107C80009C4200D17EE1D94AD94B02F017FF020095
:107C90000B00414630000A604B60390002F00EFFD5
:107CA000D34BD24A02F00AFF434601259860D960BF
:107CB0006BE0D04B9C4200DC8FE0CF4B9C4200DD60
:107CC00055E1CE4A231592469A4451460905631A56
:107CD00019001D00040003F055FA03F089FA0200B0
:107CE0000B00200029000892099302F0E7FE002211
:107CF000C34B02F071FC0F00060003F043FA03F0DF
:107D000077FA04000D0002000B00300039000A94DD
:107D10000B9502F0D3FE0022B94B02F05DFC00226D
:107D200000230C900D9101F05DFB002800D192E141
:107D3000002300222000290001F054FB434243416C
:107D40000133B04A41460192022208A800925246ED
:107D500000F07CFB4B460500002B16DA80224346E0
:107D60001206944642465B68454263445360D368BA
:107D70006344D36009E00B00020041460A604B6097
:107D80000022002300258A60CB6028000FB03CBC95
:107D900090469946A246AB46F0BD934B01F0F6FCE7
:107DA000914B06000F009C4200D13DE18F4A904B61
:107DB00001F0ECFC02000B00414630000A604B6011
:107DC000390002F07BFE894A894B01F0DFFC012576
:107DD00043466D429860D960D7E701F049F88A4A76
:107DE0008A4B06000F0002F0F7FB0022884B01F0DF
:107DF000CDFC03F0C7F9050003F0FAF9794A7A4B94
:107E00000490059102F0E8FB02000B0030003900FD
:107E100002F054FE754A06000F0004980599744B51
:107E200002F0DAFB029003911F2D00DCC7E0029AFA
:107E3000039B3000390002F041FE83468A465346D8
:107E40005B0024155B0DE31A102B6CDD049805997B
:107E5000D322674B520502F0BFFB02000B0030003B
:107E600039000292039302F029FE0A000100130078
:107E70000691079202003900300002F01FFE029ABC
:107E8000039B02F01BFE06000F0004980599614A4F
:107E9000614B02F0A1FB32003B0002F00FFE069E98
:107EA000079F0B000200390030000292039302F09A
:107EB00005FE4B005B0D83468A46E41A312C32DD09
:107EC00004980599B822544B920502F085FB0300F3
:107ED0000C000200029303940B000698079902F02D
:107EE000EDFD02000B0006000F000698079902F056
:107EF000E5FD029A039B02F0E1FD484A02900391DE
:107F000004980599464B02F067FB029A039B02F026
:107F1000D5FD02000B00300039000292039302F0FD
:107F2000CDFD83468A465A465346414630000A6094
:107F30004B60390002F0C2FD029A039B02F0BEFDC5
:107F400044460B000200A260E3604B46002B00DBBE
:107F50001BE75B46236080231B065344636080233A
:107F60001B069C466144A060E1606D420DE70B007A
:107F7000020002F0A3FD434600259860D960186016
:107F8000596002E7D3221A4B520502F097FD214AAD
:107F9000214B0D00040002F091FD02000B00414650
:107FA00020000A604B60290002F088FD1A4B194A34
:107FB00002F084FD434601259860D960E5E60200A1
:107FC0000B003000390002F079FD6B1E154A9B0052
:107FD0009B5883468A46A342A5D130E7FB21E93F5F
:107FE0007BD9024000004054FB21F93F3163621A03
:107FF00061B4D03DFB213941FFFFEF7FEAFBFFFF7A
:108000000000704138DF000083C8C96D305FE43F75
:108010000000E03F7370032E8A19A33BC14920255D
:108020009A837B39B8DE0000D3220C4B520501F055
:10803000ADFB0B4A0B4B04000D0001F0A7FB020047
:108040000B00414620000A604B60290002F036FD1B
:10805000034A044BB9E6032373E6C04661B4D03D3E
:108060007370032E8A19A33BF8B54746CE46674B7B
:1080700080B50A000F00190005003940994200D16F
:108080009BE004000100002F69DD3F1500D1B4E042
:108090005F4B12039C468023120B5B0313435B0070
:1080A000CA0F67449B184A00F80703D5D20F5B003C
:1080B0009B188A0079108C4600218020162489465E
:1080C00080030D189D4202DC29185B1B8144D50FEB
:1080D0005B00013C5B1952004008002CF1D10020EC
:1080E0008046802020250027000609E08B425CD0D6
:1080F000D40F5B00013DE31852004008002D16D05C
:10810000C4198B42F2DD27180E00002C49DB5B1AE4
:10811000A242894149425B1A121BD40F5B00013D08
:1081200080443100E31852004008002DE8D1134389
:108130004ED143465B0837494A4688464946521065
:108140004244C90702D5802109060B4361460F0549
:10815000BD18180029000CBC90469946F8BD7B005C
:108160005B0803433900002BF5D0002F3CD1E30A14
:10817000153A6405002BFAD08020400303423FD11A
:10818000002700E00F005B00791C0342FAD02500B5
:1081900020208D40401A2900D71B2200C2401A43DC
:1081A00076E7FE43F60F8E19B1E79442A0D8271860
:1081B000002CF6DB1E000023AEE702003B00280087
:1081C000390002F009FA2A003B0001F0DFFAC2E7A9
:1081D0004346013303D0434601335B08ABE7012339
:1081E00098460023C144A6E73B00020002F066FC6B
:1081F00002000B0001F0E6FDADE713000022BBE733
:108200000127210020207F42C6E7C0460000F07F02
:1082100001FCFFFF0000E03FF0B54746CE4680B5C9
:1082200087B000920193754B4F00814688467F08C6
:108230009F4263DC02F0A6FF002800D1D4E04A464A
:1082400043464846414602F0C7F904000D006C4A17
:108250006C4B02F0C1F96C4A6C4B01F097FA2200AA
:108260002B0002F0B9F96A4A6A4B02F027FC22009F
:108270002B0002F0B1F9684A684B01F087FA22003E
:108280002B0002F0A9F9664A664B02F017FC2200A7
:108290002B0002F0A1F9644A644B01F077FA220046
:1082A0002B0002F099F9029003910022604B20000C
:1082B000290002F091F9029A039B06000F002000AA
:1082C000290002F089F9009A019B04000D0048463C
:1082D000414602F081F902000B002000290002F063
:1082E000EDFB02000B003000390002F0E7FB02005A
:1082F0000B0000204F4902F0E1FB70E002000B0090
:1083000002F06AF904000D003D4A3E4B02F064F9A8
:108310003D4A3E4B01F03AFA22002B0002F05CF994
:108320003B4A3C4B02F0CAFB22002B0002F054F9FE
:10833000394A3A4B01F02AFA22002B0002F04CF99C
:10834000374A384B02F0BAFB22002B0002F044F906
:10835000354A364B01F01AFA2B00220002F03CF9A4
:10836000354B029003919F429FDD344B00229F4288
:108370003DDC334900207B182E4916001F0002F017
:108380009DFB049005910022294B2000290002F05A
:1083900023F932003B0002F091FB029A039B060096
:1083A0000F002000290002F017F9009A019B040039
:1083B0000D004846414602F00FF902000B00200074
:1083C000290002F07BFB02000B003000390002F0B4
:1083D00075FB02000B000498059902F06FFB07B0D3
:1083E0000CBC90469946F0BD00201249F7E7154BAA
:1083F000002604920593144FC5E7C046FFFF3F3E99
:10840000D43888BEE9FAA8BDC4B1B4BD9EEE213E01
:10841000AD529C804F7E923E9015CB19A001FA3E42
:108420007751C1166CC1563F4C5555555555A53F12
:108430000000E03F0000F03F3233D33F0000E93F4F
:108440000000E0FF0000E73F0000D23FF0B5DE464D
:108450004E4645465746E0B5DC4CA5440D91140008
:108460001900A49A0993DA4B9200D6584D1E039036
:108470001821E01E0696029500F0AAFEC3430100F3
:10848000DB1719404B1C9A009B1ADB001B190B9140
:1084900005934C1B771918D4A59BA5009C463F1942
:1084A00022AE6544013707E0286802F0A1FE0134DE
:1084B00003C60435BC4208D0002CF5DA00200021A8
:1084C000013403C60435BC42F6D1069B002B01DA09
:1084D00000F0FDFB069B03990133DB009A46099BE4
:1084E000DA00944600920022914672AA0492B94A98
:1084F0006144934688469AAB63449B44029B002B9D
:1085000000DABCE15D4600260027039C4D442A6842
:108510006B6803CC02F060F802000B0030003900F9
:1085200001F034F9083D06000F004445EFD1049BEB
:108530004B441E605F6008239C46E144D145DDD179
:108540000EA804218446494261448C46069A930051
:108550009C44614684460A910399083B63448C46D7
:108560000C93009B009263449B46009A0498D100B0
:1085700003008C46634408911E685F68002A33DD5F
:10858000954980468C466244D300984470AB9A4625
:108590000EAB99460022914B3000390002F01CF8D6
:1085A00002F0F0FD02F024FE00228D4B04000D00CD
:1085B00002F012F802000B003000390002F07EFADF
:1085C00002F0E0FD4B4601C39946434620001A687D
:1085D0005B68290001F0DAF808235B429C46E0441E
:1085E00006000F00D045D5D1059B30001A00390098
:1085F000984600F0DFFCFF2300229B0504000D00DD
:1086000001F0EAFF00F038FC0022764B01F0E4FFB5
:1086100002000B002000290002F050FA0D000400B7
:1086200002F0B0FD814602F0E3FD02000B002000E5
:10863000290002F043FA060040460F00002800DC43
:10864000EEE0009B18215A1E92000EAB9B58091AAF
:108650001D000D41A9448D405D1B0EAB9D5017239D
:108660001B1A1D41002D2DDD01239C46009BE1447A
:10867000002B00DC1CE20E9C0123002C00D0B5E096
:10868000009A012A09D099000EAA54580133002CEF
:1086900000D0ACE0009A9A42F5D1059B002B0EDD8C
:1086A000012B00D1A8E1022B09D1009B0EA95A1E73
:1086B00092000EAB9B5807939B029B0A8B50022D96
:1086C00000D1C1E0002300223000390000F08AFE12
:1086D000009B002800D194E2069A591E8A4210DCC1
:1086E000414A0A9894460EAA6344944600229B008D
:1086F00063441C68043B22438342FAD1002A00D021
:10870000C0E0069B0EAA013B9B00D358002B00D073
:10871000B3E001220C9B043B596801320029FAD0D6
:10872000009B9C466244110007921A0001338B4261
:1087300046DC0B9863468046A59C4344A046099CB2
:108740009B00A1464A449844D30022AA9146049A29
:1087500099449446089BA59A634484466144944690
:108760009A468B00634400934346586802F040FDEC
:108770004B4618605960029B002B24DB4D46039C3E
:108780000026002701E0286869680CCC01F024FF6E
:1087900002000B003000390000F0F8FF083D060031
:1087A0000F005C45EFD153469E60DF6004239C467A
:1087B0000433E0449C46009BE144E2449845D3D115
:1087C000079B0093D1E600260027ECE794FDFFFF0E
:1087D00080E0000018FEFFFFFFFFFF1F0000703E5B
:1087E0000000704100002040FFFFFF3F0021802279
:1087F0005204141B0EAA5450009999420EDD0EA883
:1088000084469B000EAA8900D25861446344CF4835
:1088100000E01A68821A04C38B42FAD101243CE7B3
:10882000059B002B06D1009B0EAA013B9B00D5584F
:10883000ED1517E70022C64B300000F0F7FD0028C9
:1088400000D024E100253DE732003B000020C14973
:1088500002F034F906000F00002C00D132E7059A2F
:108860000020BC4900F0A6FB02000B0030003900DC
:1088700002F024F906000F0024E7012250E7002649
:10888000002754E64B46059A079388468B000EA9AD
:10889000CB58183A08950592002B0DD18C464146CD
:1088A000AD4B43449B006344043B58680139183A7C
:1088B0000028F9D088460592059A0020A54900F0C5
:1088C00079FB434604000D00002B00DA05E29E0010
:1088D0000EAB9C464346DB0066449C46059370AB5A
:1088E0009946049F67440097306802F081FC22009B
:1088F0002B0001F071FE002238607960974B200058
:10890000290001F069FE083F04000D00043EB9454E
:10891000EAD14AAB03939B4600239A46069B424604
:10892000994643460132029204934B46002B00DAEB
:10893000AAE080208A4B009D9846C0058949002600
:108940000027002408E008239C460835E0445445ED
:1089500011DC4346186859682A686B6801F03CFED0
:1089600002000B003000390000F010FF0134060057
:108970000F00A145E7DA5B46C0C39B4601239C4636
:10898000009BE244083B0093029B9A45CDD1049B97
:108990009846A49B022B00DD8EE0002B37DC1FD114
:1089A000059B00271D00039B00249C461E00654478
:1089B000083E2A686B683800210000F0E7FE083D99
:1089C00007000C00AE42F4D1089B002B03D080239B
:1089D0001B069C4664443A0023000D990A604B60D4
:1089E0000720079B18409B239B009D443CBC90465E
:1089F0009946A246AB46F0BD009B0EA95A1E9200B6
:108A00000EAB9B5807935B025B0A8B5057E64346BD
:108A1000002B00DA70E100200021DB004AAAD61802
:108A200048AF32687368083E00F0B0FEB742F8D134
:108A3000089B002B00D025E10B0002004A984B99BF
:108A40000D9C2260636002F039F8434607000C0079
:108A5000002B13DD01254CAEB14638002E0021005D
:108A60004C4601360CCC00F091FEA146B045F7DA39
:108A7000089B07000C00002B00D015E13A002300F2
:108A80000D998A60CB60ABE70026002773E70123CE
:108A90009C46009BE1440225002B00DDEBE5320003
:108AA0003B0000202B4902F009F806000F0009E600
:108AB0000024F2E54AAB0393A49B032B00D08FE77D
:108AC0004346002B00DC14E1039ADB009B461300B5
:108AD00091465B441E685F68234B43440293DB006E
:108AE000994448AB9A464B465C681B6818002100C5
:108AF00032003B000090019100F048FE04000D00A0
:108B000002000B000098019901F0D8FF3B003200F1
:108B100000F03CFE4B469860D9601C605D60082305
:108B20005B429C46E14426002F00CA45DBD1434608
:108B3000012B00DCE3E0039A13005B441E685F68CE
:108B4000029BDB0099464A44904610E0FFFFFF007D
:108B50000000E03F0000F03FFFFFFF3F0000703EDD
:108B600040E00000FB21F93FFFFFFF1F984643460E
:108B70005C681B681800210032003B0000900191E6
:108B800000F004FE04000D0002000B0000980199A3
:108B900001F094FF32003B0000F0F8FD4346039AD9
:108BA0009860D9601C605D60083B26002F009A42E7
:108BB000DCD14D46944600260024474608356544DE
:108BC0002A686B683000210000F0E0FD083D0600D7
:108BD0000C00AF42F4D1039B4A9F5D689968D86846
:108BE000089B002B65D08022120694460D9B65449D
:108BF000604464441F605D609960D8601E615C6180
:108C0000EEE69A464B460793059B30005A423900E0
:108C1000089500F0CFF900223A4B06000F0000F053
:108C200005FC002824D0384B00223000390001F028
:108C3000D3FC02F0A7FA52460400950002F0D8FADD
:108C40000022304B01F0C8FC02000B00300039005C
:108C500001F034FF02F096FA0EAA50510122059B52
:108C6000524418339046059393000EAAD45023E63D
:108C70005346300039009C0002F084FA0EAB1851C4
:108C8000D04619E680230D9A1B06CB18106053605E
:108C90000B0002004A984B9901F010FF4346070071
:108CA0000C00002B00DDD5E680231B069C466444A7
:108CB000E4E62B003A000D9D2A606B600A00030079
:108CC000AA60EB60320023002A616B6188E6099B91
:108CD000DB00009372AB049332E4A49B022B00DD13
:108CE000E8E6002B00DD92E600D079E600270024BC
:108CF0006AE6002600246EE70020002198E60026A0
:108D0000340068E7000070410000703EF0B5CE46C8
:108D1000474680B587B000920193474A4B00814691
:108D200088465B08934207DC4146484602F02AFA2F
:108D30004146031E484666D04A4643464846414699
:108D400001F04AFC04000D0002000B0048464146B9
:108D500001F042FC394A3A4B06000F00200029007E
:108D600001F03AFC374A384B01F0A8FE22002B00F4
:108D700001F032FC354A364B00F008FD22002B0092
:108D800001F02AFC334A344B01F098FE22002B00FC
:108D900001F022FC314B324A00F0F8FC0E9B0290AD
:108DA0000391002B34D00098019900222D4B01F043
:108DB00013FC029A039B049005913000390001F0E6
:108DC0000BFC02000B000498059901F077FE2200CD
:108DD0002B0001F001FC009A019B01F06FFE224A7A
:108DE00004000D00214B3000390001F0F5FB0200BA
:108DF0000B002000290000F0C9FC02000B004846CF
:108E0000414601F05BFE07B00CBC90469946F0BDB0
:108E100002000B002000290001F0DEFB124A134B78
:108E200001F04CFE32003B0001F0D6FB4A464346BF
:108E300000F0ACFCE7E7C046FFFF3F3E7CD5CF5AD1
:108E40003AD9E53DEB9C2B8AE6E55A3E7DFEB157CB
:108E5000E31DC73ED561C119A0012A3F1111813F11
:108E6000A6F810110000E03F495555555555C53F2E
:108E700049004B0819007047474AF0B54F469146E4
:108E80004B005B0D99444646D6464A46C0B50500A0
:108E90000C000E0088460700132A27DC002A4BDB53
:108EA0003E4B13419A460B0052461340034318D0E1
:108EB0003B4A3C4B2800210000F068FC00220023C4
:108EC00000F0AAFA002847D0002C04DA80234A4692
:108ED0005B03134198444646534600279E4338009F
:108EE00031001CBC90469946A246F0BD332A08DDED
:108EF0008023DB009945F4D102000B0000F046FC12
:108F0000EFE7294A9446012263445242DA409246EE
:108F10000242E6D0224A234B2800210000F036FC12
:108F20000022002300F078FA002815D0002C1EDB68
:108F3000534646469F430FE0194A1A4B280021002A
:108F400000F024FC0022002300F066FA002803D081
:108F5000002C04DB0027002638003100C1E7640044
:108F6000640825430027002DF6D0104EF4E74B4649
:108F7000142B0BD03422D21A012393405D19BD4229
:108F800008D201239C462F00E044D1E7133B9C46C6
:108F9000E044CDE72F00CBE701FCFFFFFFFF0F0010
:108FA0009C7500883CE4377EEDFBFFFF0000F0BFBE
:108FB000002070474B0070B55B0D14000A00002BB9
:108FC0001AD14B005B08034315D0234B002201F05C
:108FD00003FB224B9C422DDB0A004B005B0D363B12
:108FE0001F4DE318AB422ADC002B0DDD1D4C1B0589
:108FF00022401A43110070BD1B4DAB42F0D102005C
:109000000B0000F0C3FBF6E71D00353519DA174BEE
:1090100002009C4209DD0B001548164900F032F8A9
:10902000134A144B01F0D8FAE5E70B001248134934
:1090300000F028F8104A114B01F0CEFADBE70200ED
:10904000E9E7084C363322401B0513431900002280
:109050000B4B01F0C1FACEE700005043B03CFFFFDC
:10906000FE070000FFFF0F80FF07000050C3000055
:109070009C7500883CE4377E59F3F8C21F6EA50149
:109080000000903C30B54A00DB0FDB0752081A4362
:10909000110030BD02B4714649084900095C49001D
:1090A0008E4402BC7047C04603B471464908400074
:1090B0004900095A49008E4403BC70470022430806
:1090C0008B4274D303098B425FD3030A8B4244D390
:1090D000030B8B4228D3030C8B420DD3FF220902D2
:1090E00012BA030C8B4202D31212090265D0030B91
:1090F0008B4219D300E0090AC30B8B4201D3CB0387
:10910000C01A5241830B8B4201D38B03C01A5241C8
:10911000430B8B4201D34B03C01A5241030B8B42CA
:1091200001D30B03C01A5241C30A8B4201D3CB02B5
:10913000C01A5241830A8B4201D38B02C01A52419A
:10914000430A8B4201D34B02C01A5241030A8B429D
:1091500001D30B02C01A5241CDD2C3098B4201D3B5
:10916000CB01C01A524183098B4201D38B01C01A33
:10917000524143098B4201D34B01C01A52410309AA
:109180008B4201D30B01C01A5241C3088B4201D359
:10919000CB00C01A524183088B4201D38B00C01A06
:1091A000524143088B4201D34B00C01A5241411A2D
:1091B00000D20146524110467047FFE701B500203A
:1091C00000F0F0F802BDC0460029F7D076E77047FE
:1091D00003460B437FD4002243088B4274D3030918
:1091E0008B425FD3030A8B4244D3030B8B4228D3B9
:1091F000030C8B420DD3FF22090212BA030C8B42DF
:1092000002D31212090265D0030B8B4219D300E07E
:10921000090AC30B8B4201D3CB03C01A5241830B03
:109220008B4201D38B03C01A5241430B8B4201D3B3
:109230004B03C01A5241030B8B4201D30B03C01ADC
:109240005241C30A8B4201D3CB02C01A5241830A56
:109250008B4201D38B02C01A5241430A8B4201D385
:109260004B02C01A5241030A8B4201D30B02C01AAF
:109270005241CDD2C3098B4201D3CB01C01A524116
:1092800083098B4201D38B01C01A524143098B429F
:1092900001D34B01C01A524103098B4201D30B0188
:1092A000C01A5241C3088B4201D3CB00C01A5241AD
:1092B00083088B4201D38B00C01A524143088B4272
:1092C00001D34B00C01A5241411A00D2014652410B
:1092D000104670475DE0CA0F00D04942031000D32A
:1092E0004042534000229C4603098B422DD3030A7F
:1092F0008B4212D3FC22890112BA030A8B420CD38F
:10930000890192118B4208D3890192118B4204D3B7
:1093100089013AD0921100E08909C3098B4201D337
:10932000CB01C01A524183098B4201D38B01C01A71
:10933000524143098B4201D34B01C01A52410309E8
:109340008B4201D30B01C01A5241C3088B4201D397
:10935000CB00C01A524183088B4201D38B00C01A44
:109360005241D9D243088B4201D34B00C01A52411B
:10937000411A00D20146634652415B10104601D3A8
:109380004042002B00D54942704763465B1000D332
:10939000404201B5002000F005F802BD0029F8D0D8
:1093A00016E770477047C046D0400B1C1141203A69
:1093B00003D49C46134118436346524293401843DA
:1093C0007047C0468446101C62468C46191C634692
:1093D00000E0C0461FB501F097F8002801D4002135
:1093E000C8421FBD10B500F0EFFF4042013010BD74
:1093F00010B501F089F8002801DB002010BD012024
:1094000010BDC04610B501F07FF8002801DD002036
:1094100010BD012010BDC04610B501F011F80028A4
:1094200001DC002010BD012010BDC04610B501F0C8
:1094300007F8002801DA002010BD012010BDC04649
:10944000F0B5CE46474615042D0C2E0080B5070416
:10945000140C3F0C9946030C7E435D436743634302
:109460007F19340CE4199C46A54203D980235B0282
:109470009846C4444B4643435143250C3604654447
:10948000360C2404A4195B19591820000CBC904612
:109490009946F0BDF0B54E4657464546DE46E0B526
:1094A00043025B0A450083B00F1C99462D0EC60F80
:1094B000002D57D0FF2D24D08020DB00C00418439E
:1094C000002381469A469B467F3D7C027A00FB0F33
:1094D000640A120E984623D0FF2A4BD0E300802462
:1094E0000020E4047F3A1C43AD186B1C47460193EF
:1094F000534677403A000F2B48D87D499B00CB5804
:109500009F46002B00D085E008339A46063B9B46D9
:109510007C027A00FB0FFF25640A120E9846DBD10D
:10952000002C00D090E0524601231A4392460120BD
:10953000DBE74C4658461700022824D0032800D108
:10954000CFE00022002301284DD15802D205400A65
:10955000FF071043384303B03CBC90469946A246EF
:10956000AB46F0BD002B5BD104239A46033B00259C
:109570009B46AAE7FF35002C60D1524602231A43CE
:1095800092460220B1E7FF220023DEE74B461B0C88
:109590009C464B462604360C180461463300220CC8
:1095A0006446000C43434E435043544380191A0C05
:1095B0001218964203D9802149028C4664441B0448
:1095C0001B0C1004C01883015E1EB341800E1843AB
:1095D000130C1B199B0103431C00230179D50123A4
:1095E00062081C401443019A7F32002A4DDD630754
:1095F00004D00F232340042B00D00434230103D5CF
:109600003C4B019A1C408032FE2ABCDCA3015B0A61
:10961000D2B29AE70C239A46093BFF259B4654E7B2
:10962000180001F071FE4A46431F76259A40002338
:109630006D4291462D1A9A469B4646E752460323B1
:109640001A439246032050E7200001F05DFE431FBD
:109650002D1A9C40763D002047E780230027DB033E
:10966000FF2272E7424666E74C463200584662E700
:1096700080234A46DB031A4222D01C4220D12343D6
:109680005B025B0A4746FF225FE701239A1A1B2A07
:1096900021DC23000199D3409E318C401A00230025
:1096A0005C1EA34113435A0704D00F221A40042A18
:1096B00000D004335A0111D49B015B0A002244E715
:1096C00080234A46DB0313435B025B0A3700FF2219
:1096D0003BE7019587E70022002336E701220023BC
:1096E00033E78023DB0323435B025B0AFF222CE783
:1096F00090E00000FFFFFFF770B500283DD0C317D2
:10970000C5185D40C40F280001F0FEFD9E22121A0C
:10971000962A07DCD2B2082833DD08388540680273
:10972000400A23E0992A0BDD052329001B1AD940A2
:1097300003001B339D402B005D1EAB4119430D0000
:10974000052801DD431F9D402B000F490B406E078C
:1097500009D00F263540042D05D004335D0102D514
:109760009F220B40121A9B01580AD2B24002D20526
:10977000400AE4071043204370BD0024002200206B
:10978000F4E76802400AF1E7FFFFFFFBF0B54F4640
:109790004646D6460C000903C0B5490A470F5E008D
:1097A00039431F03DB0F9C4665007B0A570F1F439D
:1097B0006D0DE40F760DA146C000B846D200AB1B7C
:1097C00064457BD0002B5FDD002E00D0A4E03E007E
:1097D000164300D112E15E1E002E00D09EE1871AD2
:1097E0004346B84280410125C91A4042091A0B027A
:1097F00000D431E149024E0A002E00D16EE1300062
:1098000001F082FD0300083B1F2B00DD61E12022F7
:109810003900D21A9E40D1409F400E439D4200DD48
:1098200051E15D1B6B1C1F2B00DD7CE12021C91A5F
:109830003D0030008F408840DD40791E8F4131006F
:1098400007222843D940002507433A40002A09D07F
:109850000F233B40042B05D03B1DBB42BF417F4241
:10986000C9191F000B0200D426E26A1CC64B55051D
:109870006D0D9A4200D106E1C44AFF080A40530721
:1098800052023B43120B8EE0002B00D0B8E06B1C61
:109890005B055B0D012B00DC30E1871A4346B842C3
:1098A000B641CB1A76429E1B330200D54CE13B00F9
:1098B0003343A1D100220024002570E0002B00DCFE
:1098C000E5E0002E00D183E0AF4EB54260D08026A7
:1098D00036043743B846382B00DC3EE14346134399
:1098E0001F007A1E97413F18874280414042091865
:1098F0000B0200D4B0E0A44B01359D4200D1C3E07F
:10990000A24A7B080A4001210F401F435108D30798
:1099100007221F433A4099E79B4EB54238D0802634
:1099200036043743B846382B00DDDCE01F2B00DC63
:1099300030E11E004746203EF740BC46202B04D0B5
:109940004026F31A46469E403243170063467A1E6D
:1099500097411F43CCE0002B00D104E24346134360
:1099600000D159E14B07C00818438023C9081B03E5
:10997000194208D04546ED081D4204D14346D0089F
:10998000590708432900420FC9007F4D1143C00009
:109990004B07CA087C49C00803438D4268D01203B4
:1099A0006D05120B6D0D002112031800130B0A0D2B
:1099B00012051A43764B2D0513402B435B00E40739
:1099C0005B08234319001CBC90469946A246F0BD93
:1099D0003E00164312D05E1E002E00D000E1871814
:1099E0008742804141444042091801250B0233D58A
:1099F000022585E764463300414610001D00C7E795
:109A0000002D00D0DAE00C000443F3D05C1C00D140
:109A10009FE15D4CA64200D12FE1DB43382B00DDF6
:109A200066E11F2B00DD83E120240500E41A0F000E
:109A3000DD40D940A0404346A7405B1A441EA041E8
:109A400098462F433843171ABA429241434652422E
:109A5000991A64463500CAE607223A40002A00D027
:109A6000F6E64B07CA084849FF083B438D4296D1AA
:109A70001900114300D19EE1802109030A4312031A
:109A8000120B414D8FE71500002200238BE7002BBE
:109A900000D0C7E06B1C5F057F0D012F00DCF1E0FB
:109AA000394DAB4200D1B9E085180A0085428941A1
:109AB0004244494251180722CF076D082F434908F5
:109AC0003A401D00C2E607223049ED1A31403A40C3
:109AD000BCE63E002838864000279FE6380001F0AB
:109AE00013FC20308EE6434613431F007A1E974135
:109AF000C71BB84280414042091A78E60E003B007D
:109B000006431343002D61D1002E00D0F4E0002B5A
:109B100000D11BE164463900100039E71A4FBB42FF
:109B20007AD03300FFE630001F3DE840202B03D001
:109B30004021CB1A9E4037437B1E9F41072207439B
:109B40003A400021002589E7171A4346BA42B64138
:109B5000591A76428E1B64464EE61F2B00DDADE09F
:109B600020264746F61AB740B9461700B246DF40EE
:109B70004E463E4337005646B240561EB24117434A
:109B80004246DA408918AEE6FF070000FFFF7FFF7C
:109B9000FFFF0F8020264746F61AB740B946170048
:109BA000B246DF404E463E4337005646B240561E50
:109BB000B24117434246DA40891A99E77F4CA642E0
:109BC0005BD0802424045B42214327E7002E0CD184
:109BD000002B00D1CBE0644639001000774DD7E66A
:109BE000764FBB4218D0330075E6002B14D04B07DC
:109BF000C00818438023C9081B03194207D0FC087A
:109C00001C4204D17907D0080843E14621004C46A4
:109C1000420FC9001143C000684DB9E61D00002283
:109C20000023C0E6002D5BD10D00054300D1E2E624
:109C30005D1C00D1B0E0614DAE421FD0DB43382B3C
:109C400071DC1F2B00DD96E020250F00ED1AAF40E0
:109C5000B9460700AA46DF404D463D432F00554612
:109C6000A840D940451EA84188440743BF189742E1
:109C700092415142414435003AE66446350041463E
:109C8000100085E60B000343002D00D063E6002B97
:109C9000F5D04346134300D17AE6871887428041C6
:109CA00007224144404209183A400B0200D4D5E64D
:109CB000434B01351940C9E5380069E61E004746A7
:109CC000203EF740BC46202B04D04026F31A4646DF
:109CD0009E403243170063467A1E97411F4302E6B7
:109CE000364DAE42CAD080252D045B422943A6E7FB
:109CF0000843411E8841A6E6002B00D148E6871A9A
:109D00004346B842B641CB1A76429E1B33024BD52E
:109D1000171A4346BA429241591A5242891A0722E7
:109D200064463A4092E501430F00791E8F419DE75A
:109D30001C000F00203CE740202B03D04024E31AF6
:109D400099400843411E884138437CE600220024A4
:109D500025E6171A4346BA429241591A5242891AC5
:109D60006446350043E541461000144D10E680225C
:109D70000024120380E61D000F00203DEF40BC468A
:109D8000202B03D04025EB1A994008430700634677
:109D9000781E87411F4369E7871897429B414144DA
:109DA0005B42C9183500A3E53B003343CED0072200
:109DB00031003A4052E600231A00F4E5FF070000A4
:109DC000FFFF7FFFF0B55746DE464E464546E0B5FD
:109DD000834607000E03480085B092461C00360BF0
:109DE000400DCD0F002800D19DE0954B984239D011
:109DF0008023F6001B041E43924A7B0F334399468F
:109E0000944603006344009300230026FF0002935E
:109E100023031B0B98466300E40F52465B0D01942D
:109E200000D1B3E086498B4200D19EE04246D1008A
:109E3000802212040A435146490F11438B4681493F
:109E400052468C4600996344CB1A0021D2000093FD
:109E50002B0063409A460F2E00D905E17A4BB600DD
:109E60009B599F465B463343994600D0B8E0022396
:109E70000826002700900293CAE7CB463A000299D1
:109E80000195019B9A46022927D0032900D180E23F
:109E9000012944D06D49009B8C4663441C00002C72
:109EA00038DD530700D013E2D2085B46DB0109D549
:109EB0005946674B19408B468021C9008C46009B50
:109EC00063441C00634B9C4207DC5B4664055F07F0
:109ED0005B0217431B0B620D02E000230027584A68
:109EE00000211B031C0B0B0D1B05234314055A4AB1
:109EF000380013401C4353466400DB0764081C43CE
:109F0000210005B03CBC90469946A246AB46F0BD48
:109F10000122524201231B1B382B00DCADE1002241
:109F200000230027DCE75B46334399465ED0002ED2
:109F300000D18AE1300001F0E7F903000B3B1C2B54
:109F400000DD7BE11D22D31A5A460100DA400839B0
:109F50008E4013005F46334399468F403F4B0026A7
:109F60001B1A00930023029352E7414653460B43CA
:109F70003B499B468C46009B634400935B46002B09
:109F80003BD1022300221E43022161E743461343D3
:109F90009B4637D04346002B00D162E1404601F09A
:109FA000B3F903000B3B1C2B00DD53E102004146DB
:109FB000083A914088461D21CB1A5146D9400B00E2
:109FC00041460B439B46534693401A00009B25494C
:109FD0009C46604403008C4663440093002137E7AD
:109FE0000323B14600900C26029311E7002300934F
:109FF00001330426002702930AE70323C3461E43C6
:10A00000032125E701331E430022012120E700231D
:10A010009A46802300271B03094A61E780234946AB
:10A020001B03194200D1E2E05946194200D0DEE09C
:10A030000B431B0317001B0BA246014A50E7C04607
:10A04000FF07000001FCFFFFD0E00000FF0300005D
:10A05000FFFFFFFEFE070000FFFF0F800DFCFFFF6C
:10A0600001F8FFFFF3030000D94500D9CBE000D190
:10A07000C6E03C0048460027009B013B00935B463E
:10A08000160E1B021E431302984633041B0C9946FE
:10A09000310C0191FFF798F84A4642430B04210C1A
:10A0A000050019438A4207D98919013D8E4203D818
:10A0B0008A4201D9851E8919881A0199FFF784F807
:10A0C00009048C464A46210464464243090C0300B5
:10A0D00021438A4204D98919013B8E4200D8F1E01C
:10A0E0002D041D43AB464346891A4246280C1204F0
:10A0F0001D0C5B46140C22001B041B0C5A430394DA
:10A100006B434443029568431B19150CEB189C42A2
:10A1100003D980246402A44660441C0C15041B046B
:10A120002D0C20185D19814277D373D00C1AA24AE6
:10A130007D1BAF42BF419446009B7F426344E01BBE
:10A140001C00864200D1DBE00199FFF73DF84A464A
:10A1500042430B04290C070019438A4207D9891985
:10A16000013F8E4203D88A4201D9871E8919881A75
:10A170000199FFF729F809044A46894629044D4602
:10A180004243090C030029438A4207D98919013B3C
:10A190008E4203D88A4201D9831E89193F04891A45
:10A1A0003A00039F1A43380013041B0C584381469E
:10A1B0000298150C6F43434345434846000C8446C0
:10A1C000DB1963449F4203D98020400284466544E2
:10A1D00048461F0C00041B04000C7D191818A942E6
:10A1E00000D284E000D17FE001231A4357E68023A8
:10A1F0004A461B0313431B031B0BAA466F4A6FE619
:10A20000BA4200D935E74B46DC0758087B081C43A7
:10A21000FF0734E70024AF4289D247444745A441B1
:10A220005B466442A4196418013BA6421ED2A042B8
:10A230006DD800D1B6E0241A9B4678E703005A4651
:10A24000283B9A400027914688E6584601F05CF882
:10A25000203072E603005246283B9A409346002283
:10A26000B4E6504601F050F820309AE6A642E2D11A
:10A27000B845DCD9341A9B4659E71F2B65DC504C96
:10A280000099A4465C46614408008C40110082405D
:10A29000D940501E82410C4314435A46DA40130001
:10A2A000620709D00F222240042A05D02200141D83
:10A2B0009442894149425B181A0262D50122002367
:10A2C00000270DE68A4200D80AE7831E891907E7AE
:10A2D0000F231340042B00D1E6E5171D974292414E
:10A2E00053429B44FA08E0E5002800D1D7E57118F5
:10A2F000531EB14227D3A94215D358D01A0073E791
:10A30000002B00DC04E6012300229B44CDE5022360
:10A310004744474589415B429C46494289190C198B
:10A32000E344241A03E743465F0047459B41B84690
:10A330005B429E19023A8919A94200D054E7404570
:10A3400000D051E7ABE51A00F6E71F215F4649420E
:10A350000C1BE740202B07D01A49009B8C46634416
:10A3600018005B4683401A43501E82413A43072738
:10A370000023174009D00F210023114014000429A5
:10A3800095D122005F075B021B0BD2081743002206
:10A39000A6E5802359461B030B431B0317001B0B29
:10A3A000064A9DE5BD42B2D89B460024BFE68045E3
:10A3B000B9D31A00C3E7C046FF030000FF0700003F
:10A3C0001E0400003E040000F0B54F464646D64647
:10A3D0008446C0B58046194E18030F034D00000B8C
:10A3E0005C0082463F0B6D0DC90F9146640DDB0F7B
:10A3F0000120B5420AD0B44203D0A54201D157454D
:10A400000CD01CBC90469946A246F0BD66463E4321
:10A41000F7D1AC42F5D154461443F2D10120C845DE
:10A42000EFD1994207D0002DEBD163461F4338008E
:10A43000471EB841E5E70020E3E7C046FF070000FC
:10A44000F0B54F464646D6464D00C0B50E03C90F7F
:10A450008A462C491F035C008046360B6D0D9146E1
:10A460003F0B640DDB0F8D421ED08C4216D0002DA9
:10A470001ED130438446002C01D13A4323D062469A
:10A48000002A1AD09A4529D05146022001390840A5
:10A4900001381CBC90469946A246F0BD39001143D4
:10A4A000E5D002204042F4E73043FAD1AC420FD06D
:10A4B000002C0FD13A43E7D00CE00122013B93433B
:10A4C00018000130E5E763460020002BE1D0DBE710
:10A4D0003A43E6D19A45D7D1A542D5DCA54205DB62
:10A4E000BE42D1D808D00020BE42D2D2504601236D
:10A4F000013898430130CCE7C845C5D80020C8458D
:10A50000F4D3C6E7FF070000F0B54F464646D646EF
:10A510004D00C0B50E03C90F8A462E491F035C00CB
:10A520008046360B6D0D91463F0B640DDB0F8D425F
:10A5300018D08C4211D0002D18D130438446002C05
:10A540001ED13A431CD163460020002B30D0514627
:10A5500002200139084001382AE039001143EAD0CD
:10A56000022025E03043FBD1AC4226D0002C26D17E
:10A570003A4324D15146022001390840013817E0FE
:10A580006246002A0FD09A45E1D1A54205DBBE42C2
:10A59000DDD819D00020BE420AD25046012301382E
:10A5A0009843013004E00122013B9343180001303D
:10A5B0001CBC90469946A246F0BD3A43D0D19A457C
:10A5C000C5D1A542C3DCE0E7C845C0D80020C845D6
:10A5D000E3D3EDE7FF070000F0B55746DE464E46F1
:10A5E0004546E0B5834606000F03480087B0924613
:10A5F0001D003F0B400DCC0F002800D16FE0DE4B5B
:10A60000984238D08023FF001B041F43730F3B4345
:10A610000193DA4B0027994600239B46F6008144BC
:10A620002B0369001B0B52469846490DED0F00297C
:10A6300000D185E0D04B994200D173E04346DA0067
:10A6400080231B0413435246CC48520F84461343C5
:10A65000524600206144D2008944210069400091A3
:10A660008C46012149448A460F2F00D990E0C44905
:10A67000BF00CF59BF465B463B43019300D06AE120
:10A6800002230827002681469B46C9E73200584628
:10A69000019B61460091022800D175E0032800D19A
:10A6A000FEE1012800D02CE1002300270026002530
:10A6B0003F032A0D3F0BB34812053A4302401B05E6
:10A6C0001343009A5B00D1075B080B43300019006D
:10A6D00007B03CBC90469946A246AB46F0BD5B46EF
:10A6E0003B43019300D12FE1002F00D1A5E13800B9
:10A6F00000F00AFE03000B3B1C2B00DD96E11D223F
:10A70000D31A5A460100DA405E4608398F401300DA
:10A710008E403B4301939C4B00271B1A9946002314
:10A720009B467DE7414653460B4393498C46E144A3
:10A73000002B00D01AE102220220174300228CE7EE
:10A74000134300D10DE14346002B00D181E1404687
:10A7500000F0DAFD02000B3A1C2A00DD72E1010074
:10A76000434608398B4098461D239A1A5346D340D6
:10A770001A004346134352468A404946081A824902
:10A7800089468144002068E77B4B002700268EE73E
:10A79000140C1204120C1100370C3604350C7943DA
:10A7A00028008C462E0060436044834656432100B7
:10A7B000300C80465846794340440291844506D97E
:10A7C0008846802149028C46E04441460291360485
:10A7D000010C360C00048B4681191E0C1B041B0C4B
:10A7E0000391190079438C46280075436544A846B7
:10A7F0005843050C45447743A94203D980214902B7
:10A800008C466744290C8C4639000004000C2D044A
:10A810002D186144AB4405915946049101990F04E8
:10A820003F0C080C390051434243904602008C46CD
:10A83000090C8B4662437C4344445C44A04503D9E5
:10A840008021490288464244210C88466146090419
:10A85000090C8C4639005943434370437E430F0C27
:10A86000F6182404BE19644442448C46B34203D90A
:10A8700080235B0298464044029B61469846049BB5
:10A88000370443449B46AB45AD416B420D040599EB
:10A890002D0C8C467F196744FD18A8465D462D197E
:10A8A000A542A44193466442A446C344DC448F427B
:10A8B000BF4198459B4193459241A445A4415B42C9
:10A8C0007F421F43360C52426442BF192243BF18D5
:10A8D000624638184302D20D039913436A020A43B1
:10A8E000501E82416146ED0D2A434E023243D9018A
:10A8F00000D4B3E00126500832400243DE07324361
:10A900005B08224C5444002C62DD510709D00F2013
:10A910001040042805D0101D9042924152429B18CD
:10A920000200D90104D580241948E40003405444AE
:10A930001848844200DD27E75E075B02D2081F0B40
:10A94000630516435B0DB2E60023994601330427E5
:10A9500000269B4664E60323019781460C279B460D
:10A960005EE6012201201743002276E6032303203E
:10A970001F43434671E6C046FF07000001FCFFFF8E
:10A9800010E10000FFFF0F800DFCFFFFFF03000040
:10A99000FFFFFFFEFE0700000023802700933F0318
:10A9A0000026434B83E6019B3200A446584670E6DE
:10A9B000AC466EE6802701993F0339422DD03B42D9
:10A9C0002BD11F433F033F0B00951600384B6EE61B
:10A9D00001252D1B382D00DD66E61F2D40DC354896
:10A9E0001C005044160082408440EE40501E8241BC
:10A9F00034431443EB40620709D00F222240042A5B
:10AA000005D02200141D9442804140421B181A02B6
:10AA10003ED501230027002649E68027019B3F03FE
:10AA20001F433F033F0B0094214B40E603005A466F
:10AA3000283B9A40002601926DE6584600F064FCDF
:10AA4000203057E603005246283B9A40130000226C
:10AA500093E6504600F058FC20307BE6CA4650E7AB
:10AA60001F201E004042041BE640202D03D0124C44
:10AA70005444A3401A43501E824132430726002704
:10AA8000164009D00F200023104014000428B9D12B
:10AA900022005E075B021F0BD2081643002306E666
:10AAA00080273F031F433F033F0B1600004BFEE58B
:10AAB000FF0700001E0400003E040000F8B55746E2
:10AAC0004E464546DE460C000903E0B5490A460FEE
:10AAD0005F0031431E03DB0F760A9B46530F33435F
:10AAE000C84E6500C000E40FD2006D0DA24681463D
:10AAF0007F0D9C469046B74200D1B9E05B460126E7
:10AB000073409B46EE1BA34500D183E0002E63DD1E
:10AB1000002F00D0B1E06346134300D123E1731E40
:10AB2000002B00D0BAE1861A6346B042804101256D
:10AB3000C91A4042091A0B0200D447E149024B0AE4
:10AB400098464346002B00D189E1404600F0DCFBEB
:10AB50000300083B1F2B00DD7CE120223000D21ACD
:10AB60004146D040994002009E400A439D4200DD8C
:10AB70006AE15D1B6B1C1F2B00DD94E1202110009E
:10AB80003500C91A8E40DA408840DD40711E8E4182
:10AB9000110007222843002506433240002A09D02D
:10ABA0000F233340042B05D0331DB342B641764208
:10ABB00089191E000B0200D43DE26A1C914B550519
:10ABC0006D0D9A4200D119E18F4AF6080A405707E5
:10ABD00052023743120B9BE0002E00D0C5E06E1CE2
:10ABE0007605760D012E00DC48E16746861ACB1B00
:10ABF000B042BF417F42B8461F004346FF1A3B00A8
:10AC0000B8461B0200D55FE137439AD100220024E9
:10AC1000002579E0002E00DCFAE0002F00D18DE065
:10AC2000784B9D4267D0802367461B041F43BC4678
:10AC3000382E00DC52E1634613435A1E93411E181E
:10AC400086428041404209180B0200D4BEE06D4BA1
:10AC500001359D4200D1D2E06B4A73080A400121C0
:10AC60000E401E435108D30707221E43324095E78A
:10AC70001E00164300D045E740E7624B9D423AD0A4
:10AC8000802367461B041F43BC46382E00DDEBE0E3
:10AC90001F2E00DC3AE133006746203BDF403B00DB
:10ACA000202E05D04027BF1B6646BE40324390464B
:10ACB0004646721E96413343DAE0002B00D114E27F
:10ACC0006346134300D168E180234E07C008C908DA
:10ACD0001B030643194208D06046C008184204D13D
:10ACE00063460100D2085E071643F3009946C90087
:10ACF000720F444D11434B46DE08424B4F0737431A
:10AD0000CA089D4200D16EE012036D05120B6D0D55
:10AD100000211203130B0A0D12051A433B4B2D059C
:10AD200013402B435B00E4075B0823433800190002
:10AD30003CBC90469946A246AB46F8BD63461343D9
:10AD400011D0731E002B00D007E186188642804187
:10AD500061444042091801250B0237D502257BE7E3
:10AD60003E00614691463500C5E75C46002D00D0A7
:10AD7000E1E00B000343F3D0731C00D1ACE1214BA5
:10AD80009F4200D13AE1F343382B00DD6FE11F2BE6
:10AD900000DD8CE120250E00ED1AAE40B046060025
:10ADA000AA46DE40454635432E005546D940A840C8
:10ADB0006346451EA8415B1A9C463043161AB242B0
:10ADC000924163465242991A3D00B4E6072232404E
:10ADD000002A00D0E4E60B4BF6084F073743CA08B9
:10ADE0009D4200D090E73B00134300D1A6E18023B1
:10ADF0001B031A431203120B024D89E715000022B0
:10AE0000002785E7FF070000FFFF7FFFFFFF0F80A0
:10AE1000002E00D0C7E06B1C5E05760D012E00DC15
:10AE2000F0E0C84DAB4200D1B9E085180A00854278
:10AE300089416244494251180722CE076D082E43CA
:10AE4000490832401D00A9E6BF49ED1A114007220A
:10AE50003240A3E6320028388240002686E63000E1
:10AE600000F052FA203073E6634613435A1E9341B2
:10AE7000C61AB04280414042091A5CE60E0067469D
:10AE800006431743002D5ED1002E00D0F3E0002FC3
:10AE900000D11EE15C46614691462CE7A94FBE42B7
:10AEA0007BD01E00F1E610001F3DE840202B03D0B0
:10AEB0004021CB1A9A401643731E9E410722064337
:10AEC00032400021002583E7161A6346B2428041D2
:10AED000591A40420B1A98465C4632E61F2E00DD96
:10AEE000ABE02027BB1B9A4663465746BB409946BA
:10AEF00013004F46F3401F433B005746BA40571ECE
:10AF0000BA4113436246F240891898E62027BB1BDA
:10AF10009A4663465746BB40994613004F46F34056
:10AF20001F433B005746BA40571EBA41134362467F
:10AF3000F240891A9CE7834B9F425FD080252D0405
:10AF40007342294320E7002E0CD1002F00D1D0E01E
:10AF50005C46614691467B4DCDE67A4FBE421CD0A1
:10AF60001E0065E6002F18D0C0084E07064380205B
:10AF7000C9080003014208D06346DC08044204D13A
:10AF80002100DA46D2085E071643F30099460124F1
:10AF90005346C900720F11431C406A4DABE61D00B9
:10AFA00000220027B4E6002D59D10B00034300D145
:10AFB000D6E6731C00D1B2E0624B9F421ED0F34331
:10AFC000382B6FDC1F2B00DD97E020250E00ED1ADB
:10AFD000AE40B0460600AA46DE40454635432E0048
:10AFE0005546A840D940451EA8418C440643B61892
:10AFF00096429241514261443D0025E63D00614642
:10B00000914678E60B000343002D00D055E6002B57
:10B01000F5D06346134300D16DE686188642804121
:10B0200061444042091800220B0200D4D0E6464B8E
:10B0300001351940B2E5B1465DE633006746203B75
:10B04000DF403B00202E05D04027BF1B6646BE4098
:10B05000324390464646721E96413343EFE5394BE4
:10B060009F42CBD080252D0473422943A8E7084393
:10B07000411E8841A2E6002F00D13CE66346861AB5
:10B08000CF1AB0429B415B42FB1A98461B024ED539
:10B09000161A6346B2429241591A5242891A5C46C4
:10B0A00000227BE501430E00711E8E419FE71D00CB
:10B0B0000E00203DEE40B046202B04D04025EB1A78
:10B0C00099400843814648464346411E88411843FB
:10B0D00074E60022002417E6161A6346B242924133
:10B0E000591A5242891A3D0025E561469146154D8F
:10B0F00001E680220024120379E61D000E00203DA7
:10B10000EE40B046202B04D04025EB1A994008436E
:10B1100081464E464346711E8E411E4367E78618A0
:10B1200096429B4161445B42C9183D008CE547460D
:10B130003743CED007224146324049E600273A0045
:10B14000E6E5C046FF070000FFFF7FFF70B50C4E2D
:10B150000D031C0349005B002D0B490D240B5B0DF7
:10B16000B14208D0064900208B4203D1144320008D
:10B17000441EA04170BD05430120002DFAD1F1E726
:10B18000FF07000030B5144D0A034B00120B5B0D96
:10B19000C90F0024AB4211DD104CA34210DC802407
:10B1A000640322430E4CE41A1F2C0CDD0D48C31A15
:10B1B000DA4013005C42002900D11C00200030BDA1
:10B1C000094BCC18FAE7094DE040AC4663449A407D
:10B1D00013000343EEE7C046FE0300001D04000019
:10B1E0003304000013040000FFFFFF7FEDFBFFFFAF
:10B1F00070B500282DD0C317C5185D40C40F2800B6
:10B2000000F082F8154B1B1A5B055B0D0A2815DD53
:10B210000B38854000222D032D0B002110002D033B
:10B220000A0D2D0B12052A430D4D1B052A40134311
:10B230005B00E4075B082343190070BD020029008E
:10B24000153291400A000B21081AC5402D032D0B21
:10B25000E3E70024002300250022DEE71E040000AF
:10B26000FFFF0F804100090E4B1C70B5DBB2460298
:10B27000750AC40F012B14DDE0239B006D07360B0C
:10B28000CB1800210A0D280012051C4D32435B0526
:10B290002A405B0813435B00E4075B082343190063
:10B2A00070BD002914D1002D1ED0280000F02CF80C
:10B2B0000A281CDC0B232A001B1ADA400300153372
:10B2C0009D400F4B12031B1A5B05160B5B0DD8E755
:10B2D000002D06D0320B802636036D071643094B2E
:10B2E000CFE7084B0026CCE700230026C9E7030080
:10B2F0002A000B3B9A400025E3E7C046FFFF0F8082
:10B3000089030000FF0700001C2101231B04984251
:10B3100001D3000C10391B0A984201D3000A0839E6
:10B320001B09984201D30009043902A2105C40189D
:10B330007047C04604030202010101010000000041
:10B340000000000030B51C00094B05001B6885B0EB
:10B35000D868084B002A01D1074B1A0002920193CA
:10B3600000912B002200054900F026F800F0A6FD10
:10B370007C00002050E100008BCF00005DE1000068
:10B38000014B18687047C0467C000020084B10B580
:10B390000400002B02D0002100E000BF054B18681C
:10B3A000836A002B00D09847200001F05DFBC04667
:10B3B000000000008CE100000EB403B5010003ABF7
:10B3C000044804CB0068019300F076F802B008BC92
:10B3D00003B018477C00002070B500260C4D0D4CC2
:10B3E000641BA410A64209D1002601F03FFB0A4DC0
:10B3F0000A4C641BA410A64205D170BDB300EB58E3
:10B4000098470136EEE7B300EB5898470136F2E76C
:10B410004C0200204C0200204C0200205C02002064
:10B42000002310B59A4200D110BDCC5CC454013346
:10B43000F8E710B5884202D98B18984203D300234D
:10B4400007E08B5C8354013AFBD210BDCC5CC45442
:10B4500001339A42FAD1F8E703001218934200D15F
:10B46000704719700133F9E7936810B5013B936099
:10B47000002B04DA9469A34207DB0A2905D013687C
:10B48000581C10601970080010BD00F04BFC010042
:10B49000F9E7F8B506000F001400D518AC4201D149
:10B4A000002007E021783A003000FFF7DDFF01348B
:10B4B000431CF3D1F8BD0000F0B59FB002900F001F
:10B4C00016000593002805D083690493002B01D151
:10B4D00000F0F4FD7B4B9F425BD1029B5F68BB8910
:10B4E0001B0762D53B69002B5FD0002306AC63616C
:10B4F000203363761033A37635002B78002B01D0F0
:10B50000252B5CD1AB1B04930CD032003900029880
:10B51000FFF7BFFF431C00D1C4E06269049B94465F
:10B52000634463612B78002B00D1BBE00122002330
:10B530005242626002A9543252186E1C2360E360CA
:10B54000A3601370A365317805225F4800F0D4FE34
:10B55000751C002835D12268D30604D5532302A9CF
:10B560005B1820211970130704D5532302A95B1817
:10B570002B21197033782A2B2CD0350000210A207A
:10B58000E3682A786E1C303A092A64D900292ED043
:10B5900026E04E4B9F4202D1029B9F689FE74C4B97
:10B5A0009F429CD1029BDF6899E73900029800F026
:10B5B0000FFC002899D0012040421FB0F0BD01359A
:10B5C0009BE7414B2268C01A012383401343236049
:10B5D0002E00B8E7059B191D1B680591002B01DBA8
:10B5E000099304E05B42E3600223134323602B785A
:10B5F0002E2B0AD16B782A2B35D1059B02351A1DCB
:10B600001B680592002B2BDB0793324E297803220F
:10B61000300000F071FE002806D04023801B8340DC
:10B620002268013513432360297806222A486E1CBC
:10B63000217600F061FE00283AD0284B002B25D15E
:10B640000722059B07339343083305936369039AE5
:10B650009B18636150E7434301219B18350090E735
:10B6600001235B42D0E700230A201A000135636002
:10B6700029786E1C3039092903D9002BC5D00792CF
:10B68000C3E74243012352183500F1E705AB0093AD
:10B690003A00134B2100029800E000BF0390039B87
:10B6A0000133D3D1BB895B0600D584E70B9884E7CF
:10B6B00005AB00933A000A4B2100029800F080F895
:10B6C000ECE7C046E4E1000090E1000004E2000085
:10B6D000C4E1000096E100009AE1000000000000D3
:10B6E00093B40000F7B5150001938A680B690090C8
:10B6F0000C00934200DA130022002B6043321278D0
:10B70000002A01D001332B6023689B0602D52B68E9
:10B7100002332B60062723681F4027D023004333C2
:10B720001B785A1E93412268920630D42200019958
:10B7300043320098089EB047431C25D0062320685A
:10B740002A68E16803400025042B03D18D1AEB43DE
:10B75000DB171D40A3682269934201DD9B1AED1897
:10B760000027BD4220D1002010E00137E3682A689D
:10B770009B1ABB42D2DD22000123193201990098A5
:10B78000089EB047431CF0D101204042FEBD30204E
:10B79000E1184331087021005A1C45310978A2187C
:10B7A000433202331170C1E7220001231A3201999A
:10B7B0000098089EB047431CE6D00137D1E700004F
:10B7C000F0B589B004920A004332059303900292C7
:10B7D0000A7E0C000E9B6E2A00D186E01FD8632AD9
:10B7E00033D008D8002A00D18CE0582A4DD025004B
:10B7F00042352A7030E0642A01D0692AF7D11968ED
:10B8000025680A1D280629D508681A60002803DA69
:10B810002D23029A404213706B4E0A274FE0732A81
:10B8200074D008D86F2A1FD0702AE0D1202209686E
:10B830000A43226003E0752A16D0782AD7D1220065
:10B84000782145321170614E22E025001A68423598
:10B85000111D196013682B70012365E008681A60D8
:10B860006906D3D500B2D1E719682568081D1860AC
:10B8700008682E0605D5544E08276F2A1BD00A27C4
:10B8800019E06D06F7D580B2F5E745314E4E0A70E6
:10B8900018682268011D00681960150621D5D307B4
:10B8A00002D520231A4322601027002803D1202329
:10B8B00022689A4322602300002243331A7063688F
:10B8C000A360002B58DB04222168914321600028EB
:10B8D00054D1029D002B5AD02500337842352B706D
:10B8E00055E05506DBD580B2D9E71A680D68101D02
:10B8F0004969186013682E0601D5196002E06D06CB
:10B90000FBD519800023029D23614FE01A68111DA9
:10B910001960156800216268280000F0EDFC00281D
:10B9200001D0401B6060636823610023029A13709A
:10B930003CE023692A0004990398059DA847431C0D
:10B940003ED023689B0715D4079BE068984239DAFC
:10B95000180037E022000123193204990398059E4C
:10B96000B047431C2CD00135E368079A9B1AAB42C1
:10B97000F0DCE9E70025F7E70028ADD0029D3900AB
:10B98000FDF722FC735C013D2B700028F7D1082FD6
:10B9900009D12368DB0706D563682269934202DC7C
:10B9A0003023013D2B70029B5B1B2361059B07AA83
:10B9B00000932100049B0398FFF794FE431CB8D129
:10B9C0000120404209B0F0BDA1E10000B2E1000059
:10B9D0000D4B70B51C680500A36B002B0FD1182010
:10B9E00000F06EFC094BA0630360094B0122436029
:10B9F000084B83600B238381002302614361002293
:10BA0000A36B1D615A6170BD7C0000200E33CDAB6D
:10BA100034126DE6ECDE0500124B10B51C68A36B0A
:10BA2000002B0FD1182000F04BFC0F4BA0630360DC
:10BA30000E4B012243600E4B83600B238381002356
:10BA400002614361A46B0B4A206961690A4BFDF7EF
:10BA5000F7FC0122002380185941206161614800F0
:10BA6000400810BD7C0000200E33CDAB34126DE6D3
:10BA7000ECDE05002D7F954C2DF451580CB430B5FB
:10BA8000164B9DB00C1E1D6808DA8B2301202B601D
:10BA900040421DB030BC08BC02B01847822302A946
:10BAA0009B008B810023029008619C4200D0631EA2
:10BAB0008B604B6101235B42CB81209A21AB280034
:10BAC000019300F055FD431C01DA8B232B60002C01
:10BAD000DFD00023029A1370DBE7C0467C00002011
:10BAE0000EB400B50B499CB01DAB029006900791B7
:10BAF00004910948094904CB0591006802A9019302
:10BB000000F036FD0023029A13701CB008BC03B08D
:10BB10001847C046FFFFFF7F7C0000200802FFFFA0
:10BB2000020010B51378541C002B05D1CC5CD45402
:10BB30000133002CFAD110BD2200F3E7C9B203781B
:10BB4000002B04D08B4200D170470130F7E74B4205
:10BB5000594149420840F7E702780B78002A03D0A0
:10BB6000013001319A42F7D0D01A70470023C25CED
:10BB70000133002AFBD1581E7047002330B59A428A
:10BB80000AD0013AC45CCD5CAC4204D1934202D0ED
:10BB90000133002CF6D1631B180030BD30B5050011
:10BBA000002A00D130BD0C78013A6B1C2C70013199
:10BBB000002C05D19A189A42F4D01C700133FAE790
:10BBC0001D00EDE710B50378002B0FD10B785A421A
:10BBD00053415B42184010BD0023CA5C002AFAD0D2
:10BBE000C45C944201D10133F7E701300378002BA4
:10BBF000F2D11800EFE70000F0B51F000E0087B08B
:10BC00000590019102920C98347800F0EAFA08222B
:10BC100000194378751C134036D12D2C36D1B51C34
:10BC200074780126002F62D0102F09D1302C07D153
:10BC300020222B789343582B54D110276C7802354F
:10BC40002D4B3900F31818000393FDF7BDFA04914A
:10BC500001210023494202008C461800210030399E
:10BC600009291AD80C00A74223DD591C09D06346C4
:10BC7000824206D302D10499A14202DB0123784318
:10BC800020182C780135E9E72E00BCE72B2C01D0D9
:10BC90001E00C7E7B51C7478FAE72100413919295D
:10BCA00001D8373CDFE721006139192901D8573C19
:10BCB000D9E75A1C08D1059A23331360029B0398D5
:10BCC000002B09D107B0F0BD002E00D04042029AEF
:10BCD000002AF7D0002B01D06B1E0193029B019A22
:10BCE0001A60EFE73024002FAAD10827A8E7302CEC
:10BCF0009ED00A27A4E7C046FFFFFF7F37B5130099
:10BD0000064A05001068046A002C00D1044C0A00A1
:10BD100000942900FFF770FF3EBDC0467C00002064
:10BD2000E0000020F8B505000E001400002804D043
:10BD30008369002B01D100F0C1F9224B9C422DD127
:10BD40006C68A369A360A3891B0731D52369002B05
:10BD50002ED023682269F7B2981A6369F6B283423B
:10BD600005DC2100280000F03BF9002826D1A3685B
:10BD70000130013BA36023685A1C22601F70636975
:10BD8000834204D0A389DB071AD50A2E18D12100DB
:10BD9000280000F025F9002812D00FE00A4B9C4241
:10BDA00001D1AC68CDE7094B9C42CAD1EC68C8E729
:10BDB0002100280000F00CF80028CAD001267642A5
:10BDC0003000F8BDE4E1000004E20000C4E100003E
:10BDD000364B70B51D6806000C00002D05D0AB6910
:10BDE000002B02D1280000F069F9314B9C420FD1A1
:10BDF0006C680C23E25E93B219072DD4D90611D4D6
:10BE000009230120336037331343A381404270BDBF
:10BE1000284B9C4201D1AC68EBE7274B9C42E8D110
:10BE2000EC68E6E75B0713D5616B002908D02300B7
:10BE30004433994202D0300000F06AFA0023636371
:10BE40002422A3899343A381002363602369236091
:10BE50000823A2891343A3812369002B0BD1A021BE
:10BE60008022A389890092000B40934203D02100D5
:10BE7000300000F0E1F90123A289134011D0002322
:10BE8000A36063695B42A361002023698342BED142
:10BE90000C23E25E1306BAD540231343A381013875
:10BEA000B5E7920700D46369A360EDE77C0000204A
:10BEB000E4E1000004E20000C4E1000010B5062047
:10BEC00000F090FC012000F0CFFD0000F7B58A895A
:10BED00005000C00130760D44B68002B04DC0B6CCE
:10BEE000002B01DC0020FEBDE76A002FFAD0002302
:10BEF0002E682B6080235B01216A1A4034D0606D6C
:10BF0000A3895B0706D56368C01A636B002B01D059
:10BF1000236CC01A0200216A00232800E76AB84790
:10BF2000A189431C06D12B681D2B30D82B4ADA403F
:10BF3000D3072CD50023636023692360CB0405D588
:10BF4000431C02D12B68002B00D16065616B2E6011
:10BF50000029C7D023004433994202D0280000F0C2
:10BF6000D7F900206063BEE701232800B847431CCF
:10BF7000C6D12B68002BC3D01D2B01D0162B01D1AD
:10BF80002E60AFE74023A2891343A381ABE7402390
:10BF90000B430120A3814042A5E70F69002FA1D0E8
:10BFA0000B680F60DB1B01930023920700D14B69E4
:10BFB000A360019B002B00DC94E7019B3A00216AFF
:10BFC0002800A66AB047002803DC4023A289134357
:10BFD000DFE7019B3F181B1A0193EAE701004020AD
:10BFE0000B6970B505000C00002B01D1002070BD5D
:10BFF000002804D08369002B01D100F05FF80B4BBF
:10C000009C4209D16C680C22A35E002BEED021006B
:10C010002800FFF75BFFEAE7054B9C4201D1AC68C3
:10C02000F1E7044B9C42EED1EC68ECE7E4E1000060
:10C0300004E20000C4E10000002310B50400036026
:10C040004360836081814366C28103614361836190
:10C05000190008225C30FFF7FFF9054B2462636288
:10C06000044BA362044BE362044B236310BDC04640
:10C0700025C800004DC8000085C80000B1C80000F8
:10C0800010B5024900F08CF810BDC046E1BF0000B9
:10C0900070B568254A1E55430E002900743100F022
:10C0A00081F9041E08D000212A00016046600C308E
:10C0B000A0606832FFF7D0F9200070BD836913B526
:10C0C0000400002B28D18364C3640365134B144A16
:10C0D0001B6882620193984201D101238361200091
:10C0E00000F020F86060200000F01CF8A060200044
:10C0F00000F018F80022E06004216068FFF79CFF60
:10C1000001220921A068FFF797FF02221221E068AF
:10C11000FFF792FF0123A36113BDC0468CE100002D
:10C1200081C00000F8B51C4B07001E68B369002BE6
:10C1300002D13000FFF7C2FF4836B4687368013B94
:10C1400004D53368002B07D03668F6E70C22A55ECD
:10C15000002D0DD06834F2E704213800FFF798FF76
:10C1600030600028F0D10C2304003B602000F8BDB3
:10C1700020000A4B656625606560A560E360256167
:10C180006561A561082229005C30FFF765F96563E8
:10C19000A563A564E564E9E78CE100000100FFFF09
:10C1A000F7B504000700002601914834002C01D1A6
:10C1B0003000FEBD6368A5680093009B013B0093BF
:10C1C00001D52468F2E7AB89012B08D90E22AB5EBA
:10C1D000013304D029003800019B98470643683595
:10C1E000EBE7EC300068704770B50E001D000E23C1
:10C1F000C95E96B01400002907DA00232B60B389CA
:10C200001B0611D48023DB000FE06A4600F088FB98
:10C210000028F2DBF022019B12021340054A9B1812
:10C220005A4253412B60EDE740230020236016B0B3
:10C2300070BDC04600E0FFFFF7B502268B89050000
:10C240000C00334206D023004733236023610123CF
:10C250006361F7BD01AB6A46FFF7C6FF00990700AF
:10C26000280000F09FF8002808D10C22A35E9A0550
:10C27000EFD4032293431E43A681E4E70F4BAB6246
:10C280008023A28920601343A381009B2061636106
:10C29000019B002B0DD00E23E15E280000F052FB25
:10C2A000002806D00322A38993431A0001231343D5
:10C2B000A381A0893843A081CBE7C04681C000009C
:10C2C00010B5034B0100186800F06CF810BDC046B3
:10C2D0007C00002082B0002900D101A9101E06D0E8
:10C2E000002B06D013780B601078431E984102B0E3
:10C2F000704702204042FAE7C9B28218904201D149
:10C300000020704703788B42FBD00130F6E7000035
:10C3100070B50500002910D00C1F2368002B00DA2F
:10C32000E418280000F034FB1D4A1368002B05D1E7
:10C3300063601460280000F02CFB70BDA34209D993
:10C34000216860188342F3D118685B684118216046
:10C35000EEE713005A68002A01D0A242F9D9196801
:10C360005818A0420BD12068091858181960824249
:10C37000E0D110685268411819605A60DAE7A042AB
:10C3800002D90C232B60D5E721686018824203D1C3
:10C39000106852684118216062605C60CAE7C0465C
:10C3A0001C1C0020032370B5CD1C9D4308350600DE
:10C3B0000C2D1ED20C25A9421DD8300000F0E8FA41
:10C3C000254A14682100002919D1244C2368002B28
:10C3D00003D1300000F0CAF920602900300000F0DD
:10C3E000C5F9431C2BD10C233000336000F0D1FA87
:10C3F00003E0002DDFDA0C233360002070BD0B68F2
:10C400005B1B19D40B2B03D90B60CC18256003E000
:10C410004B688C420DD11360300000F0BAFA200056
:10C4200007220B30231D9043C31AE7D05A42E25033
:10C43000E4E763600C00EFE70C004968C3E70323FF
:10C44000C41C9C43A042E1D0211A300000F08EF9B8
:10C45000431CDBD1C7E7C0461C1C0020201C002069
:10C46000F8B507000D001600002905D11100FFF7EF
:10C4700099FF04002000F8BD002A03D1FFF748FF10
:10C480003400F7E700F086FA2C00B042F2D2310017
:10C490003800FFF787FF041EECD029003200FEF7BA
:10C4A000BFFF29003800FFF733FFE3E7F0B58E68E0
:10C4B00085B007000C00039201939E423CD8902364
:10C4C0008A89DB001A4234D00325096923685B1A84
:10C4D0000293636902985D43EB0F5D19019B6D1038
:10C4E00001331B18AB4200D91D00530532D529007A
:10C4F0003800FFF757FF061E09D10C233B6040238D
:10C500000120A28940421343A38105B0F0BD029AE5
:10C510002169FEF785FFA389144A1A40802313433B
:10C52000A381029B2661F61826606561019EED1AC3
:10C53000A560019B9E4200D9019E320003992068AC
:10C54000FEF777FFA36800209B1BA36023689E195A
:10C550002660DAE72A003800FFF782FF061EE0D1E6
:10C5600021693800FFF7D4FEC7E7C0467FFBFFFF15
:10C57000F0B59FB0029005938B890F0016001B0643
:10C5800011D50B69002B0ED14021FFF70BFF38604E
:10C590003861002805D10C23029A013813601FB0BE
:10C5A000F0BD40237B61002306AC636120336376DA
:10C5B0001033A37635002B78002B01D0252B46D1E4
:10C5C000AB1B04930CD0320039000298FFF76EFFCA
:10C5D000431C00D1AEE06269049B944663446361EE
:10C5E0002B78002B00D1A5E001220023524262608B
:10C5F00002A9543252186E1C2360E360A3601370CA
:10C60000A365317805225448FFF776FE751C002893
:10C610001FD12268D30604D5532302A95B18202119
:10C620001970130704D5532302A95B182B21197025
:10C6300033782A2B16D0350000210A20E3682A78A7
:10C640006E1C303A092A4ED9002918D010E0013565
:10C65000B1E7414B2268C01A012383401343236092
:10C660002E00CEE7059B191D1B680591002B01DBF1
:10C67000099304E05B42E3600223134323602B78B9
:10C680002E2B0AD16B782A2B35D1059B02351A1D2A
:10C690001B680592002B2BDB0793304E2978032271
:10C6A0003000FFF729FE002806D04023801B83407E
:10C6B00022680135134323602978062228486E1C1E
:10C6C0002176FFF719FE00283CD0264B002B25D100
:10C6D0000722059B07339343083305936369039A45
:10C6E0009B18636166E7434301219B183500A6E769
:10C6F00001235B42D0E700230A201A000135636062
:10C7000029786E1C3039092903D9002BC5D007922E
:10C71000C3E74243012352183500F1E705AB00930C
:10C720003A00114B2100029800E000BF0390039BE8
:10C730000133D3D1BB890B985B0600D42FE70120CE
:10C7400040422CE705AB00933A00074B21000298CA
:10C75000FFF736F8EAE7C04690E1000096E10000F6
:10C760009AE1000000000000ADC40000002370B595
:10C77000064C05000800236000F060F9431C03D15B
:10C780002368002B00D02B6070BDC046B02F002066
:10C7900070B504000D001F2904D916230360012081
:10C7A000404270BD436C002B04D08A009B181A686D
:10C7B000002A08D1200000F031F82A0001002000F2
:10C7C00000F01AF8EDE70020012AEAD0511C03D14D
:10C7D000162301302360E4E7002428001C60904702
:10C7E0002000DEE710B5034B01001868FFF7D0FF0B
:10C7F00010BDC0467C000020002370B5064C05002B
:10C8000008001100236000F001F9431C03D12368E4
:10C81000002B00D02B6070BDB02F002010B500F0B1
:10C82000E5F810BD70B50C000E25495F00F0BAF8B0
:10C83000002803DB636D1B18636570BDA389024A82
:10C840001340A381F9E7C046FFEFFFFFF8B51F00D3
:10C850008B8905000C001600DB0505D50E23C95E8B
:10C860000022022300F080F8A389054A2800134023
:10C87000A38132000E23E15E3B0000F02BF8F8BDEF
:10C88000FFEFFFFF70B50C000E25495F00F06CF85C
:10C89000A389421C03D1054A1340A38170BD8022A5
:10C8A00052011343A3816065F8E7C046FFEFFFFF25
:10C8B00010B50E23C95E00F021F810BD0B1E04D088
:10C8C000FF2A04D98A2303608B3B180070470A7043
:10C8D0000123FAE770B50500080011000022064C9C
:10C8E00022601A0000F0B8F8431C03D12368002B23
:10C8F00000D02B6070BDC046B02F0020002370B563
:10C90000064C05000800236000F060F8431C03D1CA
:10C910002368002B00D02B6070BDC046B02F0020D4
:10C92000002370B5064C050008001100236000F0DC
:10C9300055F8431C03D12368002B00D02B6070BD39
:10C94000B02F0020002370B5064C050008002360BE
:10C9500000F054F8431C03D12368002B00D02B6057
:10C9600070BDC046B02F002070B505000800110052
:10C970000022064C22601A0000F050F8431C03D13C
:10C980002368002B00D02B6070BDC046B02F002064
:10C99000704770470B1F1B68181F002B01DA0B58DC
:10C9A000C018704770B50500080011000022064C41
:10C9B00022601A0000F03AF8431C03D12368002BD0
:10C9C00000D02B6070BDC046B02F0020582201203F
:10C9D000014B40421A607047B02F002058220120BE
:10C9E000014B40421A607047B02F002058220120AE
:10C9F000014B40421A607047B02F00205822024B72
:10CA000000201A607047C046B02F00205822012035
:10CA1000014B40421A607047B02F0020582201207D
:10CA2000014B40421A607047B02F0020582201206D
:10CA3000014B40421A607047B02F0020044A13682F
:10CA4000002B00D1034B1818106018007047C04627
:10CA5000241C0020B82F002058220120014B404206
:10CA60001A607047B02F0020FEE7C046F8B5C046F8
:10CA7000F8BC08BC9E467047F8B5C046F8BC08BC78
:10CA80009E467047646174610000000008CB00009E
:10CA9000EF01000011CB0000E302000019CB000001
:10CAA0000909000020CB0000190A000025CB000076
:10CAB0003105000030CB00005303000035CB0000EF
:10CAC000710C000041CB00001F0200004BCB0000A6
:10CAD0001108000059CB0000BD06000066CB000025
:10CAE000F104000072616E646F6D00616C6C006C2B
:10CAF0006173740066616C736500747275650025FE
:10CB00002E3135732E2E2E006D616B654C6973745A
:10CB1000006164644C6173740064656C65746500E5
:10CB20006A6F696E00636F707946726F6D546F0043
:10CB300066696E64006A6F696E537472696E6773BA
:10CB400000756E69636F6465417400756E69636F2B
:10CB50006465537472696E67006E657742797465B7
:10CB6000417272617900667265654D656D6F7279AB
:10CB700000000000D9CB0000D9100000DECB00007F
:10CB8000F710000019CB0000FB100000E4CB000000
:10CB9000DD100000EECB0000FF100000F7CB00001E
:10CBA0000311000001CC0000071100000CCC0000B4
:10CBB0000B11000018CC0000E110000021CC000097
:10CBC000EF1000002BCC0000E510000036CC000078
:10CBD000F310000066696C65006F70656E00636C31
:10CBE0006F736500656E644F6646696C65007265BB
:10CBF00061644C696E650072656164427974657345
:10CC000000617070656E644C696E6500617070657E
:10CC10006E6442797465730066696C6553697A6500
:10CC20000073746172744C697374006E6578744932
:10CC30006E4C6973740073797374656D496E666FB9
:10CC400000000000381300004813000062130000C9
:10CC5000E0130000181400004E14000086140000B9
:10CC6000AC140000E81400002A1500008015000034
:10CC7000C415000030160000781600009E16000053
:10CC8000D61600001C1700004217000070170000A5
:10CC90009E170000D417000058180000201900004B
:10CCA00096190000061A0000521A0000721A0000BD
:10CCB000941A0000461B00008C1B0000041C00009E
:10CCC000321C0000621C0000981C0000001D0000C7
:10CCD000801D0000C61D00000E1E0000841E000006
:10CCE000FA1E0000421F0000881F0000BE1F000047
:10CCF000042000004A20000092200000E6200000EE
:10CD00004421000082210000EC21000022220000CA
:10CD10006A220000B2220000FA2200003423000040
:10CD20007C230000C42300003025000070170000A1
:10CD3000381300002C240000381300006224000087
:10CD40008E240000C4240000F024000038130000EA
:10CD5000381300003813000038130000AA25000023
:10CD6000EC250000381300003813000032260000C4
:10CD700082260000A8260000D626000038130000F6
:10CD800038130000FA2600002A2700005A27000066
:10CD900090270000BA270000F02700001A280000A2
:10CDA000422800006A2800009A280000CA280000D3
:10CDB000F42800004C2900007C290000A62900006E
:10CDC0003813000038130000381300003813000037
:10CDD00038130000D6290000022A00002E2A000085
:10CDE0005A2A0000862A0000BC2A0000F22A00000D
:10CDF000282B00005E2B00008A2B0000B62B0000C1
:10CE0000EC2B00003813000038130000381300002A
:10CE100038130000381300003813000038130000E6
:10CE200038130000381300003813000038130000D6
:10CE3000381300003813000038130000182C0000CD
:10CE40004E2C00005B2564206974656D206C69734D
:10CE5000745D002825642062797465732900286F49
:10CE6000626A65637420747970653A2025642900CC
:10CE7000537461636B20756E646572666C6F7700C6
:10CE8000626F6F6C65616E006E756D6265720073C6
:10CE90007472696E67006C697374006279746520DE
:10CEA0006172726179000000070000000300000059
:10CEB00001CF0000712D000009CF0000212E0000DD
:10CEC00012CF0000CB2E00001BCF0000752D0000FC
:10CED00024CF0000CF2E00002CCF0000B92E000080
:10CEE0001500000001000000020000000400000026
:10CEF000050000000600000043616C6C696F7065FE
:10CF000000686173546F6E6500706C6179546F6E68
:10CF10006500686173536572766F0073657453655D
:10CF200072766F00646163496E697400646163576F
:10CF30007269746500474320746F6F6B202564200D
:10CF400075736563733B2066726565202564207781
:10CF50006F726473003C496E74656765723E003C95
:10CF60004C6973743E003C4F626A6563743E003CDA
:10CF70004279746541727261793E000D0A564D2006
:10CF800050616E69633A2025730D0A006D69736301
:10CF900000000000C9CF0000953B0000D2CF000088
:10CFA000253B0000D6CF0000793A0000DECF00001C
:10CFB0001F3A0000E8CF0000B5390000F4CF0000B0
:10CFC000B73800006E756C6C00686578546F496EF8
:10CFD000740073696E006A736F6E476574006A73DC
:10CFE0006F6E436F756E74006A736F6E56616C7509
:10CFF000654174006A736F6E4B657941740000007F
:10D000005CD00000013C000064D00000053C000042
:10D010006ED00000233C000077D000002D3C0000C3
:10D0200082D00000373C00008ED00000413C000060
:10D03000A3D000004B3C0000B8D00000553C0000DD
:10D04000C4D000005F3C0000D4D000000F3C0000C2
:10D05000E0D00000193C00006E65740068617357F1
:10D060006946690073746172745769466900737424
:10D070006F705769466900776966695374617475A2
:10D0800073006D794950416464726573730068740C
:10D090007470536572766572476574526571756513
:10D0A000737400726573706F6E64546F487474703B
:10D0B000526571756573740068747470436F6E6E39
:10D0C00065637400687474704973436F6E6E656352
:10D0D000746564006874747052657175657374006A
:10D0E00068747470526573706F6E7365000D0E0F07
:10D0F00004050C0B0A0607080900000000000808D8
:10D100000800080A4A4000000A5FEA5FEA0ED92ECA
:10D11000D36E19324489330C924C924D08080000AA
:10D120000004880808040804848488000A448A40AB
:10D1300000048EC480000000048800000EC00000BF
:10D140000000080001224488100C9252524C048CBA
:10D1500084848E1C824C901E1EC244924C06CA527D
:10D160005FE21FF01EC13E02448ED12E1FE24488B2
:10D17000100ED12ED12E0ED12EC48800080008002A
:10D1800000048004880244880482000EC00EC00897
:10D19000048244880ED126C0040ED135B36C0C92A3
:10D1A0005ED2521C925C925C0ED010100E1C9252F9
:10D1B000525C1ED01C901E1ED01C90100ED01371FD
:10D1C0002E12525ED2521C8808081C1FE242524C9A
:10D1D0001254981492101010101E113B75B1311199
:10D1E0003935B3710C9252524C1C925C90100C92D7
:10D1F000524C861C925C92510ED00C825C1FE484CF
:10D200008484125252524C1131312A44113135BBAF
:10D210007112524C9252112A4484841EC488101EEA
:10D220000EC808080E10080482410EC242424E0485
:10D230008A400000000000001F0804800000000E6B
:10D24000D2524F10101C925C000ED0100E02424EB3
:10D25000D24E0C925C900E06C81C88080ED24EC2AC
:10D260004C10101C92520800080808024002424C60
:10D2700010149814920808080806001B75B13100B4
:10D280001C925252000C92524C001C925C90000E68
:10D29000D24EC2000ED010100006C8049808080E26
:10D2A000C807001252524F0011312A440011313583
:10D2B000BB00124C8C9200112A4498001EC4881E98
:10D2C00006C48C8486080808080818080C8818000A
:10D2D000000C83600000000001000000020000005C
:10D2E000030000000400000005000000060000002C
:10D2F0000700000008000000090000000A0000000C
:10D300000B0000000C0000000D0000000E000000EB
:10D310000F000000100000001200000014000000C8
:10D3200016000000180000001A0000001C00000099
:10D330001E00000020000000230000002600000066
:10D34000290000002C0000002F0000003200000027
:10D35000360000003A0000003E00000042000000DD
:10D36000460000004B000000500000005500000087
:10D370005A00000061000000680000006F0000001B
:10D38000760000007D000000840000008B0000009B
:10D390009200000099000000A0000000A70000001B
:10D3A000AE000000B5000000BC000000C30000009B
:10D3B000CA000000D1000000D8000000DF0000001B
:10D3C000E6000000ED000000F4000000FB0000009B
:10D3D000FF00000024D40000813C00002FD4000096
:10D3E000D141000039D400003D3E000046D4000089
:10D3F000414000004DD400009140000056D4000090
:10D40000E140000062D40000D93F000073D4000066
:10D41000AD3E000080D40000693F00006469737075
:10D420006C6179006C696768744C6576656C006D39
:10D4300062446973706C6179006D62446973706CE9
:10D4400061794F6666006D62506C6F74006D625555
:10D450006E706C6F74006D624472617753686170B6
:10D4600065006D625368617065466F724C657474D7
:10D470006572006E656F506978656C53656E640007
:10D480006E656F506978656C53657450696E004EB7
:10D490006F7420656E6F75676820726F6F6D2065A1
:10D4A00076656E20616674657220636F6D7061636E
:10D4B00074696F6E00436F6D7061637465642046BC
:10D4C0006C61736820636F64652073746F72650AA2
:10D4D000256420627974657320757365642028253E
:10D4E00064252529206F662025640042616420722E
:10D4F00065636F726420666F756E6420647572690F
:10D500006E6720696E697469616C697A6174696FAC
:10D510006E0025642025642025642028256420775A
:10D520006F72647329002564207265636F7264737F
:10D530002C20256420776F7264732C206D617849EC
:10D54000442025642C20636F6D70616374696F6E75
:10D55000206379636C657320256400526573746F72
:10D56000726564202564207363726970747300535C
:10D5700074617274656400726164696F0000000018
:10D5800010D60000A14B00001DD600003D4E00004B
:10D590002DD60000BD4D00003BD60000D14F00004D
:10D5A00046D60000C94B000056D60000514C000082
:10D5B0006AD60000394C000079D60000B351000053
:10D5C00085D60000315100008ED60000D5500000F5
:10D5D00099D600001D500000A4D60000595000004C
:10D5E000ADD600008D500000B6D60000D94B00002B
:10D5F000C5D60000B94B0000CED60000E94B0000B4
:10D600006E6F6E65006F746865720070616972009C
:10D6100064697361626C65526164696F006D657302
:10D6200073616765526563656976656400706163FF
:10D630006B657452656365697665007061636B65DF
:10D640007453656E64007265636569766564496EDE
:10D6500074656765720072656365697665644D65BA
:10D660007373616765547970650072656365697687
:10D670006564537472696E670073656E64496E7495
:10D68000656765720073656E6450616972007365E9
:10D690006E64537472696E67007365744368616E7B
:10D6A0006E656C0073657447726F75700073657496
:10D6B000506F776572007369676E616C5374726541
:10D6C0006E677468006465766963654944006C61DF
:10D6D00073744D657373616765494400556E6B6E75
:10D6E0006F776E207072696D6974697665205B254D
:10D6F000733A25735D000000000000009630077744
:10D700002C610EEEBA51099919C46D078FF46A7035
:10D7100035A563E9A395649E3288DB0EA4B8DC7955
:10D720001EE9D5E088D9D2972B4CB609BD7CB17ED5
:10D73000072DB8E7911DBF906410B71DF220B06AA5
:10D740004871B9F3DE41BE847DD4DA1AEBE4DD6DB5
:10D7500051B5D4F4C785D38356986C13C0A86B64B5
:10D760007AF962FDECC9658A4F5C0114D96C0663D5
:10D77000633D0FFAF50D088DC8206E3B5E10694CB5
:10D78000E44160D5727167A2D1E4033C47D4044BF5
:10D79000FD850DD26BB50AA5FAA8B5356C98B242D5
:10D7A000D6C9BBDB40F9BCACE36CD832755CDF4555
:10D7B000CF0DD6DC593DD1ABAC30D9263A00DE5185
:10D7C0008051D7C81661D0BFB5F4B42123C4B35675
:10D7D0009995BACF0FA5BDB89EB802280888055FF5
:10D7E000B2D90CC624E90BB1877C6F2F114C685855
:10D7F000AB1D61C13D2D66B69041DC760671DB0143
:10D80000BC20D2982A10D5EF8985B1711FB5B60614
:10D81000A5E4BF9F33D4B8E8A2C9077834F9000F54
:10D820008EA8099618980EE1BB0D6A7F2D3D6D08F4
:10D83000976C6491015C63E6F4516B6B62616C1CE4
:10D84000D83065854E0062F2ED95066C7BA5011B14
:10D85000C1F4088257C40FF5C6D9B06550E9B712B4
:10D86000EAB8BE8B7C88B9FCDF1DDD62492DDA1574
:10D87000F37CD38C654CD4FB5861B24DCE51B53A94
:10D880007400BCA3E230BBD441A5DF4AD795D83D94
:10D890006DC4D1A4FBF4D6D36AE96943FCD96E34D4
:10D8A000468867ADD0B860DA732D0444E51D0333B4
:10D8B0005F4C0AAAC97C0DDD3C710550AA410227C4
:10D8C00010100BBE86200CC925B56857B3856F2094
:10D8D00009D466B99FE461CE0EF9DE5E98C9D929F4
:10D8E0002298D0B0B4A8D7C7173DB359810DB42E34
:10D8F0003B5CBDB7AD6CBAC02083B8EDB6B3BF9A80
:10D900000CE2B6039AD2B1743947D5EAAF77D29D0B
:10D910001526DB048316DC73120B63E3843B6494EB
:10D920003E6A6D0DA85A6A7A0BCF0EE49DFF0993EB
:10D9300027AE000AB19E077D44930FF0D2A308875B
:10D9400068F2011EFEC206695D5762F7CB6765800B
:10D9500071366C19E7066B6E761BD4FEE02BD3890B
:10D960005A7ADA10CC4ADD676FDFB9F9F9EFBE8E6B
:10D9700043BEB717D58EB060E8A3D6D67E93D1A1AB
:10D98000C4C2D83852F2DF4FF167BBD16757BCA68B
:10D99000DD06B53F4B36B248DA2B0DD84C1B0AAF2B
:10D9A000F64A0336607A0441C3EF60DF55DF67A8AB
:10D9B000EF8E6E3179BE69468CB361CB1A8366BC3B
:10D9C000A0D26F2536E2685295770CCC03470BBB8B
:10D9D000B91602222F260555BE3BBAC5280BBDB28B
:10D9E000925AB42B046AB35CA7FFD7C231CFD0B52B
:10D9F0008B9ED92C1DAEDE5BB0C2649B26F263EC1D
:10DA00009CA36A750A936D02A906099C3F360EEB2A
:10DA10008567077213570005824ABF95147AB8E2EA
:10DA2000AE2BB17B381BB60C9B8ED2920DBED5E5CA
:10DA3000B7EFDC7C21DFDB0BD4D2D38642E2D4F11A
:10DA4000F8B3DD686E83DA1FCD16BE815B26B9F6AA
:10DA5000E177B06F7747B718E65A0888706A0FFF0A
:10DA6000CA3B06665C0B0111FF9E658F69AE62F8CA
:10DA7000D3FF6B6145CF6C1678E20AA0EED20DD7CA
:10DA80005483044EC2B30339612667A7F71660D0EA
:10DA90004D476949DB776E3E4A6AD1AEDC5AD6D92A
:10DAA000660BDF40F03BD83753AEBCA9C59EBBDE4A
:10DAB0007FCFB247E9FFB5301CF2BDBD8AC2BACAFA
:10DAC0003093B353A6A3B4240536D0BA9306D7CD6A
:10DAD0002957DE54BF67D9232E7A66B3B84A61C48A
:10DAE000021B685D942B6F2A37BE0BB4A18E0CC34A
:10DAF0001BDF055A8DEF022D416C6C207461736B36
:10DB0000732073746F70706564007630383600204F
:10DB10002573202573004D656D6F727920636C65E8
:10DB200061726564004E6F20667265652074617372
:10DB30006B20656E747269657300000084DB000001
:10DB40002D65000091DB0000856400009DDB000076
:10DB500055640000A3DB000065640000A9DB000041
:10DB600075640000AFDB000079610000B9DB0000E4
:10DB7000A1640000C1DB0000A562000073656E7344
:10DB80006F727300616363656C65726174696F6E57
:10DB90000074656D70657261747572650074696C8E
:10DBA00074580074696C74590074696C745A007408
:10DBB0006F756368526561640069326352656164C0
:10DBC00000693263577269746500000040DC000030
:10DBD000E56500004EDC0000E965000057DC000050
:10DBE000F565000061DC0000F96500006ADC0000FA
:10DBF000FD6500006FDC00000166000074DC0000C1
:10DC00000566000080DC00000966000087DC00007B
:10DC10000D66000090DC00001166000095DC00003D
:10DC200015660000A0DC000019660000AADC0000F8
:10DC3000ED650000B4DC0000F1650000746674005E
:10DC4000656E61626C65446973706C6179006765CB
:10DC500074576964746800676574486569676874B7
:10DC600000736574506978656C006C696E6500724C
:10DC700065637400726F756E6465645265637400E9
:10DC8000636972636C6500747269616E676C6500CC
:10DC90007465787400746674546F756368656400A5
:10DCA000746674546F7563685800746674546F7545
:10DCB00063685900746674546F7563685072657355
:10DCC000737572650076617273000000ECDC000011
:10DCD000A96A0000F6DC0000896A0000FFDC000091
:10DCE000656A00000BDD0000F16900007661724595
:10DCF0007869737473007661724E616D6564007348
:10DD000065745661724E616D6564007661724E6134
:10DD10006D65466F72496E6465780057656C636F18
:10DD20006D6520746F204D6963726F426C6F636B19
:10DD3000732100705F73706920213D204E554C4C5B
:10DD4000002F686F6D652F6769742F2E706C61747A
:10DD5000666F726D696F2F7061636B616765732F9A
:10DD60006672616D65776F726B2D61726475696E35
:10DD70006F6E6F726469636E7266352F6C69627262
:10DD800061726965732F5350492F5350492E637048
:10DD90007000535049436C6173733A3A535049438E
:10DDA0006C617373284E52465F5350495F547970CB
:10DDB000652A2C2075696E74385F742C2075696E25
:10DDC00074385F742C2075696E74385F7429000094
:10DDD0000000000000000000B56C0000716C000045
:10DDE000976C0000A16C0000AB6C0000956C00000B
:10DDF000000000000100000002000000160000000A
:10DE000004000000050000000600000007000000FC
:10DE100008000000090000000A0000000B000000DC
:10DE20000C0000000D0000000E0000000F000000BC
:10DE30001A0000001B000000140000001300000086
:10DE40001100000003000000100000001C00000092
:10DE50001D0000001E000000120000001500000060
:10DE6000170000001800000019000000000000006A
:10DE7000000000006571000095780000E571000069
:10DE8000F9710000EF710000617100005571000030
:10DE90000572000081710000517100000000000057
:10DEA000000000000000304300000000000030C30C
:10DEB0007371727400000000FB21F93FFB210940DF
:10DEC0007CD91240FB2119407A6A1F407CD922403C
:10DED000BBFD2540FB2129403A462C407A6A2F4061
:10DEE0005C4731407CD932409C6B3440BBFD3540AF
:10DEF000DB8F3740FB2139401BB43A403A463C4067
:10DF00005AD83D407A6A3F404C7E40405C47414091
:10DF10006C1042407CD942408CA243409C6B4440F0
:10DF2000AC344540BBFD4540CBC64640DB8F474047
:10DF3000EB584840FB21494083F9A200444E6E0053
:10DF4000FC291500D1572700DD34F50062DBC00045
:10DF50003C999500419043006351FE00BBDEAB004D
:10DF6000B761C5003A6E2400D24D42004906E00078
:10DF700009EA2E001C92D100EB1DFE0029B11C0005
:10DF8000E83EA700F535820044BB2E009CE98400E2
:10DF9000B4267000417E5F00D6913900538339006A
:10DFA0009CF439008B5F840028F9BD00F81F3B000A
:10DFB000DEFF97000F980500112FEF000A5A8B0023
:10DFC0006D1F6D00CF7E360009CB2700464FB7008E
:10DFD0009E663F002DEA5F00BA277500E5EBC7009B
:10DFE0003D7BF100F739070092528A00FB6BEA0093
:10DFF0001FB15F00085D8D00300356007BFC4600BA
:10E00000F0AB6B0020BCCF0036F49A00E3A91D00F2
:10E010005E619100081BE60085996500A0145F0011
:10E020008D40680080D8FF0027734D000606310040
:10E03000CA561500C9A873007BE260006B8CC00053
:10E0400000000040FB21F93F000000002D44743E19
:10E05000000000809846F83C0000006051CC783BFE
:10E0600000000080831BF0390000004020257A3832
:10E07000000000802282E336000000001DF36935B5
:10E080000200000003000000040000000600000081
:10E090008C950000369500003695000064960000CF
:10E0A00032950000329500005A96000064960000F8
:10E0B000329500005A9600003295000064960000E8
:10E0C0006896000068960000689600007096000050
:10E0D00068A00000DA9E00001E9F0000829E0000E3
:10E0E0001E9F00000EA000001E9F0000829E0000E8
:10E0F000DA9E0000DA9E00000EA00000829E000062
:10E100007A9E00007A9E00007A9E00001CA000000B
:10E1100090A7000092A6000092A60000B0A90000FF
:10E120008CA600008CA6000098A90000B0A90000F1
:10E130008CA6000098A900008CA60000B0A90000E1
:10E14000A6A90000A6A90000A6A90000B4A9000085
:10E150002C2066756E6374696F6E3A20006173736C
:10E16000657274696F6E2022257322206661696C66
:10E1700065643A2066696C6520222573222C206C28
:10E18000696E65202564257325730A0080000020D0
:10E19000232D302B2000686C4C0065666745464790
:10E1A0000030313233343536373839414243444513
:10E1B0004600303132333435363738396162636482
:10E1C0006566000000000000000000000000000084
:10E1D000000000000000000000000000000000003F
:10E1E000000000000000000000000000000000002F
:10E1F000000000000000000000000000000000001F
:10E20000000000000000000000000000000000000E
:10E2100000000000000000000000000000000000FE
:10E22000000000004300504F5349580000202020B8
:10E2300020202020202028282828282020202020B6
:10E240002020202020202020202020202088101086
:10E2500010101010101010101010101010040404E2
:10E2600004040404040404101010101010104141A0
:10E27000414141410101010101010101010101018E
:10E2800001010101010101011010101010104242A2
:10E29000424242420202020202020202020202025E
:10E2A00002020202020202021010101020000000FE
:10E2B000000000000000000000000000000000005E
:10E2C000000000000000000000000000000000004E
:10E2D000000000000000000000000000000000003E
:10E2E000000000000000000000000000000000002E
:10E2F000000000000000000000000000000000001E
:10E30000000000000000000000000000000000000D
:10E3100000000000000000000000000000000000FD
:10E3200000000000000000000000000000000000ED
:04E3300000000000E9
:08E33400D41DFF7F0100000071
:10E33C00FFFFFFFF4006000001000000E803DC05C2
:10E34C00DC05DC05DC050000FFFFFFFFFFFFFFFF26
:10E35C001800000019FCFFFFFFFFFFFF0200000088
:10E36C0003000000FFFFFFFF0000000001000000A1
:10E37C000000020001000000FFFFFFFF0000000092
:10E38C00020000000000040002000000FFFFFFFF7D
:10E39C000000000003000000000008000300000063
:10E3AC000A000000080000000100000080000020AE
:10E3BC0000000000E4E1000004E20000C4E1000001
:10E3CC000000000000000000000000000000000041
:10E3DC000000000000000000000000000000000031
:10E3EC000000000000000000000000000000000021
:10E3FC000000000000000000000000000000000011
:10E40C000000000000000000000000000000000000
:10E41C0043000000000000000000000000000000AD
:10E42C0000000000000000000000000000000000E0
:10E43C00430000000000000000000000000000008D
:10E44C0000000000000000000000000000000000C0
:10E45C00430000000000000000000000000000006D
:10E46C0000000000000000000000000000000000A0
:10E47C00430000000000000000000000000000004D
:10E48C000000000000000000000000000000000080
:10E49C00430000000000000000000000000000002D
:10E4AC000000000000000000000000000000000060
:10E4BC00430000000000000000000000000000000D
:10E4CC000000000000000000000000000000000040
:10E4DC0043000000000000000000000000000000ED
:10E4EC000000000000000000000000000000000020
:10E4FC00BDC80000D5C20000000000002CE20000E6
:10E50C0006CB00008BCF00008BCF00008BCF000020
:10E51C008BCF00008BCF00008BCF00008BCF000087
:10E52C008BCF00008BCF0000FFFFFFFFFFFFFFFF33
:10E53C00FFFFFFFFFFFF000001004153434949006B
:10E54C0000000000000000000000000000000000BF
:10E55C000000000000000000000041534349490046
:10E56C00000000000000000000000000000000009F
:10E57C00000000000000000000000000E9000000A6
:10E58C00416C0000896F0000B1740000C1000000F4
:040000030000702564
:00000001FF
